:1000000038060120F97100001BC30200E5710000F1
:10001000E5710000E5710000E5710000E571000088
:10002000000000000000000000000000D572000089
:10003000E5710000000000005D740000E571000043
:10004000F9740000F9740000F9740000F9740000FC
:10005000F9740000F9740000F9740000F9740000EC
:10006000F9740000F9740000F9740000F9740000DC
:10007000F9740000F9740000F9740000F9740000CC
:1004800081F0004102E000BF83F0004330B54FEA45
:1004900041044FEA430594EA050F08BF90EA020FB2
:1004A0001FBF54EA000C55EA020C7FEA645C7FEA45
:1004B000655C00F0E2804FEA5454D4EB5555B8BF68
:1004C0006D420CDD2C4480EA020281EA030382EAD9
:1004D000000083EA010180EA020281EA0303362D6B
:1004E00088BF30BD11F0004F4FEA01314FF4801C3E
:1004F0004CEA113102D0404261EB410113F0004F50
:100500004FEA03334CEA133302D0524263EB430306
:1005100094EA050F00F0A780A4F10104D5F1200EA4
:100520000DDB02FA0EFC22FA05F2801841F10001FF
:1005300003FA0EF2801843FA05F359410EE0A5F1D3
:1005400020050EF1200E012A03FA0EFC28BF4CF004
:10055000020C43FA05F3C01851EBE37101F00045BA
:1005600007D54FF0000EDCF1000C7EEB00006EEBC7
:100570000101B1F5801F1BD3B1F5001F0CD3490851
:100580005FEA30004FEA3C0C04F101044FEA4452A8
:1005900012F5800F80F09A80BCF1004F08BF5FEA2F
:1005A000500C50F1000041EB045141EA050130BD0F
:1005B0005FEA4C0C404141EB0101013C28BFB1F521
:1005C000801FE9D291F0000F04BF01460020B1FA6C
:1005D00081F308BF2033A3F10B03B3F120020CDA3F
:1005E0000C3208DD02F1140CC2F10C0201FA0CF01D
:1005F00021FA02F10CE002F11402D8BFC2F1200C82
:1006000001FA02F120FA0CFCDCBF41EA0C01904037
:10061000E41AA2BF01EB0451294330BD6FEA040480
:100620001F3C1CDA0C340EDC04F11404C4F120026B
:1006300020FA04F001FA02F340EA030021FA04F37D
:1006400045EA030130BDC4F10C04C4F1200220FAD4
:1006500002F001FA04F340EA0300294630BD21FA12
:1006600004F0294630BD94F0000F83F4801306BFD8
:1006700081F480110134013D4EE77FEA645C18BFCC
:100680007FEA655C29D094EA050F08BF90EA020F63
:1006900005D054EA000C04BF1946104630BD91EA5B
:1006A000030F1EBF0021002030BD5FEA545C05D15E
:1006B0004000494128BF41F0004130BD14F580049D
:1006C0003CBF01F5801130BD01F0004545F0FE4111
:1006D00041F470014FF0000030BD7FEA645C1ABF46
:1006E000194610467FEA655C1CBF0B46024650EA7D
:1006F000013406BF52EA033591EA030F41F40021A9
:1007000030BD00BF90F0000F04BF0021704730B52E
:100710004FF4806404F132044FF000054FF0000103
:1007200050E700BF90F0000F04BF0021704730B5C4
:100730004FF4806404F1320410F0004548BF404299
:100740004FF000013EE700BF42004FEAE2014FEAEE
:1007500031014FEA02701FBF12F07F4393F07F4FC9
:1007600081F06051704732F07F4208BF704793F0CC
:100770007F4F04BF41F40021704730B54FF46074DF
:1007800001F0004521F000411CE700BF50EA0102E2
:1007900008BF704730B54FF000050AE050EA01028B
:1007A00008BF704730B511F0004502D5404261EBFB
:1007B00041014FF4806404F132045FEA915C3FF43C
:1007C000D8AE4FF003025FEADC0C18BF03325FEAD9
:1007D000DC0C18BF033202EBDC02C2F1200300FA8A
:1007E00003FC20FA02F001FA03FE40EA0E0021FAAF
:1007F00002F11444BDE600BF70B54FF0FF0C4CF49D
:10080000E06C1CEA11541DBF1CEA135594EA0C0F4E
:1008100095EA0C0F00F0DEF82C4481EA030621EA89
:100820004C5123EA4C5350EA013518BF52EA0335C4
:1008300041F4801143F4801338D0A0FB02CE4FF076
:100840000005E1FB02E506F00042E0FB03E54FF0A6
:100850000006E1FB03569CF0000F18BF4EF0010E9E
:10086000A4F1FF04B6F5007F64F5407404D25FEA9A
:100870004E0E6D4146EB060642EAC62141EA55514D
:100880004FEAC52040EA5E504FEACE2EB4F1FD0C8F
:1008900088BFBCF5E06F1ED8BEF1004F08BF5FEA0D
:1008A000500E50F1000041EB045170BD06F00046BF
:1008B00046EA010140EA020081EA0301B4EB5C046C
:1008C000C2BFD4EB0C0541EA045170BD41F4801164
:1008D0004FF0000E013C00F3AB8014F1360FDEBF89
:1008E000002001F0004170BDC4F10004203C35DA65
:1008F0000C341BDC04F11404C4F1200500FA05F3E8
:1009000020FA04F001FA05F240EA020001F0004288
:1009100021F0004110EBD37021FA04F642EB0601FE
:100920005EEA430E08BF20EAD37070BDC4F10C0428
:10093000C4F1200500FA04F320FA05F001FA04F2EC
:1009400040EA020001F0004110EBD37041F10001D8
:100950005EEA430E08BF20EAD37070BDC4F12005E3
:1009600000FA05F24EEA020E20FA04F301FA05F24B
:1009700043EA020321FA04F001F0004121FA04F2F3
:1009800020EA020000EBD3705EEA430E08BF20EAC3
:10099000D37070BD94F0000F0FD101F000464000FD
:1009A00041EB010111F4801F08BF013CF7D041EA7F
:1009B000060195F0000F18BF704703F00046520083
:1009C00043EB030313F4801F08BF013DF7D043EA54
:1009D0000603704794EA0C0F0CEA135518BF95EA0A
:1009E0000C0F0CD050EA410618BF52EA4306D1D191
:1009F00081EA030101F000414FF0000070BD50EAB0
:100A0000410606BF1046194652EA430619D094EA39
:100A10000C0F02D150EA013613D195EA0C0F05D123
:100A200052EA03361CBF104619460AD181EA030177
:100A300001F0004141F0FE4141F470014FF000002F
:100A400070BD41F0FE4141F4780170BD70B54FF0CA
:100A5000FF0C4CF4E06C1CEA11541DBF1CEA13554A
:100A600094EA0C0F95EA0C0F00F0A7F8A4EB05042C
:100A700081EA030E52EA03354FEA013100F0888023
:100A80004FEA03334FF0805545EA131343EA1263EC
:100A90004FEA022245EA111545EA10654FEA0026A1
:100AA0000EF000419D4208BF964244F1FD0404F55A
:100AB000407402D25B084FEA3202B61A65EB0305B6
:100AC0005B084FEA32024FF480104FF4002CB6EB73
:100AD000020E75EB030E22BFB61A754640EA0C00F3
:100AE0005B084FEA3202B6EB020E75EB030E22BF33
:100AF000B61A754640EA5C005B084FEA3202B6EB74
:100B0000020E75EB030E22BFB61A754640EA9C0032
:100B10005B084FEA3202B6EB020E75EB030E22BF02
:100B2000B61A754640EADC0055EA060E18D04FEAC0
:100B3000051545EA16754FEA06164FEAC30343EA60
:100B400052734FEAC2025FEA1C1CC0D111F4801F2D
:100B50000BD141EA00014FF000004FF0004CB6E726
:100B600011F4801F04BF01430020B4F1FD0C88BFC5
:100B7000BCF5E06F3FF6AFAEB5EB030C04BFB6EBD0
:100B8000020C5FEA500C50F1000041EB045170BDC3
:100B90000EF0004E4EEA113114EB5C04C2BFD4EBF0
:100BA0000C0541EA045170BD41F480114FF0000E74
:100BB000013C90E645EA060E8DE60CEA135594EAF0
:100BC0000C0F08BF95EA0C0F3FF43BAF94EA0C0FF3
:100BD0000AD150EA01347FF434AF95EA0C0F7FF468
:100BE00025AF104619462CE795EA0C0F06D152EABC
:100BF00003353FF4FDAE1046194622E750EA4106A0
:100C000018BF52EA43067FF4C5AE50EA41047FF4B0
:100C10000DAF52EA43057FF4EBAE12E74FF0FF3C15
:100C200006E000BF4FF0010C02E000BF4FF0010CE6
:100C30004DF804CD4FEA410C7FEA6C5C4FEA430C5F
:100C400018BF7FEA6C5C1BD001B050EA410C0CBFAE
:100C500052EA430C91EA030F02BF90EA020F002010
:100C6000704710F1000F91EA030F58BF994208BF77
:100C700090422CBFD8176FEAE37040F00100704734
:100C80004FEA410C7FEA6C5C02D150EA013C07D18B
:100C90004FEA430C7FEA6C5CD6D152EA033CD3D0D6
:100CA0005DF8040B704700BF8446104662468C46D0
:100CB0001946634600E000BF01B5FFF7B7FF002803
:100CC00048BF10F1000F01BD4DF808EDFFF7F4FF2C
:100CD0000CBF012000205DF808FB00BF4DF808EDB7
:100CE000FFF7EAFF34BF012000205DF808FB00BFDA
:100CF0004DF808EDFFF7E0FF94BF012000205DF8FC
:100D000008FB00BF4DF808EDFFF7CEFF94BF0120B0
:100D100000205DF808FB00BF4DF808EDFFF7C4FFA9
:100D200034BF012000205DF808FB00BF4FEA4102FC
:100D300012F5001215D211D56FF47873B3EB62522D
:100D400012D94FEAC12343F0004343EA505311F054
:100D5000004F23FA02F018BF404270474FF00000E6
:100D6000704750EA013005D111F0004008BF6FF024
:100D7000004070474FF00000704700BF4A0011D29A
:100D800012F5001211D20DD56FF47873B3EB6252E5
:100D90000ED44FEAC12343F0004343EA505323FAF1
:100DA00002F070474FF00000704750EA013002D166
:100DB0004FF0FF3070474FF0000070474FEA41029C
:100DC000B2F1E04324BFB3F5001CDCF1FE5C0DD9A9
:100DD00001F0004C4FEAC0024CEA5070B2F1004FF3
:100DE00040EB830008BF20F00100704711F0804FF6
:100DF00021D113F13872BCBF01F00040704741F4BB
:100E000080114FEA5252C2F11802C2F1200C10FABE
:100E10000CF320FA02F018BF40F001004FEAC123A2
:100E20004FEAD32303FA0CFC40EA0C0023FA02F346
:100E30004FEA4303CCE77FEA625307D150EA01331C
:100E40001EBF4FF0FE4040F44000704701F00040EC
:100E500040F0FE4040F40000704700BF80F00040CA
:100E600002E000BF81F0004142001FBF5FEA410382
:100E700092EA030F7FEA226C7FEA236C6AD04FEA82
:100E80001262D2EB1363C1BFD218414048404140C7
:100E9000B8BF5B42192B88BF704710F0004F40F479
:100EA000000020F07F4018BF404211F0004F41F495
:100EB000000121F07F4118BF494292EA030F3FD061
:100EC000A2F1010241FA03FC10EB0C00C3F1200374
:100ED00001FA03F100F0004302D5494260EB400003
:100EE000B0F5000F13D3B0F1807F06D340084FEA6E
:100EF000310102F10102FE2A51D2B1F1004F40EB63
:100F0000C25008BF20F0010040EA030070474900CA
:100F100040EB0000013A28BFB0F5000FEDD2B0FA67
:100F200080FCACF1080CB2EB0C0200FA0CF0AABF8A
:100F300000EBC25052421843BCBFD0401843704728
:100F400092F0000F81F4000106BF80F4000001322E
:100F5000013BB5E74FEA41037FEA226C18BF7FEA05
:100F6000236C21D092EA030F04D092F0000F08BF47
:100F70000846704790EA010F1CBF0020704712F02E
:100F80007F4F04D1400028BF40F00040704712F16D
:100F900000723CBF00F50000704700F0004343F0D2
:100FA000FE4040F4000070477FEA226216BF084608
:100FB0007FEA23630146420206BF5FEA412390EACB
:100FC000010F40F4800070474FF0000304E000BFC1
:100FD00010F0004348BF40425FEA000C08BF704772
:100FE00043F0964301464FF000001CE050EA010236
:100FF00008BF70474FF000030AE000BF50EA01024B
:1010000008BF704711F0004302D5404261EB410137
:101010005FEA010C02BF84460146002043F0B6435C
:1010200008BFA3F18053A3F50003BCFA8CF2083A81
:10103000A3EBC25310DB01FA02FC634400FA02FC8A
:10104000C2F12002BCF1004F20FA02F243EB020091
:1010500008BF20F00100704702F1200201FA02FCF3
:10106000C2F1200250EA4C0021FA02F243EB0200E6
:1010700008BF20EADC7070474FF0FF0C1CEAD0522A
:101080001EBF1CEAD15392EA0C0F93EA0C0F6FD0EB
:101090001A4480EA010C400218BF5FEA41211ED0C9
:1010A0004FF0006343EA501043EA5111A0FB0131B5
:1010B0000CF00040B1F5000F3EBF490041EAD3718A
:1010C0005B0040EA010062F17F02FD2A1DD8B3F106
:1010D000004F40EBC25008BF20F00100704790F075
:1010E000000F0CF0004C08BF49024CEA502040EAC7
:1010F00051207F3AC2BFD2F1FF0340EAC25070478D
:1011000040F400004FF00003013A5DDC12F1190FCA
:10111000DCBF00F000407047C2F10002410021FA3C
:1011200002F1C2F1200200FA02FC5FEA310040F154
:10113000000053EA4C0308BF20EADC70704792F0CD
:10114000000F00F0004C02BF400010F4000F013A05
:10115000F9D040EA0C0093F0000F01F0004C02BF00
:10116000490011F4000F013BF9D041EA0C018FE76F
:101170000CEAD15392EA0C0F18BF93EA0C0F0AD075
:1011800030F0004C18BF31F0004CD8D180EA01009B
:1011900000F00040704790F0000F17BF90F0004F34
:1011A000084691F0000F91F0004F14D092EA0C0F16
:1011B00001D142020FD193EA0C0F03D14B0218BFA9
:1011C000084608D180EA010000F0004040F0FE40EF
:1011D00040F40000704740F0FE4040F4400070478B
:1011E0004FF0FF0C1CEAD0521EBF1CEAD15392EA0A
:1011F0000C0F93EA0C0F69D0A2EB030280EA010CFA
:1012000049024FEA402037D04FF0805343EA111192
:1012100043EA10130CF000408B4238BF5B0042F1F0
:101220007D024FF4000C8B4224BF5B1A40EA0C0095
:10123000B3EB510F24BFA3EB510340EA5C00B3EBC7
:10124000910F24BFA3EB910340EA9C00B3EBD10FB5
:1012500024BFA3EBD10340EADC001B0118BF5FEA07
:101260001C1CE0D1FD2A3FF650AF8B4240EBC25030
:1012700008BF20F0010070470CF0004C4CEA5020F1
:101280007F32C2BFD2F1FF0340EAC250704740F440
:1012900000004FF00003013A37E792F0000F00F032
:1012A000004C02BF400010F4000F013AF9D040EAB0
:1012B0000C0093F0000F01F0004C02BF490011F444
:1012C000000F013BF9D041EA0C0195E70CEAD1533C
:1012D00092EA0C0F08D142027FF47DAF93EA0C0F23
:1012E0007FF470AF084676E793EA0C0F04D14B0207
:1012F0003FF44CAF08466EE730F0004C18BF31F0B9
:10130000004CCAD130F000427FF45CAF31F00043B2
:101310007FF43CAF5FE700BF4FF0FF3C06E000BF4B
:101320004FF0010C02E000BF4FF0010C4DF804CD6E
:101330004FEA40024FEA41037FEA226C18BF7FEA7E
:10134000236C11D001B052EA530C18BF90EA010F80
:1013500058BFB2EB030088BFC81738BF6FEAE1700F
:1013600018BF40F0010070477FEA226C02D15FEAAB
:10137000402C05D17FEA236CE4D15FEA412CE1D017
:101380005DF8040B704700BF844608466146FFE7DE
:101390000FB5FFF7C9FF002848BF10F1000F0FBDC0
:1013A0004DF808EDFFF7F4FF0CBF012000205DF8B9
:1013B00008FB00BF4DF808EDFFF7EAFF34BF01203E
:1013C00000205DF808FB00BF4DF808EDFFF7E0FFD7
:1013D00094BF012000205DF808FB00BF4DF808ED28
:1013E000FFF7D2FF94BF012000205DF808FB00BF8B
:1013F0004DF808EDFFF7C8FF34BF012000205DF86D
:1014000008FB00BF4FEA4002B2F1FE4F0FD34FF08E
:101410009E03B3EB12620DD94FEA002343F0004361
:1014200010F0004F23FA02F018BF404270474FF00F
:101430000000704712F1610F01D1420205D110F096
:10144000004008BF6FF0004070474FF00000704749
:101450007BB972B90029BEBF00204FF0004106E001
:1014600008BF00281CBF6FF000414FF0FF3000F0B4
:1014700057B8ADF1080C6DE904CE002909DB002B4B
:101480001ADB00F069F8DDF804E0DDE9022304B0BE
:101490007047404261EB4101002B1BDB00F05CF820
:1014A000DDF804E0DDE9022304B0404261EB4101D4
:1014B000524263EB43037047524263EB430300F035
:1014C0004BF8DDF804E0DDE9022304B0404261EBB3
:1014D00041017047524263EB430300F03DF8DDF8F1
:1014E00004E0DDE9022304B0524263EB430370479A
:1014F00053B94AB9002908BF00281CBF4FF0FF317B
:101500004FF0FF3000F00CB8ADF1080C6DE904CEDF
:1015100000F022F8DDF804E0DDE9022304B07047B2
:10152000704700BF10F8012B11F8013B012A28BFBA
:101530009A42F7D0D01A7047034611F8012B03F8EE
:10154000012B002AF9D17047034613F8012B002A1A
:10155000FBD1181A013870472DE9F0478C468E46AA
:10156000089E154604461946002B40F0D08072456F
:1015700047D9B2FA82F74FB1C7F120030EFA07FC40
:10158000BD40BC4020FA03F343EA0C0C4FEA154E71
:10159000A8B2230CBCFBFEF80EFB18CC08FB00F92C
:1015A00043EA0C43994528D9EB1808F1FF3204D2DD
:1015B000994502D9A8F102022B44A3EB0903A4B276
:1015C000B3FBFEFC0EFB1C330CFB00F044EA0344AF
:1015D000A04214D92C190CF1FF3304D2A04202D935
:1015E000ACF102032C44241A43EA02401EB1FC4031
:1015F000002334607360BDE8F0874246DDE7634650
:10160000F1E7002A79D0B2FA82F3002B3FD01946D5
:10161000C1F1200302FA01F500FA01F42EFA03F2F7
:101620000EFA01FE20FA03F3AFB243EA0E034FEACB
:10163000154EB2FBFEFC0EFB1C201A0C0CFB07F82F
:1016400042EA004290455AD9AA180CF1FF3004D260
:10165000904502D9ACF102002A44A2EB08029BB2E9
:10166000B2FBFEFC0EFB1C220CFB07F743EA024315
:101670009F4246D9EB180CF1FF3204D29F4202D9A7
:10168000ACF102022B44DB1B42EA004202E0AEEB6B
:10169000020301224FEA154EAFB2200CB3FBFEFC51
:1016A0000EFB1C330CFB07F840EA034398452AD98C
:1016B000EB180CF1FF3004D2984502D9ACF10200CE
:1016C0002B44A3EB0803A4B2B3FBFEFC0EFB1C33BC
:1016D0000CFB07F744EA0344A74216D92C190CF176
:1016E000FF3304D2A74202D9ACF102032C44E41B1D
:1016F00043EA00400F46114678E71F2188E760461D
:10170000ABE76246BFE76046DBE76346EFE773455A
:1017100006D916B9002108466DE7C6E9000EF9E7BB
:10172000B3FA83F787B9734501D3824207D8841A85
:101730006EEB030301209C461EB900215BE738468F
:10174000FAE7C6E9004CF8E7C7F1200CBB4000FA05
:1017500007F422FA0CF520FA0CF1BA401D432EFAD8
:101760000CF30EFA07FE4FEA154941EA0E011FFA83
:1017700085FEB3FBF9F809FB18300B0C08FB0EFAD9
:1017800043EA00439A4540D9EB1808F1FF3004D2F0
:101790009A4502D9A8F102002B44A3EB0A0389B2AF
:1017A000B3FBF9F809FB183308FB0EFE41EA0341CD
:1017B0008E452CD9691808F1FF3304D28E4502D921
:1017C000A8F10203294443EA0040A1EB0E01A0FB6B
:1017D00002984145CE46434602D306D14C4504D239
:1017E0000138B9EB020E68EB0503002EA5D0B4EB6F
:1017F0000E0261EB030101FA0CFC22FA07F3F94037
:101800004CEA0303C6E9003197E74046C5E7434683
:10181000D9E70000000000002DE9F04704460F461C
:1018200016468AB038F06DFB4FF47A75A0FB050CB4
:1018300047F6122205FB01C10023FFF759FE012FD5
:1018400080460D4608D1CDE90001294A08212046ED
:1018500029F025FE002012E0766826483146FFF781
:1018600061FE78B131462448FFF75CFE50B1204656
:1018700033460121214A29F012FE6FF004000AB01C
:10188000BDE8F087404618A3D3E900232946FFF7B7
:10189000DFFD06460D4610461946194A0023FFF79C
:1018A000D7FD80460F46104619464EF660220023AB
:1018B000FFF7CEFD82468946104619464FF47A72EC
:1018C0000023FFF7C5FDCDE904A9CDE90601CDE967
:1018D000082308212046CDE90287CDE90065094AA1
:1018E00029F0DDFDB6E700BF005C26050000000022
:1018F0008CF303009DF30300A0F30300A9F303009E
:1019000080EE3600C1F303002DE9F04F914691B00F
:10191000DFF834A198469DF868304F2204460F4600
:1019200048465146099336F006F9DFF820B10546DE
:1019300013225946404636F0FEF81822064600218A
:101940000AA838F047FD002D08DA4B46404A01212D
:10195000204629F0A4FD11B0BDE8F08F002E02DA78
:1019600043463C4AF3E7A9B2B2B2BB68D3F804805D
:10197000B8F1000F15D038460AABC047A0B110F13E
:10198000160F02D1099B002BE5D05BF826300190A1
:101990000093012120465AF825302F4A29F07FFD77
:1019A000D9E76FF05700F0E70F98FEF7BBFE24A3CE
:1019B000D3E90023FFF74AF880460E988946FEF7E0
:1019C000B1FE02460B4640464946FEF75FFDCDE9B3
:1019D00006010D98FEF7A6FE19A3D3E90023FFF731
:1019E00035F880460C988946FEF79CFE02460B4669
:1019F00040464946FEF74AFDCDE904010B98FEF743
:101A000091FE0FA3D3E90023FFF720F880460A9840
:101A10008946FEF787FE02460B4640464946FEF7DA
:101A200035FD5BF82630CDE9020101935AF82530E7
:101A30000821009320463B68084A29F030FD8AE7D8
:101A40000000000080842E4164EB030018EB0300CB
:101A50008C860400A2860400A4870400D1870400B9
:101A60002DE9F04F0028D3B01791119307DA012127
:101A7000344A586853B0BDE8F04F29F010BD119BAF
:101A8000186883685B69002B37D12F4B1F930024A4
:101A90002E4D2F4E1F9BDB680BB10E2C3DD14FF00E
:101AA000000B2C4B139300221FFA8BF31FFA8BF1C0
:101AB00014931F9BADF88010ADF8822021925B68D3
:101AC000209823AA22A9984770B9229B802B40F224
:101AD00082828022CDE90132009011985B4601217B
:101AE0001D4A406829F0DBFC139B0BF1010B04330A
:101AF000BBF14E0F1393D6D10CE01FA998470028D5
:101B0000C5D0119B11981B6801211B68134A4068BE
:101B100029F0C5FC53B0BDE8F08F1798A1B29847E3
:101B200068B10C236343EB581198002B08BF334670
:101B30000093082123460A4A406829F0B0FC01348A
:101B4000A8E700BFBC890400A0EC030070EA030012
:101B50008465040064EB0300058A0400C98904005D
:101B6000E989040025462646A146A046A246274606
:101B70003822214624A8219438F02CFC149BCDE96E
:101B80001A4423F00403CDE918449BB21094169331
:101B90001F9B17989B6821AA9C46149BADF8803028
:101BA000159BADF8823032AB009320990123E047BA
:101BB000002800F3F480119BBBF10F0F5B681593B5
:101BC000BDF84830169300F0648100F23B81149B0D
:101BD00023F00403032B03D0BBF10B0F40F09A81D9
:101BE000109B2246CDE93237012340465146ADF8DD
:101BF000D030E3178DF8D850FFF77AFC22468046A4
:101C000049463790E3173046FFF722FC22468146CB
:101C10003890E317DDE91801FFF71AFC22463990E6
:101C2000E3170646DDE91A01FFF712FC139BB44ADD
:101C30001B6882461A93109B3A9018EB030847F1F1
:101C400000031D93AF4B32EA290228BF1A46B9F1AF
:101C5000000FB8BFC9F10009002D109280F2F58085
:101C60006B4229FA03F900234FEAD97242EA43038F
:101C7000002129F000401B93FEF788FD9CA3D3E9C7
:101C80000023FEF7B9FD9CA3D3E90023FEF7DEFE97
:101C9000FFF774F89A4A9B4B1C9032EA260228BF41
:101CA0001A46002EB8BF7642002D189280F2D980D5
:101CB0006B42DE400023F70F26F00040002147EA88
:101CC0004307FEF763FD8AA3D3E90023FEF794FDE3
:101CD00089A3D3E90023FEF7B9FEFFF74FF8884A3E
:101CE000884B064632EA2A0228BF1A46BAF1000F8C
:101CF000B8BFCAF1000A002D199280F2BD804FF0E2
:101D000000096B422AFA03FA00212AF00040FEF78C
:101D10003DFD77A3D3E90023FEF76EFD76A3D3E95B
:101D20000023FEF793FEFFF729F84FEADA7343EA40
:101D300049030D93199B0E90CDE90B63189B082165
:101D400009931C9BCDE9025408931B9B6E4A079391
:101D5000109B159806931D9B0A970593169BCDF82B
:101D6000108001931A9B00935B4629F098FB129B0D
:101D700001331293BDF84830149A1593ADF88020C2
:101D8000159A1F9BADF882201B68209917980DF1BA
:101D90007A029847044600283FF4E4AEA4E6BBF17B
:101DA0000F0F2BD027D8169B032B02D0BBF10B0FA4
:101DB00037D114B9329B339F1093379B189A13EB8A
:101DC00008039846389B4AF1000A9E1949EBE379CB
:101DD000399B9DF9D8509A181892199A42EBE373DF
:101DE00019931A9A3A9B9A181A921B9A42EBE37328
:101DF0001B930134CCE6BBF1340FD9E714B9329B05
:101E0000339F1093369B13EB080398469DF8DC3004
:101E10004AF1000A03F001039B191E4649F100092B
:101E2000E7E714B9329B339F1093379B9DF9D85045
:101E300013EB08039846389B4AF1000A9E1949EBB8
:101E4000E379D6E7BBF1340FC8E6A5F12003C5F16D
:101E5000200209FA03F329FA02F2134309FA05F9F9
:101E600002E7A5F12003C5F1200206FA03F326FAE2
:101E700002F21343AE401EE7A5F12009C5F120038D
:101E80000AFA09F92AFA03F349EA03090AFA05FAF0
:101E90003AE7109B2246CDE9323701234046ADF8A0
:101EA000D0305146E317FFF723FB22463690E31765
:101EB000054649463046FFF7CBFA9DF8DC3000F086
:101EC000010060F300038DF8DC30109B0690ED18E4
:101ED000169B47F1000701930C4B08210093CDE9B5
:101EE00004575B460A4A1598029429F0D8FA3EE74F
:101EF0000000000080842E410000C0FFFFFFDF4192
:101F0000EC670400DCFC0300598A04000A8B04001F
:101F1000BF8A0400109B2246CDE932370123404698
:101F2000ADF8D0305146E3178DF8D850FFF7E0FAFE
:101F30008046224649463790E3173046FFF788FA35
:101F4000139B2B4A1B6880EAE0761893109B38900D
:101F500018EB0308274B47F1000732EA200928BF96
:101F60009946002DA6EBE07629DA4FF0000A6B4285
:101F7000DE4026F000400021FEF708FC18A3D3E95C
:101F80000023FEF739FC18A3D3E90023FEF75EFD1A
:101F9000FEF7F4FE169BF60F0193189B46EA4A06DD
:101FA0000890009308215B46CDE90696CDE90487A9
:101FB000CDE90254104A159829F071FAD7E6A5F137
:101FC000200AC5F1200306FA0AFA26FA03F34AEAC0
:101FD000030AAE40CDE71290CCE600BFAFF300801D
:101FE0000000000080842E410000C0FFFFFFDF41A1
:101FF000EC670400DCFC03000F8B04000000000011
:102000002DE9F04721F00042B34F88B00446BA42B0
:102010000D464FEAD17632D9B04FBA4212D9C1F348
:1020200013030246034305D00B46FEF72FFA04467E
:102030000D4602E0002E40F01F812046294608B0E0
:10204000BDE8F0878EA3D3E90023FEF765FE0746BF
:1020500028B1002008B0BDE8F04727F05DBA8AA398
:10206000D3E9002320462946FEF738FE002800F079
:102070008580384608B0BDE8F04738F075BB984B0E
:102080009A4240F2A780974B9A4277D8964BF40039
:1020900086F0010A03EBC603AAEB060AD3E9002384
:1020A000FEF7F2F9914B804689462344D3E9003488
:1020B000CDE90034DDE9002340464946FEF7E4F966
:1020C00004460D4622462B4620462946FEF794FB41
:1020D00006460F466EA3D3E90023FEF78DFB6EA3E1
:1020E000D3E90023FEF7D0F932463B46FEF784FBE6
:1020F0006BA3D3E90023FEF7C9F932463B46FEF74E
:102100007BFB69A3D3E90023FEF7BEF932463B46C9
:10211000FEF772FB66A3D3E90023FEF7B7F9324658
:102120003B46FEF769FB02460B4620462946FEF772
:10213000ABF902460B4606460F4620462946FEF7F7
:102140005BFBCDE90201BAF1000F5AD100224FF03A
:10215000804330463946FEF797F902460B46DDE9E3
:102160000201FEF773FC22462B46FEF78DF902466C
:102170000B4600205E49FEF787F958E75D4B204685
:10218000294603EBC6064CA3D3E90023FEF734FB34
:10219000D6E90023FEF77AF9FEF7C8FD8246FEF77E
:1021A000C1FA06460F4646A3D3E90023FEF724FBF7
:1021B00002460B4620462946FEF766F980468946C8
:1021C0003046394640A3D3E90023FEF715FBCDE99D
:1021D00000016FE7484B9A420ED83DA3D3E9002394
:1021E000FEF754F90022424BFEF796FD38B100226B
:1021F0003F4B2046294618E74FF0000A62E7824627
:1022000060E732463B4600204FF08041FEF73CF944
:1022100002460B46DDE90201FEF718FC02460B46BA
:10222000DDE90001FEF730F942464B46FEF72CF996
:1022300002460B4600202E49FEF726F90B460C46B7
:102240006FF47F7102468A4508DBCDE90423DDE99E
:10225000042304EB0A5314461D46EEE60AF57A7A87
:10226000CDE906230022DDE9060103EB0A514FF018
:10227000B873FEF7C1FADAE600240025DDE600BFF8
:10228000EF39FAFE422E864051302DD5104987C0D5
:10229000D0A4BE726937663EF16BD2C541BDBB3E6C
:1022A0002CDE25AF6A56113F93BDBE166CC1663F4A
:1022B0003E5555555555C53FFE822B654715F73F91
:1022C0000000E0FE422EE63F763C7935EF39EA3DEC
:1022D0009C7500883CE4377E412E8640FFFFEF7FEF
:1022E000422ED63FB1A2F03FD8C30300C8C30300BB
:1022F0000000F03FE8C30300FFFFEF3D00000000D7
:1023000030F0004201462DE9F84F034604D1012088
:10231000BDE8F84F27F00CB9002803DABDE8F84F04
:1023200027F00EB9B0F1FF4F03DBFEF79DFDBDE8CE
:10233000F88FB0F5000F35DA4FF09841FEF79CFEAC
:102340006FF018020346C3F31604DE15764B4FF008
:102350007E517F3E2344164403F4000006EBD3561F
:1023600080F07E502043FEF77DFD04F10F026F4B9D
:1023700005461340002B3ED10021FFF711F898B11C
:10238000002E00F0C8803046FEF722FE6849054660
:10239000FEF772FE044667492846FEF76DFE0146C9
:1023A0002046C2E70022CEE75DA1D1E90001FEF799
:1023B00005FD2946FEF760FE01464FF07C50FEF712
:1023C00051FD044629462846FEF756FE01462046A2
:1023D000FEF752FE04460EB921466FE03046FEF786
:1023E000F7FD07465249FEF747FE52490646384672
:1023F000FEF742FE72E04FF08041DFF83CB1FEF79D
:1024000033FD01462846A344FEF7EAFE81463046E6
:10241000FEF7DEFD494680464846FEF72DFE0146A2
:102420008246FEF729FE45490746FEF725FE444948
:10243000FEF71AFD3946FEF71FFE4249FEF714FD6E
:102440003946FEF719FE4049FEF70EFD5146FEF7EC
:1024500013FE3E4982463846FEF70EFE3C49FEF723
:1024600003FD3946FEF708FE3A49FEF7FDFC394602
:10247000FEF702FE01465046FEF7F6FCC4F5571380
:10248000074603F5227343EA0B03002B30DD4FF0C0
:102490007C512846FEF7F0FD2946FEF7EDFD01468A
:1024A00004463846FEF7E0FC4946FEF7E5FD0746E0
:1024B00046B901462046FEF7D5FC01462846FEF700
:1024C000D1FC34E71A494046FEF7D6FD19490646C5
:1024D0004046FEF7D1FD3946FEF7C6FC01462046D0
:1024E000FEF7C0FC2946FEF7BDFC01463046E6E794
:1024F00001462846FEF7B6FC4946FEF7BDFD0446F8
:10250000002E3FF469AF0A494046FEF7B5FD094980
:10251000064640466CE7002009E700BFAFF30080A5
:10252000555555555555D53F20FB4A00F0FF7F00C6
:102530008071313FD1F71737305CCFFF9788173E56
:1025400025333A3E2549923EABAA2A3F4FD01C3E46
:10255000298E633ECDCCCC3E70B50C4C4FF420227E
:102560002669A5683368092123F400733360204687
:102570002B68984733684FF400719B05204654BF81
:10258000EB682B699847002070BD00BFE0AA0300EC
:102590002DE9F0478A4600AF00297AD004680E1F63
:1025A000361BF50826F0070604EB0608B8F80230DB
:1025B00013F0010319D13848026852070DD0E946DB
:1025C00088B06A463549CDE9051A032142F8101F43
:1025D0004FF4C25101F0AAF8CD46002383F31188CD
:1025E000BFF36F8F0423184602DF2946204626F0EA
:1025F000B0FF284434F83030C01A85421AD026483B
:10260000036859070ED0E94688B06A46244BCDE9E5
:10261000053A032342F8103F00234FF4C25101F062
:1026200085F8CD46002383F31188BFF36F8F042311
:10263000184602DFB8F80230294623F00103A8F853
:102640000230204626F085FF05EB000804EBC803A6
:102650005B88DA0708D44146204626F0C3FF42468D
:102660002946204627F003F8A65BAE1B04EBC60301
:102670005B88DB0709D43146204626F0B3FF2A46A3
:102680003146204626F0F3FF35462946204626F0FF
:1026900065FFBD46BDE8F087B828002039EF03008C
:1026A00010EF03000E4A0346904202D30D4A9042B7
:1026B00011D30D4A22B1934202D30C4A93420AD35A
:1026C0000B4A52B10B48834234BF01200020934291
:1026D00038BF00207047012070471046704700BF88
:1026E000B0A803007894040000000000000000007F
:1026F00000000000000000002DE9F04F91B000AF95
:10270000164605468B46BA6E7B6351B9037890F83E
:102710000180807800EB83002844D84520D8A0EBC6
:10272000050B02F0010395F80280FB60EB78B8F12D
:10273000000F0CBF002402F00104BB620BB1930731
:1027400019D4C4B93EB159467A6B2846B0472146E0
:1027500020467A6BB04758464437BD46BDE8F08FF7
:10276000441C2046BA66FEF7EFFE0130BA6E2044E4
:102770000BF1010BD1E72B78990008EB8303BB61C8
:10278000EB18FB62BB6A79615B00BB60BB6A69687E
:1027900008EB4303202B396100F2368112F0040369
:1027A0007B6211D04FF0000A0124D14604FA08F4EC
:1027B000013CC7F830800023C7E9073302F0020369
:1027C00008F101083B603DE002F00103002B00F03E
:1027D00099804FF001097B6A09FA08F9C2461C4644
:1027E00009F1FF393B63E6E7FB6A0233FB62002E27
:1027F0005ED013F8021C386927F0EFF9002857D093
:10280000834B1B6813F0060F17D0C7F804D08AB0AB
:102810006A46804B05933B69CDE906314FF400735E
:10282000ADF820307C4B42F8103F00234FF412519A
:10283000774800F07BFFD7F804D0FB6908F1020865
:102840000133FB61FB69BA6A9342CDD32B7887F8D9
:102850003C306B78534487F83D303B6A87F83F3013
:102860003B6B87F83E30002E53D14FF0010AD7F86A
:10287000148005EB08033B63002C5AD1B9F1000F1B
:102880006FD1B869BB681844BBEB000400F0B78097
:10289000002E00F0B18021467A6B2844B047002812
:1028A000FFF65AAFA04400217A6B0846B047A9E072
:1028B000FB6A13F8013C55F82300FFF7F3FEA0B1C3
:1028C000FB683BB1012303FA08F349EA03090AF163
:1028D000010AB2E77B6A002BAFD0012303FA08F3A9
:1028E0001C433B6B01333B63A7E73B68002BE9D1FB
:1028F000032208F1FF3302FA03F31C433B6A01335E
:102900003B629AE702F0010AD1465446C7F830A06C
:1029100051E704217A6B07F13C00B0470028FFF62D
:102920001BAF7B697A6B191F281DB04700289CDA02
:1029300012E794FAA4F3B3FA83F33A6BD25C0AFA7F
:1029400003F387F83B2024EA03043EB101217A6BAC
:1029500007F13B00B0470028FFF6FEAE08F1010882
:102960008AE799FAA9F3B3FA83F33A6BD25C55F884
:1029700022A087F83B20012202FA03F329EA030987
:102980004EB101217A6B07F13B00B0470028FFF6FA
:10299000E3AEFB6ECBB90021204B08F10108BAF180
:1029A000000F08BF9A46C6B95046FEF7CDFDFB6E34
:1029B00001308044002B3FF461AF3B6F9C423EBF2F
:1029C000FB6E23F81400013458E73B6F9C42E2D2BF
:1029D000FB6E33F814100134DEE741B150467A6BD8
:1029E00089B2B0470028FFF6B7AE804446E75046AC
:1029F000FEF7AAFD411CF1E708EB0400ACE6002E4F
:102A00007FF451AF4046A7E66FF01B00A4E600BF7D
:102A1000542800206DEF03000400000166EF03005E
:102A200030B50446EFF31185202383F31288BFF3FA
:102A30006F8F044B0FCB84E80F0085F31188BFF331
:102A40006F8F30BD602E002001281FB50C4605D0C9
:102A500004281ED06FF0150004B010BD37F051FAF5
:102A600047F612220023FEF743FD4FF4FA435A4380
:102A7000C4E90001A2606846FFF7D2FF694620461C
:102A800027F0C8F818B90A4B0FCB84E80F000020D4
:102A9000E2E737F036FA47F612220023FEF728FD68
:102AA0004FF4FA435A43C4E90001A260EFE700BFC4
:102AB00000C0030001287FB50D462DD18A68184B50
:102AC0009A4229D837F01DFA47F612220023FEF762
:102AD0000FFD144B404202FB03F361EB4101CDE9D2
:102AE00000016846029300F0ABF82946684627F0DB
:102AF00091F8EFF31186202383F31288BFF36F8FD1
:102B00009DE80F00084D85E80F0086F31188BFF39C
:102B10006F8F002004B070BD6FF01500FAE700BFA2
:102B2000FFC99A3B0083FFFF602E0020014B186015
:102B3000704700BFE81C00202DE9F84340F26C7399
:102B400044690569E1170135E41841F10001022DDE
:102B50008CBF00230123E41AC76861F1000100293A
:102B6000064607F1FF374EDA6FF4C7704FF4C872AC
:102B70000023201861F10001FEF76AFC244B4FF09E
:102B80003C0E03FB0044D6E900834FEAE37C994600
:102B90006346032D024634BF09206FF00200B66879
:102BA0000544C6FB0E93A9FB0EC60EFB036640F25E
:102BB0006D1E9920A3080EFB04333B446427454354
:102BC0000520B4FBF7F40235B5FBF0F51B1B114CE7
:102BD0001CEB080CA2FB042004FB01012B4446EB78
:102BE000E87698180C4A41F1000380180B4A63F10B
:102BF0000003A0FB020102FB031110EB0C0041EBF0
:102C00000601BDE8F8834FF4C87200232046B3E7FD
:102C100070FEFFFFB13A02009405F5FF80510100FC
:102C200010B5FFF789FF0024024604F077FC0B463D
:102C3000024944501046194610BD00BF0C00000068
:102C400070B51F4B82689A4215DDD0E9001601333A
:102C500092FBF3F3012976F100054FEAE3741CDAE5
:102C6000C91844EB0604C0E90014164901FB03230C
:102C70008360012070BD002AFBDAD0E90041124ECA
:102C80009B1A0029B3FBF6F310DA01F100459C42D0
:102C900075F100050ADA0020ECE7CD439D426FF0A4
:102CA0000045A5EB0605A541DADAF4E706FB0322A9
:102CB000E41A61F10001C0E900418260D9E700BF78
:102CC000FFC99A3B003665C400CA9A3B08B500F0BC
:102CD000B7F8012200230949C0E9002241610849EF
:102CE000C0E902330A60074903610A60064A1360BB
:102CF000064A1360064A136008BD00BFEC67040073
:102D0000081D0020041D0020886500208465002027
:102D1000806500202DE9F04781468846174600F07F
:102D20008FF8C36804461BB943691A78002A3ED15C
:102D30000023E36063684B4558F8232008DB314BE0
:102D40006361204600F060F84FF0FF30BDE8F08787
:102D5000511C616192F800A0BAF12D0FEFD1951CC2
:102D6000656156782D2EA66004D1927872B9013330
:102D70006360E4E756B9234D51463846656137F044
:102D80005CFB0028DDD05646C4F808A03146384622
:102D900037F053FB3A2E00D070B92B7813B9636823
:102DA00001336360204600F02FF83F20CEE75D1C22
:102DB00045611E788660E9E743783A2B0BD0002303
:102DC00023612B7813B9636801336360204600F0F8
:102DD0001BF8A068BAE72B780A4A33B96368013355
:102DE0009945636004DD58F82350C4E90452EAE7CA
:102DF00062613D7820463A2DD5D100F005F828468D
:102E0000A4E700BFEC6704000168084A084B1160A2
:102E10004168084A11608168074A1160074AC16821
:102E2000116002691A6005F0E7BB00BF081D0020B1
:102E300080650020041D0020886500208465002036
:102E400000487047EC1C00202DE9F047858B0446B4
:102E5000280717460CD501290CBF45F0100545F091
:102E60002005A58387F31188BFF36F8FBDE8F08736
:102E7000022905F0070540F09480204627F08DFBDD
:102E8000052864D801A353F820F000BF652E000088
:102E9000A32F00004F2F0000112F00002B2F000048
:102EA0003D2F000001F007035A1F012A1FD80022FE
:102EB00021F00701062BD4F8008089B2C4E9002272
:102EC00009D1434603E0E28B0132E2831B68002B09
:102ED000F9D141F002012046A18327F05EFB4FF0BB
:102EE000000900286DD041F02001A18369E0042B86
:102EF0000AD121F0070189B22046A18327F04DFBBA
:102F000010B141F02001A1834FF00008C14658E004
:102F10002369D3F80090A38B23F0070343F0060343
:102F20004FF00008A38346464BE02369D3F8049092
:102F3000A38B23F0070343F00403F1E72369D3F8DD
:102F40000890A38B23F0070343F00503E8E74FF055
:102F50000008C146E7E7012243F00803A38387F393
:102F60001188BFF36F8F002A3BD1B8F1000F4AD10F
:102F7000B9F1000F02D020462C49C847EFF3118762
:102F8000202383F31288BFF36F8FA38B23F00803F2
:102F90009BB2A383D9063FD523F01002A28303F08E
:102FA0000705A669A18B002EBFF67CAF00239946CA
:102FB000D4F8008021F00701C4E9003341F0010199
:102FC000A183A38B03F0070AAA4502D0A268002AB6
:102FD000C1D1B8F1000F02D1B9F1000FDAD000224F
:102FE000BAE7A1680029C0D00D680029BDD03346DA
:102FF000524620464F68B8471DB12B6829461D46EA
:10300000F3E72B46FAE74146334652462046D8F8C6
:10301000008027F0EEFAA8E79A067FF523AF23F0A9
:103020002002A28303F0070527E700BF1FA60200C6
:103030002DE9F047044607464FF00109DFF84C80C0
:1030400094FAA4F5B5FA85F509FA05F32E0108EB13
:1030500005156FEA030A24EA03042B7B63B158F8D1
:1030600006301B696BB94644736803222846196809
:1030700007EA0A0727F074FC002CE1D13846BDE8C6
:10308000F087284698470028F6D1ECE768BA030095
:1030900010B5002288B00E490E4836F07AFF0022A3
:1030A00000230024CDE906230E234FF44072CDE91E
:1030B0000334CDE90144084B08490094084823F043
:1030C00053FE0849064823F005FD204608B010BD10
:1030D000E9300000483300203534000008A3002008
:1030E000702E00202CF00300014823F0B9B900BF76
:1030F0000C2C00202DE9F047804621480F4627F090
:103100000BFC0646002833D000252846BDE8F08792
:10311000237B83B12368DB680BB120469847636843
:1031200083F8069023681B69D3B96368032220469D
:10313000196827F015FC013610345445E8D3B8F16E
:10314000000FE2D0002DDFD02846FFF771FF0546C3
:10315000002FF7D0002140F2391036F0EBFCF1E7F8
:10316000204698470028E0D009FA06F31D43E2E71D
:1031700005464FF00109034CDFF80CA0DDE700BF66
:103180009C65002068BA030078BA030008B50346BE
:1031900008462BB1044A136000F046FD002008BD2C
:1031A0006FF01500FBE700BF0C1D002010B5044CAC
:1031B000237813B9034823F053F90123237010BD7A
:1031C000668000200C2C002010B50446094827F02A
:1031D000A3FB3CB1084BD3E8EF1F0139C3E8E21F62
:1031E000002AF8D1054824F0B5FCBDE81040044899
:1031F00023F036B9946500209865002048330020FC
:103200000C2C00200022044BD3E8EF0FC3E8E12F81
:103210000029F9D1704700BF9465002070B5FFF711
:10322000F1FF0546074C084EB44200D370BD6368F9
:103230005B792BB123685B6813B129462046984718
:103240001034F1E768BA030078BA030010B5044CF3
:103250000449204626F01EFE034B1C6010BD00BF33
:1032600008280020F8C303008C65002000230E4AC4
:1032700010B513700D4A0E4913600E4A0E481360C4
:10328000FFF784FFFFF7E2FF00F080F90B4B0C49DA
:1032900018468B4200D310BD1A1A5C681211013215
:1032A00022711033F5E700BF67800020946500208D
:1032B00040420F009865002015A9020068BA03007B
:1032C00078BA0300014600220023014826F003BE1D
:1032D00008280020014826F09ABE00BF08280020D8
:1032E000024B0146186826F0EDBE00BF8C65002039
:1032F000014826F022BF00BF082800202DE9F04138
:10330000354B1B78002B64D0FFF7E4FF0446002800
:103310005BD1324B324D1B68002B19DD36F0F1FDCD
:103320004FF47A76A0FB060747F61222002306FB2D
:103330000171FEF7DDF8D5E90032C01A40F2E93339
:1033400061EB0201984271F1000101D3FFF766FFC2
:10335000D5E9003213F57A7342F10002C5E9003273
:10336000002C36D0BDE8F041FFF7C2BF6B685B7937
:103370003BB121784B0713D52B68214628461B68A3
:10338000984710354545F1D32046FFF7A9FF154B67
:10339000D3E8EF1F0139C3E8E21F002AB9D0F7E7ED
:1033A00020462688C1F3C20700F09EFAC6F38216B3
:1033B0000246002EE0D00028DEDB012339462846F5
:1033C00000F08EF9B042DCD3D6E7074DDFF81C8061
:1033D000D8E70020BDE8F0816680002094650020D9
:1033E000403300209865002068BA030078BA0300D3
:1033F00070B50D4D297861B90120FFF77BFE0B4CAC
:103400000B4EB44206D3FFF779FF0028FBD101230E
:103410002B7070BD63685B791BB1236820469B6885
:1034200098471034EDE700BF6780002068BA0300BA
:1034300078BA030000212DE9F8430846FFF75AFE49
:10344000044648B340F21B684FF0000904F066F8E8
:103450001A4B1B4A1B58136033B11A4B1B68092BBC
:1034600002DD194822F0FCFF0025184F44B1204628
:10347000FFF7DEFD044618B94FF0FF384FF0FF3973
:10348000FFF73CFF064628B9B5B90F4842464B4600
:1034900023F022F83546E9E74FF0FF384FF0FF39C7
:1034A000D4E72B689B691BB1002228461146984738
:1034B0001035BD42F5D3E8E7054DFAE708000000F6
:1034C00090650020986500200C2C002078BA03003D
:1034D00068BA030013B5184827F01EFA174B1B787B
:1034E00073B1EFF31184202383F31288BFF36F8F3E
:1034F000FFF704FF84F31188BFF36F8F02B010BD94
:103500000F4B1B68002BF9D050B9002200230D4847
:10351000CDE9002347F61222002324F0F5FAEDE767
:103520000928EBD1074824F015FB074802B0BDE895
:10353000104022F095BF00BF9865002067800020F2
:1035400090650020483300200C2C002010B5064B5D
:1035500004461B6898472146A060044826F038FDC1
:10356000BDE81040FFF7B6BF0C1D00200828002062
:10357000044A054B9B1AB1EBD30F34BF52F831000C
:1035800000207047F8B8030068BA03000021084B18
:10359000084A09489B1ADB08994200D17047026823
:1035A000013122F0070242F0030240F8042BF3E756
:1035B00068BA0300F8B8030050280020F8B50646A2
:1035C00000240A4F0A4BDB1BDD08AC4203D14FF04D
:1035D000FF342046F8BD57F8340020B13146FDF7DE
:1035E000A1FF0028F5D00134EFE700BFF8B80300D1
:1035F00068BA030000282DE9F047884615461F46A3
:103600001DDA4FF0000A5446DFF89090244EA6EBE6
:1036100009063609B24509F1100902D12046BDE874
:10362000F08759F80C0C3B462A4641460079FFF7D3
:10363000E1FF844238BF04460AF1010AEAE7194B68
:10364000194AD21AB5EBD20F26D203EBC5031C7967
:10365000BC4228BF3C460722144EC0B200EB4000DB
:1036600056F82530824023EA020304F00702824024
:1036700013430021032223FA02F000F007008142E5
:1036800002F1030238BF01461E2AF4D123F00703DA
:103690000B4346F82530C1E70024DCE768BA030095
:1036A00078BA0300F8B8030068BA03005028002075
:1036B000F8B506460F460024074D084BED1AED08F5
:1036C000AC4200D3F8BD002122B23B463046013463
:1036D00027F03EF9A4B2F3E768BA0300F8B8030094
:1036E00070B14168097973B1002A17DBCBB20C497C
:1036F00003EB430351F82200D84000F00700704765
:103700004FF0FF31EFE707490748401AB2EBD00FFF
:103710003ABF01EBC2010879184670470420704790
:1037200050280020F8B8030068BA03002DE9F04FD4
:103730008FB0C1F34A2604AF0D469046B8607B6057
:103740000C0D002E65D04FF000090A234FF0040B3A
:1037500007F1140AFE60C7E90799C7F8249000939F
:10376000CDF808B0CDF804A007F11C034A46404646
:10377000F968FEF7C1FFB0F5006F034620D3294872
:10378000036813F0060F17D06C468AB0D8F80410FF
:1037900004AB254D1A46C3E9055140F2FF71D961CA
:1037A0004FF400711984214B42F8103F4FF412512D
:1037B0004B46FFF7BBFFA5462C37BD46BDE8F08F53
:1037C000C0F30A0604F11700184420F0070080082F
:1037D0003B60FFF777FD66F35325044680B13B68F5
:1037E00000F11001C7E908390A23F961CDE901ABFD
:1037F000009340460E4AF96807F11C03FEF77CFF70
:1038000066F353252A4620467B68B96827F0DCF822
:10381000D2E704F1170020F007008008FFF752FDFF
:103820000446EDE78028002041F003000400000179
:103830009BA902002DE9F04F87B00546DDE9106B2A
:10384000DDE9127A884614469946DFB110213B46DD
:103850005A460020CDF800A0CDF814A025F0E4FFD2
:10386000B0F5006F01460FD31D48036813F0060F33
:1038700032D040F2FF7302211A4A07B0BDE8F04F80
:1038800027F0FBB83946384604F0070305F0070473
:10389000E40044EA831444EA402444EA065406F16E
:1038A0001700084420F0070080080391FFF70AFD85
:1038B000054640B13FB13B465A460399CDF800A0BA
:1038C000103025F0B1FF4B4622464146284607B04E
:1038D000BDE8F04F27F078B807B0BDE8F08F00BF23
:1038E0008028002080F00300406820B1034BC01AFC
:1038F00040F38F0070474FF0FF3070475028002092
:103900000EB403B503AB53F8042B014604480193EE
:1039100004F044F802B05DF804EB03B0704700BF58
:10392000DDAA0200CA0605D48B064CBF0249034932
:10393000FFF7E6BF704700BF9EF6030013100400B8
:103940002DE9F04F8BB099469DF85880179B04469F
:1039500007930D46DDE918A31A9F06920593B8F167
:10396000000F00F0BF80844B07F0020B13F8083003
:10397000089307F48073099326F0E8FF02460028B5
:103980007DD020467D49FFF7BBFF0646BBF1000F07
:1039900008D017F0440F74D12A4620467849FFF723
:1039A000AFFF064407F0010353B1764B204653F8AE
:1039B0002820754B7549002A08BF1A46FFF7A0FF5B
:1039C00007F48073002B07F0080318BF4FF00009BD
:1039D000002B00F082806E4B204653F828206D4962
:1039E000FFF78EFF0546069B2BB11A4620466A4913
:1039F000FFF786FF0544B9F1000F0DD0089B002B9F
:103A00006ED06649664BB8F1040F18BF19464A4696
:103A10002046FFF775FF054462483544079B1BB1FC
:103A20002246614926F0A8F8059B002B00F0908003
:103A3000DDF814903946B9F1100F204628BF4FF039
:103A400010090026FFF76EFFB54252DC0026334610
:103A500020461AF803205549FFF752FF0136102E71
:103A60004DD0710703D120465149FFF749FF4E451C
:103A70003346EDD320464F49FFF742FFEEE70646B7
:103A800084E74D4B186800288BD04C4B4FF47A7B61
:103A90001B684FF03C0CB5FBF3F5B5FBF0F14FF4B0
:103AA000616300FB11550BFB05F5B1FBF3F2B5FBB0
:103AB000F0FE03FB121100FB1E55B1FBFCF30BFBE8
:103AC00005F5B5FBF0F50CFB131120460091CDE98F
:103AD00001E53B49FFF714FF63E707F0080582E7BC
:103AE0002F4994E7B9F1010F45460CBF2D483548E1
:103AF00094E720462E49FFF703FF0136A4E700268E
:103B000020463149FFF7FCFE33461AF803202046D1
:103B1000A2F120035F2B28BF2E222C49FFF7F0FED5
:103B20000136102E0DD0720703D120462049FFF731
:103B3000E7FEB1453346E8D820461D49FFF7E0FED1
:103B4000EEE7059BCA44B3EB090305937FF470AF1E
:103B5000B8F1000F0AD0FB0704D520460A4A0B49EA
:103B6000FFF7CEFE39462046FFF7DCFE20460BB0BD
:103B7000BDE8F04F26F0A5BFF49304003201040025
:103B8000C6F003000CC40300B8F0030068F903009A
:103B900020C40300ECF00300F2F00300BDF00300CA
:103BA000C1F00300DDAA02009D790000F6F00300D9
:103BB000A4420400A2420400A4650020A0650020E5
:103BC000D0F003000BAB0200FCF003001601040070
:103BD00042F20F7373B58B4228BF0B46056804464B
:103BE000052168460D4A24F045FA064663682846D2
:103BF0000B225B680A4926F056FF63683246694625
:103C000028465B6826F04FFF63681B2228465B68E6
:103C1000044926F048FF02B070BD00BF0C1104003B
:103C2000E8930400CC93040000210123064A90424B
:103C300006D8064A01B901231360054B1860704786
:103C4000012140085B00F2E740420F00A065002020
:103C5000A4650020014B03600020704734C40300BA
:103C600003289ABF024B53F820000248704700BF58
:103C700034C40300EC67040070B5046A0D469CB3BD
:103C80001E4A2379565CB34231D01D4A525C9A4297
:103C900030D1A3689847002810DA022D0CD0032DEC
:103CA0000BD110F1860F07D0D4E8EF3F43F00203A9
:103CB000C4E8E23F002AF6E7267170BD022D2671A6
:103CC00001D00020F9E7D4E8EF3F23F00403C4E873
:103CD000E23F002AF7D1D4E8EF3F23F00203C4E823
:103CE000E23F002AEDD0F6E76FF05700E5E76FF00E
:103CF0007700E2E76FF08500DFE700BFFD93040087
:103D0000F9930400024B187880F00100704700BF5F
:103D1000FDA2002010B50024094B86B0094803938A
:103D2000CDE9044435F04FFD03AB00934FF48062BE
:103D300023460549034822F093FD204606B010BDF6
:103D40003DF103008033002008A600202DE9F84F44
:103D5000046A80468B462046052100AF26F07EFF90
:103D600092469946064620B900252846BD46BDE83C
:103D7000F88FEFF31182202383F31288BFF36F8F44
:103D8000E368012B8ABF03F1FF330026E36082F36F
:103D90001188BFF36F8F002EE6D1FFF7B3FF88BB0A
:103DA00035F06FFD421E66F1000304F1180026F0A5
:103DB0005BFF051E5ADB5E46E3682BBB2D4802689D
:103DC00012F0060F13D06D4688B0D8F800106A467E
:103DD000294ECDE905614FF40071ADF81C1027495B
:103DE00042F8101F4FF4E451FFF7A0FCAD466FF00E
:103DF0007705FFF787FF0028B7D104F1180026F0F8
:103E000035FFB2E73546D7E7013BE360002BF0D141
:103E10004EB102235246237104F140014B4618482B
:103E200022F05EFDE5E73146A36860699847051E0C
:103E300003DAE3680133E360DBE701232371022146
:103E4000D8F8200026F00AFF0028D2D0D8F8203079
:103E5000186926F00DFFD8F82030D3E8EF1F21F0C5
:103E60000401C3E8E21F002AC3D0F6E76FF00F0594
:103E70007BE700BFBC28002052F1030003000001D3
:103E800080330020F8B5056A0646002D5ED0052176
:103E9000284626F0E3FE00285BD1304626F082FE5D
:103EA0000446002857D10821306A26F0D7FEE0B139
:103EB000356AEFF31187202383F31288BFF36F8FE6
:103EC000297931B93046AB689847041E07DB0123D6
:103ED0002B712B6843F020032B600023EB6087F3EA
:103EE0001188BFF36F8F2046F8BDFFF70BFF38B97D
:103EF0004FF0FF324FF0FF3305F1180026F0B4FE0B
:103F00006B692BB915496E6105F1400035F061FC14
:103F10002979C9B9AB6868699847041E0BDB01238E
:103F20002B710023EB60D5E8EF3F43F02003C5E899
:103F3000E23F002AF7D1FFF7E5FE0028D3D105F1D3
:103F4000180026F093FECEE70024EAE76FF0850420
:103F5000C9E70024C7E76FF00F04C4E787AE02008B
:103F600010B50C46054927F0D8FC00B100680023C5
:103F7000C4E901332060E36010BD00BF67AF0200F9
:103F800073B505465068164627F0D4FC044650B970
:103F9000012128467368124A27F081FA6FF0120453
:103FA000204602B070BD26F0CDFF40B92368012144
:103FB00028460C4A27F073FA6FF01504F0E7204604
:103FC0000022002326F09BFF041E07DA0121284669
:103FD000054B064A009427F062FAE1E70024DFE788
:103FE00069F103007DF10300A0F10300B2F10300C9
:103FF00073B505465068164627F09CFC044650B938
:10400000012128467368114A27F049FA6FF012041B
:10401000204602B070BD26F095FF40B9236801210B
:1040200028460B4A27F03BFA6FF01504F0E72046CC
:1040300026F01EFE041E07DA01212846054B064A1B
:10404000009427F02CFAE3E70024E1E769F103008C
:104050007DF10300C7F10300B2F1030073B505461B
:104060005068164627F066FC044650B901212846E0
:104070007368114A27F013FA6FF01204204602B059
:1040800070BD26F05FFF40B92368012128460B4A26
:1040900027F005FA6FF01504F0E7204626F007FE3A
:1040A000041E07DA01212846054B064A009427F032
:1040B000F6F9E3E70024E1E769F103007DF103008D
:1040C000D3F10300B2F1030073B5054650681646FC
:1040D00027F030FC044650B9012128467368124A83
:1040E00027F0DDF96FF01204204602B070BD26F013
:1040F00029FF064640B12368012128460B4A27F0D4
:10410000CEF96FF01504EFE720460121FFF7B4FD6B
:10411000041E07DA01212846054B064A009427F0C1
:10412000BEF9E1E73446DFE769F10300DFF10300A0
:104130001DF20300B2F1030073B506465068154640
:1041400027F0F8FB044650B9012130466B68124A4B
:1041500027F0A5F96FF01204204602B070BD26F0DA
:10416000F1FE054640B12368012130460B4A27F095
:1041700096F96FF01504EFE701462046FFF77CFD46
:10418000041E07DA01213046054B064A009427F049
:1041900086F9E1E72C46DFE769F10300DFF1030070
:1041A00024F20300B2F1030010B5044634F0EEFB34
:1041B00008210346024A204627F071F9002010BD6D
:1041C00041F3030037B513460022044601920A2149
:1041D000586801AA01F0DCFE019D95B947F6122C42
:1041E00020EAE074294640F2E7304FF47A72002367
:1041F000E4FB0C01FDF77CF935F09CFC284603B08C
:1042000030BD2B4601212046024A27F048F9019D86
:10421000F4E700BF66F3030008B50821024B034A28
:1042200027F03DF9002008BD53F403005AF40300C1
:10423000F7B51746002305460A2101AAB86801937D
:1042400001F0A6FE0321194AC6B2284627F027F935
:10425000019C4CB1234601212846154A27F01FF93D
:10426000019C204603B0F0BD042E0AD9334601213B
:104270002846104A27F013F9284627F046F901246A
:10428000EFE77868FFF79AF9021E08DA012128465D
:104290007B68094A27F003F96FF01504E1E733461C
:1042A0002146204612B226F053FBDAE77DF40300E4
:1042B000E3F403000AF5030021F50300002307B52A
:1042C0000090694604488DF8043023F0A3F99DF866
:1042D000040003B05DF804FB71AF020038B504467A
:1042E000EFF31185202383F31288BFF36F8F20F043
:1042F0003FF9034685F31188BFF36F8F08212046ED
:10430000064A27F0CCF82046054A082127F0C7F8CE
:104310002146044823F098F9002038BD79F50300C0
:1043200098F5030029430000F0B599B004460D4606
:10433000D0F8B46035F0ABFA024603F0EFF8364B34
:104340001958364B2846002A18BF1346344ACDE97F
:104350000043344B8C4218BF13460821324A27F0E1
:104360009EF8D4E90823CDE9022394F90E30082100
:104370000093A38928462D4A27F091F8202210A9FE
:10438000204622F0BDFBE26F03460821284600923A
:10439000274A27F084F804A9204635F090FA07460A
:1043A0000AA835F096FA07431FD1DDE90A236421F4
:1043B000049FDDF814E0A7FB010C01FB0EC1FDF723
:1043C00097F83B460090082128461A4A27F067F8DC
:1043D00020460AA935F069FA034660B1082128464B
:1043E000154A27F05CF819B0F0BD08212846134A99
:1043F00027F055F8ECE764230A9A2846B11A4B4394
:10440000B3FBF6F3CDE90021CDE902630821334681
:104410000B4A27F044F8E6E708000000A2F5030085
:10442000A4420400640B0400A5F50300B1F50300E9
:10443000DDF50300F4F503003CF6030019F6030074
:1044400069F6030030B5044693B00AAD202200217E
:10445000284635F0BFFF1A222021284635F0BAFF42
:104460002146114823F0F0F809AA4FF400610F48E3
:1044700035F00FFA6423099A0195C2F500614B43A8
:10448000DB0A002506934FF400632046CDE90413B0
:10449000CDE902320821054B054A009526F0FFFFC1
:1044A000284613B030BD00BFB5440000F8F8002026
:1044B000B5F60300F0B504460D46D0F8B46089B0F7
:1044C00007A935F0F2F9034630B1082128460F4A12
:1044D00026F0E5FF09B0F0BD204635F0D8F9642399
:1044E000079A0B4FB11A4B43002818BF0746B3FB7E
:1044F000F6F3CDE90221CDE90463082123462846DD
:10450000CDE90076034A26F0CAFFE3E73CF6030054
:10451000A2F50300FEF6030038B513460546102247
:104520000021586823F068FE0446FFF7C7FE40B933
:104530002346012128460E4A26F0B1FF6FF01500F0
:1045400038BD02F0EBFF0B4B1B589C4205D10121FB
:104550002846094A26F0A3FFF0E7204622F0A2FBF6
:10456000284623460821054A26F099FF0020E7E760
:1045700062F70300080000007DF70300A5F70300C1
:1045800038B51346054610220021586823F034FE42
:104590000446FFF793FE40B92346012128460E4A00
:1045A00026F07DFF6FF0150038BD02F0B7FF0B4B12
:1045B0001B589C4205D101212846094A26F06FFF6D
:1045C000F0E7204622F08EFB284623460821054AC4
:1045D00026F065FF0020E7E762F70300080000000F
:1045E000DCF7030002F8030038B513460546102235
:1045F0000021586823F000FE0446FFF75FFE40B933
:104600002346012128460E4A26F049FF6FF0150087
:1046100038BD02F083FF0B4B1B589C4205D1012192
:104620002846094A26F03BFFF0E7204602F000FF4B
:10463000284623460821054A26F031FF0020E7E7F7
:1046400062F703000800000036F803005BF803007F
:1046500010B50C46002127F065F900B10068002371
:10466000024A2060C4E90123E36010BD4B7D0400D1
:1046700010B50C46002127F059F900B1006800235D
:10468000024A2060C4E90123E36010BD4B7D0400B1
:1046900073B505461646506821F092FA044648B9AB
:1046A000284601217368174A26F0F9FE6FF01200C0
:1046B00002B070BD26F046FC40B92846012173685F
:1046C000114A26F0ECFE6FF08500F1E720460DF16F
:1046D000070126F05EFA9DF8072073684AB928465C
:1046E00008210A4A26F0DBFE204626F0C1FA002007
:1046F000DEE728460821064A26F0D1FE204626F0AD
:10470000D6FAF4E793F80300A8F80300DCF80300F6
:10471000F7F8030010B5034600680C46114608B1CF
:10472000027822B92046024A23F0A4FC204610BD9C
:1047300012F9030010B50C68D1E90112FFF7EAFF86
:1047400008210346024A204626F0A9FE002010BD9B
:1047500017F9030070B505460C4634F06AFC70B9D1
:10476000D4E9011228462668FFF7D4FF0121034649
:10477000044A304626F093FE6FF0150070BD00200D
:10478000FCE700BF27F903002DE9F04F93B0044682
:1047900002A88846914621F007FA2823029F0821A3
:1047A00003FB00773C4A204626F079FE029DBD427D
:1047B00003D3002013B0BDE8F08F0DF1180A3022AA
:1047C00051462846FFF7A6FFB8F1020F064606D16C
:1047D000D9F8041035F09FFE08B92835E7E73346CD
:1047E000082120462D4A26F05AFE284634F021FCA6
:1047F00000283ED00023284603A98DF80C3026F06F
:10480000C8F9002833D19DF80C00FFF729FA0646B5
:10481000284626F09DFB00282DDB0090334608211A
:1048200020461F4A26F03BFE302328461D4903AA96
:104830000593CDE9034A34F007FC6B6A002BCCD01A
:104840001E68002EC9D03368002BC6D00821204630
:10485000154A26F024FEB3464FF0000A336853454C
:1048600010D808212046114A26F019FEB5E7104E4F
:10487000CEE7104ECCE73346082120460E4A26F0FC
:104880000EFED1E7082120465BF8043F0B4A26F0D4
:1048900006FE0AF1010AE1E75CF9030066F903008C
:1048A0006BF90300354700007CF903009EF6030016
:1048B0004DF9030053F903008139040067F903003F
:1048C000F0B5054693B05068164627F03EF8074607
:1048D00050B9012128467368164A26F0E0FD6FF0B2
:1048E0001204204613B0F0BD34F0A3FB38B1736856
:1048F000114A0221284626F0D2FD0024F1E706AB3A
:104900000493302338460D4903AA0395059334F0E8
:104910009BFB041EE5DB384634F082FB73680446DB
:1049200030B1009001212846054A26F0B8FDD8E7AD
:10493000044ADEE793F803008EF9030055470000B0
:10494000B0F90300DDF90300F7B5137806463A2BFA
:104950000F46154614D1541C23783A2B29D1013423
:104960000A22204601A923F0D3FB019A0346A24262
:10497000386018D01078B0B93C2B16D9164A0EE022
:104980000A22284601A923F0C3FB019CB860AC426F
:1049900009D023783A2B06D1172808D90F4A0121CC
:1049A000304626F07CFD6FF0150003B0F0BD0134F9
:1049B000D2E70A22204601A923F0AAFB019B7860D6
:1049C000A342F0D01A783A2AEDD13B2801D9044A03
:1049D000E5E75C1CC4E700BFBFFA0300A1FA0300CF
:1049E000AFFA03002DE9F0410D4696B008A9044640
:1049F00001201746FEF728F80DA908A823F08EFA23
:104A0000032D57D17D680A22284607A923F080FB91
:104A1000079E8046B54216D032782D2A13D1013632
:104A20000A22304607A923F073FB079B9E420AD057
:104A30001A782D2A07D1451E0B2D0DD9314A012197
:104A4000204626F02CFD204626F05FFD6FF0150570
:104A5000284616B0BDE8F0815E1C0A22304607A940
:104A600023F056FB079B9E42EDD01B78002BEAD12A
:104A7000431E1E2B01D9244AE1E7A8F26C73CDE94D
:104A80001153BA68109020460DA9FFF75DFF00286A
:104A9000D9D10DA8FEF7C4F8B1F1FF3F08BFB0F1BE
:104AA000FF3FCDE9080109D101212046174A26F030
:104AB000F6FCCBE7022DC6D17A68E4E700230A931F
:104AC000012008A9FDF7F6FF054630B10346012194
:104AD00020460F4A26F0E3FCB8E70D9B082104931B
:104AE0000E9B204603930F9B0A4A0293109B01934F
:104AF000119B01330093129B03F26C7326F0CFFCE1
:104B0000A6E700BFCFFA0300DEFA0300EBFA0300CA
:104B100014FB03002BFB030010B5044694B006A958
:104B20000120FDF791FF0BA906A823F0F7F90B9BD5
:104B3000204604930C9B082103930D9B074A029384
:104B40000E9B01930F9B01330093109B03F26C7338
:104B500026F0A5FC002014B010BD00BF2BFB030005
:104B60002DE9F3411446884607461022002160686B
:104B700023F042FBB8F1020F064620D90A22002199
:104B8000A06823F039FBC5B22B4608213846224ADB
:104B900026F085FCB8F1030F22D8102D11D0202D5E
:104BA00012D0082D12D13378DBB200220821CDE9D2
:104BB00000323846194A26F072FC00200DE020250C
:104BC000E2E733889BB2F0E73368EEE73846082126
:104BD000134A26F064FC6FF0150002B0BDE8F081C6
:104BE0001022E068002123F06DFB0E4ACDE90001A0
:104BF00004460821384626F052FC102D06D0202D00
:104C000007D0082DE2D1E4B23470D6E7A4B23480E4
:104C1000D3E73460D1E700BF76FB0300A1FB0300BC
:104C20008BFB0300B4FB030000232DE9F047914602
:104C30004FF0FF35012286B00193514B074688465D
:104C40001A602026FEF742F82C46494640464D4A57
:104C5000FEF760F8431C07D1691C43D14A4A012181
:104C6000384626F01CFC18E073281BD0772829D082
:104C7000612812D1DFF814A11021DAF8000001AA8E
:104C800001F086F9019B0546002BDED0DAF80030F2
:104C90003F4A0121384626F002FC6FF0150006B0AD
:104CA000BDE8F087DFF8E4A00021DAF8000001AAEF
:104CB00001F06EF9019B0446002BC6D0DAF80030F3
:104CC000344AE6E7DFF8C4A00021DAF8000001AAC0
:104CD00001F05EF9019B0646002BB6D0DAF80030F1
:104CE0002D4AD6E7621C01D12C4AB8E75FFA86F854
:104CF000A8F10803DBB2182BC6F3C40604D8284A6F
:104D000022FA03F3DB0721D443460821254AC1E7F1
:104D1000B8F1100F21D0B8F1200F24D0B8F1080F4E
:104D200001D10A781A70314433444218102AEFD95D
:104D3000102CA14628BF4FF0100929464B46384693
:104D400002AA01F04DF91035A4EB0904B4B1A64252
:104D5000EED8294602AB701BE7E70A8892B21A70B8
:104D6000120A5A70DFE70A68C2F3072C1A70120C95
:104D70009A70120A83F801C0DA70D4E720468EE7F1
:104D8000041D002004FC03000BFC030080650020D0
:104D9000CAFB0300DDFB0300F0FB030028FC03005B
:104DA0000101000142FC030070B50F4E04460D46A0
:104DB000337831B12BB10121BDE870400B4A26F0A8
:104DC0006EBB83F00103337033B108212046084ADB
:104DD00026F065FB0123337029462046BDE870406C
:104DE000002226F0ACBB00BF688000205CFC030002
:104DF00097FC03002DE9F04105460C46DFF8EC80F6
:104E00003B4E8F18BC4201D1BDE8F08198F80020DC
:104E100014F8013B182A23D1112B21D10026354C3F
:104E2000082123682846344A88F8006026F037FBBA
:104E300028463146FFF7B8FF304B18780028E3D1F9
:104E40002F4A23681168042B2EDC08B123601160FF
:104E500013F003012FD1126813681BBA1360D3E754
:104E6000A3F13002092A88F8003004D923F0200287
:104E7000413A052A04D83168224A5354013131603D
:104E80003368022BBED1102200211E4823F0B4F952
:104E90001D4A136803F8010B1360164A13680133A7
:104EA000136000233360ADE70868043B00BA41F8A3
:104EB000040B0120C7E75B4203F0030358BF5942CC
:104EC000022904D1126813685BBA9BB2C6E70329B2
:104ED0009AD1106802681104C2F3074301F47F01FC
:104EE0000B4302F47F42134303608DE76980002087
:104EF000A8650020AC650020C1FC03006A8000208A
:104F0000B06500206B800020B46500202DE9F843D7
:104F10000023804617460D462649274E0B60274939
:104F200033700B60012DB94657F8044F1DD902228A
:104F30002046234935F0A8FA70B9A378003B18BF82
:104F400001231C44022220461E4935F09DFA28B94F
:104F500001233370013DE5E70023F2E720461849BD
:104F6000FCF7E0FAC0B909F104090022D9F80400FD
:104F7000114623F041F90022134B11461860D9F86D
:104F8000040023F039F9114B114918604046FFF72E
:104F90000BFF0020BDE8F88323782D2BE5D1637843
:104FA000002BE2D02346082140460A4A26F077FA31
:104FB000D0E700BFA86500206A800020AC65002013
:104FC000DBFC0300DEFC0300B4650020B0650020BC
:104FD000F54D0000E1FC030007B5094834F029F85D
:104FE00058B104233A22009305490123054800F0F3
:104FF000C3FE002003B05DF804FB6FF01200F9E778
:1050000058AB03007CBA030070B5044608466168DB
:10501000C1E900028B6025F04AFE00282BDB6468A2
:10502000264604F1480356F8285BA3634423E36350
:10503000042384F840300122002104F1100034F0F0
:10504000A5FA304604F1380133F006F8304632F064
:1050500046FFAB6806461B681BB122462846064938
:10506000984794F83420AB683146DC68284642F211
:105070001073A047002070BDB5B002000048704713
:105080007CBA030010B5044681681C3101F046FB70
:10509000A1682046BDE81040014A1C3101F0DEBA8B
:1050A00070FE03002DE9F341064614460F46D0F882
:1050B000088021B9A8F8441002B0BDE8F081184872
:1050C00026F068F8B8F83E500444A4B22D1A95FBB7
:1050D000F4F5384626F05EF8B8F84430ADB25A1C04
:1050E000A8F84420B3FBF5F205FB1233241A9BB257
:1050F000A4B26BB906213046094B0A4A009726F044
:1051000029FE2146304602B0BDE8F04100F0ECBF78
:105110003B4606213046044A26F01CFEF1E700BF5C
:10512000A34204007EFE030068F903008368D3F8FD
:1051300080329B0603D50249406926F008B87047C3
:105140002CC0030010B5044626F03EF8A3680146C3
:105150009B6C0BB120469847002202F0DFF9A36850
:10516000C3F8B022014B185802F062F908000000A1
:10517000014925F0ECBF00BF9EF6030014222DE983
:10518000F04FA5B0044600210DEB020035F022F9E6
:10519000542200210FA835F01DF900230493A368C1
:1051A00020466033029326F004FD204626F047FC9B
:1051B00010B96069FFF7DCFF00274FF0FF38BA46EF
:1051C0003D463E46B946A068142200211C3035F009
:1051D00001F9204626F066FBA168E068B1F8582086
:1051E000603127F042F80DF13C0B0397049B012B33
:1051F00005D0142D00F0D480B8F1000F1AD1B9F108
:10520000000F0AD099F81130FE2B06D124AB03EB26
:10521000850353F8543C03B10135A068836A002B21
:1052200040F08A80CFB1036A9F422BD00B9700F1E8
:105230001C0522E059460223029A04A826F032FAFD
:105240005BF8042F04990346029231B101290AD177
:1052500048B1574A204626F07DFD6FF007052846E5
:1052600025B0BDE8F08FC5B15BF8040C01F086FAFB
:1052700098B167B1A5680B971C350AAE0FCE0FC564
:1052800033682B602046FFF7FDFE0125E7E701218B
:105290002046484A26F05EFDDFE7039B33B94846C7
:1052A0005BF8041C05AA26F0ADFA064608F1FF38A3
:1052B0003EB3F368ABB1B646A36803F11C0CBEE87D
:1052C0000F00ACE80F00DEF80030CCF80030B36817
:1052D00033B9737CFE2B04BF96F8108008F1FF38B9
:1052E000AA46D6F804C0BCF1000F08D0B6460AAFF3
:1052F000BEE80F000FC7DEF800303B606746B146DE
:1053000002E055B101230393B8F1000F03D1049BD0
:10531000022B7FF46BAF013568E7A3681B6B13B1F9
:10532000DB68002BEED1244B0121009320460F9B1C
:10533000224A26F00FFDE5E790F82C30A5EB0A0590
:10534000BBB14FF6FF7290F82D10FF2918BF0A4627
:105350009D4202D313449D420BD9C36901212046CB
:10536000174A26F0F7FC2046FFF78CFE6FF0150574
:1053700075E7012125F04EFFA06825F03FFFA368E7
:105380000FAA29469B6A02EB8A02204698470546E7
:10539000A06825F037FF0021A06825F03BFF5EE7FD
:1053A000022B7FF42CAF0121064B074A52E700BFC6
:1053B00084FE030098FE0300B6FE03007329040078
:1053C000EEFE0300CAFE03004F3A040070B5044627
:1053D00083689E7D012E3BD1A368D3F880329A0664
:1053E00003D51F49606925F0B2FE2046FFF79EFEF7
:1053F000E06926F0DAFD012E05462DD1A368D3F829
:1054000080329B0603D51749606925F0A0FEA3688A
:105410009B6923B108212046134A26F09BFC2046B5
:1054200000F078FE204626F030FBA368B3F8583031
:1054300023B140F2D510002134F07CFB3DB1A068CF
:10544000012100F5227025F0B5FE0028C2D070BD04
:10545000204626F0D9FBCBE7204600F0DFFFE4E74B
:1054600031C0030035C0030068F90300022210B503
:10547000836804461A758368DB6CBBB925F05CFE53
:105480008368D3F88432DB040BD50321084B094A27
:1054900026F060FCA0686FF4805100F5217025F0C3
:1054A0006EFE2046BDE8104000F0B8BF10BD00BF42
:1054B00009FF030068F9030000232DE9F04F0446BB
:1054C000ADB00593A3686068DE6C026815692EB301
:1054D0001F6D102205AB17A9A84700281BDB059BF1
:1054E000CBB10121A06825F095FEA06825F086FECD
:1054F0003B46059A17A92046B047A06825F082FED2
:105500000021A06825F086FEA368DB6C002BD9D1B2
:105510002046FFF7ABFF2DB0BDE8F08F012205ABB1
:105520000DF11301A8470028F5DB059B002BF2D0F5
:105530009DF913109DF813300029A268C2DB517D3C
:10554000032900F2B683DFE811F0040036034D03AF
:10555000B4030D2BD2F8841241D00A2B3FD021F096
:10556000FF01092BC2F884126BD028D8002B00F061
:105570002B81082B00F09982A268D2F880128F0745
:1055800040F12281013B162B00F21E81DFE813F06F
:105590007A03AC02B002A8027403C9021C011C0108
:1055A0001C011C01CD02D1021C01E6021C01EB0210
:1055B0001C011C011C01ED02FD021C010B031B2B35
:1055C0003BD07F2B00F07E82A3F120025E2AD3D84D
:1055D0000121A06825F029FE9DF8131015E1C9B23C
:1055E00021B1D2F88412C9B28B42C5D1D2F884124B
:1055F00063F30701C2F88412A568AB7D012B06D1C5
:105600006069FFF7B5FD0222A3689A7583E7B5F8D4
:10561000581061B9284625F008FEE06826F0F7FD2D
:105620006069FFF7A5FD2046FFF720FF4AE7204607
:10563000FFF7A4FDC5F8B402F5E70122A3685A7587
:10564000C2E0A068D0F880329E07C3F3400940F161
:10565000BB80012125F0E9FDA068857D002D40F08B
:10566000B380B0F85830FF2B00F0AE80B0F85A206D
:1056700000F1600100F5B07034F086FEA368B3F865
:105680005A20134483F86051A068B0F85A5055B1BD
:10569000054495F85F50202D00F08880093D042DC9
:1056A0008CBF0025012500F5B07002461378114625
:1056B0000132DBB1202BF9D0093B042BF6D98DB98F
:1056C0000A4611F8013B13F0DF0F02D0093B042B0F
:1056D000F6D8013A12F8013F43B1202BFAD0093B2A
:1056E000042BF7D94FF4807126F0B7F8A26817A9F8
:1056F000142302F5B07207A825F0D4FF07991429E6
:1057000062D800222CAB03EB810343F8542C19B16F
:10571000002D4ED101294BD100250695069E002E65
:1057200040F0FA80DDF85CA0B046504625F032FD2E
:105730003746314603904B1C284612AA029300F0CC
:10574000C3FB0146002843D1012E62D1069B2CAA3F
:1057500002EB8303384653F8546C25F01BFD0546D5
:10576000304625F017FD854205D02A1A92B2391825
:10577000204626F036FBA068B0F85A30034493F870
:105780006030202B3BD0093B042B38D9D0F8803235
:10579000DD0739D5002125F0A1FD2021204600F0AC
:1057A00005FE0121A06825F099FD0DE001257AE7AD
:1057B0000139002008AB0093019006AB17AA26F030
:1057C0004FF805460028A9D1606925F0C3FE79E6A7
:1057D000D1F800B0039A5146584625F0E1FC60B17B
:1057E0005846FBF7B1FE404538BF4046002E18BF73
:1057F000BB465F461FFA80F8013602999BE70121FC
:10580000204626F067F9DFE72021204600F0CEFD94
:10581000DAE70290D8D9069B2CAA02EB830353F84F
:1058200054AC504625F0B6FC0646A3680299A3F88E
:105830004410284612AA01F1010B00F045FB07466F
:1058400048BB6069FFF794FC204600F0E7FD069B2B
:105850002CAA02EB830353F854BC4FF6FF7658464C
:1058600025F098FC394680464B1C284612AA029324
:1058700000F02AFB8246E0B94FF6FF739E42A3D0A8
:10588000002EA1D0A6EB080292B207EB0801204639
:1058900026F0A7FA98E73F6832465146384625F089
:1058A0007FFC20B1424639462046FFF7FBFB5946B4
:1058B000BFE7DAF80030424659461846039325F010
:1058C0006FFC88B1A068039BB9F1000F0ED04FF0B8
:1058D00000091946FF2200F5B07034F0E7FDA36817
:1058E00083F85F92DAF800700299BDE74A4600F249
:1058F0005F1010F801CF995C614500D111B9904556
:1059000005D9F1E74FF6FF7101328A42F1D1B24277
:10591000A8BF324696B2E7E72CAB03EB860656F8F3
:1059200054BC0026584625F035FCB1468246374621
:10593000B0464146284612AA00F0C6FA0346D8B936
:10594000012E31D1069B2CAA02EB830353F8540C91
:1059500025F020FCA2680646394628461C3200F095
:10596000B3FA0568284625F015FC86423FF403AFDC
:10597000821B92B2A919FBE61B685246594618468B
:10598000029325F00DFC60B1029B1846FBF7DCFD8D
:10599000484538BF4846002E08BF47461FFA80F9E1
:1059A000013608F10108C4E703907FF60DAF069AAF
:1059B0002CAB03EB820252F854ACB046504625F0B3
:1059C000E9FBBB46A268039B0290A2F84430A268A0
:1059D000594628461C3200F077FA0BF1010B036898
:1059E000BAF1000F09D043B118465146029A039309
:1059F00025F0D6FB039B0028E9D04A4619462046ED
:105A0000FFF750FBB8F10108E1D16069FFF7B0FB87
:105A1000204600F003FD069B2CAA02EB830353F8FB
:105A2000540C25F0B7FB39460DAA8046284600F0F5
:105A30004BFA07F101090746A0683968FF2200F513
:105A4000B07034F033FD3B684FF6FF77BA460293EF
:105A50004946284612AA09F1010B00F035FAD8B1DF
:105A60000022A168036801F25F1111F801EF985C50
:105A7000704503D110B101325245F6D1B8F1000F93
:105A800001D0424506DBBA42A8BF3A46013E012E8C
:105A900097B201D0D946DBE7002F3FF495AE0299CB
:105AA000A7EB080292B24144F1E6A068D0F8803238
:105AB00099077FF589AE012125F0B7FB204626F036
:105AC000B1F981E6A068D0F880329A077FF57CAE04
:105AD000012125F0AAFBA368D3F880321B07EDD47F
:105AE000204626F080F96FE6204626F06BF86BE63C
:105AF000204626F05EF8204625F0A1FF10B9606927
:105B0000FFF736FB0121A06825F08FFBA3689A7D83
:105B1000012A02D103229A7556E62046FFF7A6FC19
:105B200052E6204626F057F84EE6204626F05EF86C
:105B30004AE6D2F880329E0603D55F49606925F0B7
:105B400006FBA368D3F880329D0603D55B496069E4
:105B500025F0FDFA204600F061FC35E600212046E4
:105B600025F06EFB30E60121F9E7E06983681B79D7
:105B7000012B02D126F0DAF926E6022B7FF424AEBF
:105B80002146526D26F0BBF91EE6204626F00AF8A3
:105B9000204625F0D1FA0121A06825F046FB2046D9
:105BA000FFF7C4FA10E6204600F02EFB0121A068A2
:105BB00025F03BFB08E65B2B02D10223537503E67D
:105BC000D2F88022900706D5622B07D14FF0FF3123
:105BD000204625F0A8FF0022A36830E5662BFAD105
:105BE0000121F5E700215175A268D2F880128907DA
:105BF0007FF568AC313B1B2B3FF6E6AD01A151F8B8
:105C000023F000BF815C00008D5C0000A15C0000FF
:105C1000755C0000C9570000C9570000C957000053
:105C2000C9570000C9570000C9570000C9570000F4
:105C3000C9570000C9570000C9570000C9570000E4
:105C4000C9570000675B00005D5B0000235B00003C
:105C5000E95A0000C9570000795C0000C9570000EC
:105C6000855C0000C9570000C9570000C9570000F3
:105C7000915C000003235375204625F09AFFA3E5AD
:105C800003235375204625F08DFF9DE503235375AF
:105C9000A068D0F8801201F0010181F0010182E5D5
:105CA00003235375A368D3F880329B077FF58CAD2F
:105CB00016E7002382E700BF39C003003EC003009F
:105CC000D3B5044625F0B9FB38BB4FF0FF364FF093
:105CD000FF37A06800F5227000220721CDE9006798
:105CE00034F006FBA06825F08DFA042120460C4A0A
:105CF00025F003FB012120460A4A25F0FEFA204642
:105D00000221094A25F0F9FA606803685B6903B16A
:105D10009847A06825F072FADBE702B0D0BD00BF5B
:105D20004551000009B40200CD53000010B50446EF
:105D300008210C4A25F0B3FB204608210A4A25F029
:105D4000AEFB20460821094A25F0A9FB2046082180
:105D5000074A25F0A4FB20460021064A00F07EFCFD
:105D6000002010BD4DFF03008BFF0300EAFF03007E
:105D70003E000400D90004002DE9F041044680688B
:105D80008846D0F8B06215461F4688B0002E6AD10A
:105D90004FF42E72314634F01DFBA06800F52270DE
:105DA00034F095FAA06800F526700122114633F010
:105DB000EDFBA3694FF400711E60A06866F38205D5
:105DC00000F5217025F0D0F95022A3682046DA872B
:105DD0001822A3689A87216825F070FBA3684146C2
:105DE000C3F880526068214A03681D682346A847AB
:105DF0000546B8B90122A3681A75A06800F521709C
:105E0000A7B14FF4804125F0AFF9A3680E9A0021A5
:105E10005A65606803689B689847054658B12046F4
:105E200025F0D2F9284608B0BDE8F0816FF4804132
:105E300025F0A5F9E9E7D4E90A0100220023CDE91C
:105E400006230E234FF48052CDE90253CDE90045DD
:105E5000074B049520F088FFA368C3F8B002616A7D
:105E600020F038FEDEE76FF07705DBE727B30200AE
:105E7000C15C000010B5044613460A4601460648B8
:105E800001F08CFD23691B7923B12046BDE8104049
:105E900025F060BB10BD00BF6DB5020010B5044613
:105EA0000B4602460649074823F066FE23691B7924
:105EB00023B12046BDE8104025F04CBB10BD00BF0B
:105EC0009D7900006DB5020010B50B46144648B927
:105ED0001749184A521AB3EB920F05D251F82340D2
:105EE000204610BD82680AB90024F9E712498A42A7
:105EF0000FD312498A420CD2A27C214622F003021F
:105F0000A27482681846126890472368002BE7D174
:105F1000EAE70B498A4202D30A498A4205D312684A
:105F200014214B43D418D358F0E70133F8E700BFEE
:105F3000ACBA0300F4BA0300A4BF0300FCBF030023
:105F4000F4BA0300A4BF0300F7B5054601F0E6FA72
:105F5000002306460D4F1446C3510A46284601A9A0
:105F600022F0D6F8F359222B05D16FF0210300203F
:105F7000236003B0F0BD2BB9019BAB4202D01B786C
:105F8000002BF6D06FF01503F1E700BF0C00000006
:105F9000F7B5037804462D2B154605D16FF0150390
:105FA00000202B6003B0F0BD01F0B8FA00230646D4
:105FB0000A4F0A46C35101A9204622F01DF9F359A0
:105FC000222B02D16FF02103EAE7002BE6D1019BDF
:105FD000A342E3D01B78002BE4D0DFE70C000000E5
:105FE000F8B516461F46254A0B46082104460025EB
:105FF00025F055FAAF4210D908212046735D204A9A
:1060000025F04DFA0135102D0DD06A07F2D1082187
:1060100020461C4A25F043FAECE7082120461A4A9C
:1060200025F03DFAEEE708212046184A25F037FA18
:106030000025BD4215D2735D0821A3F120025F2A1D
:1060400028BF2E232046124A25F029FA0135102DAB
:106050000DD06B07EDD1082120460A4A25F01FFA22
:10606000E7E708212046074A25F019FAEEE720461F
:10607000BDE8F8400821074A25F011BA08010400DC
:10608000F6F00300A4420400A2420400FCF0030066
:10609000160104000F0104008368D3F880329B06C8
:1060A00003D50249406925F0ABBC704744C00300EA
:1060B000014925F0A5BC00BF9EF603000A1E0DDCB9
:1060C0000ED042238168D1F88012890608D5002AB3
:1060D00004494069B8BF524225F092BC4123F1E720
:1060E000704700BF120104000A1E0DDC0ED04423CD
:1060F0008168D1F88012890608D5002A04494069D0
:10610000B8BF524225F07CBC4323F1E7704700BF83
:10611000120104002DE9F0478468054604F160008F
:10612000FBF712FA0022914694F8408087B2E68F7E
:10613000A6EB0806BE4209DB002F21DD603268694C
:1061400022441049BDE8F04725F05ABC16443444B7
:1061500094F860A084F86090AB6860321A440A49F1
:10616000686925F04DFCAB683246334483F860A083
:10617000AC68E38FA3EB0803FF1A4FF00008D6E7E3
:10618000BDE8F08768F903004F3A040008290A4681
:1061900017D8836893F84210914212D083F84220B6
:1061A0008368082AD3F8803205D0990609D50549B5
:1061B000406925F025BC9B0603D50349406925F0BD
:1061C0001FBC70471901040049C0030038B50D46D3
:1061D00009780446FFF7DAFF6A78072A11D8A3681E
:1061E00093F8431091420CD083F84320A368D3F86E
:1061F00080329B0605D560690249BDE8384025F02C
:10620000FFBB38BD22010400F8B583680446B3F82B
:106210005820002A55D0B3F85A10002951D05F31C8
:1062200003F160050B441846A84206D3014611F855
:106230000169202E3CD0A8423CD286B29DB2AB1B55
:106240009BB2591C471CD21A0144384634F0A9F8B5
:10625000A268711BB2F85830204613FA81F3A2F8F5
:106260005830A36809B2B3F858201344002283F8C9
:10627000602025F02FFCA368D3F880329A0603D55E
:106280001049606925F0BCFB3B46082120460E4AB8
:1062900025F060FD2046FFF7FFFEA368D3F88032AB
:1062A0009B060ED560690949BDE8F84025F0A8BBFA
:1062B0000846B9E7014611F80169202EBDD008460D
:1062C000B9E7F8BD4EC0030068F9030052C00300EF
:1062D0002DE9F04704460F4690460AB1FFF7DCFE71
:1062E000A668D6F88032B6F85A505B0723D505F178
:1062F00060003044FBF728F90546B5B9A368B3F848
:106300005820A3F85A20A06825F087FB30B1B8F1D7
:10631000000F00D017B16069FFF7CAFE794220462E
:10632000BDE8F04709B225F0D5BB1D49606925F0ED
:1063300067FB013DE1E73046FBF706F9B6F85890F8
:10634000F38F19FA80F915FA80F0B0FBF3F2B9FB7C
:10635000F3F39A42AA461AD04845A368CEDADA8FF8
:10636000451CB0FBF2F302FB130313B96069FFF79E
:106370009FFEA36820465344082193F86030094AE1
:106380000AF1010625F0E6FCB2462846E4E760354E
:1063900008212046044A731925F0DCFCAEE700BF53
:1063A000640B04001601040068F9030013B5836848
:1063B0008DF80710D3F880220446D00725D5B3F80E
:1063C0005A10B3F858208A421FD0481C9DF8072065
:1063D000A3F85A000B4483F86020A368D3F8801216
:1063E000890710D5D3F88032606913F0040F18BF05
:1063F0002A22094925F004FB204625F020FB10B194
:106400006069FFF755FE02B010BD012220460DF174
:10641000070125F0ACFCF6E71601040010B583680F
:1064200004469A7D1AB90221084A25F093FCA36814
:10643000D3F880329B0707D52046FFF76BFE204636
:10644000BDE8104025F021BB10BD00BF68F9030076
:106450002DE9F843436807461C680E46A268E369C5
:10646000D2F880529A68C5F300151279012A03D038
:10647000032A4FD0BDE8F883D868D3F814800B788E
:1064800047F6122E5A0758BF0B684FF47A725CBF5A
:10649000C3F34A254B8840F2E7318C464FF00001A8
:1064A000E0FB0EC15EBF05EB1315173525F00705A0
:1064B0004FF0000360464CBF0025AD08FBF718F80D
:1064C00002460B464046294623F005FD814628B981
:1064D0003846BDE8F843012125F0D9BC012DF7D994
:1064E000314651F8043B0268C3F39D0363F39F02F6
:1064F00040F8042B6A1E920033F046FF404649469E
:1065000023F066FDA06800F522700221BDE8F84383
:1065100033F0E3BE2046D3F8049025F075FBA36862
:1065200005F18E0793F8168033F0ABF90546002885
:1065300042D0EFF31185202383F31288BFF36F8FCE
:10654000B8F1010FA36841D1D3F880329B0603D57F
:106550002A49606925F08EFCA368D3F8803298063A
:1065600003D52749606925F085FC3A4631464846FF
:1065700024F0D9FAB8F1010FA3682FD1D3F88032F3
:106580009A0603D51F49606925F074FCA3689B69CE
:1065900023B1082120461C4A25F0DCFB2046FFF7EA
:1065A000B9FD204625F071FA33F06BF9F0B185F3AF
:1065B0001188BFF36F8F5DE7A06800F526704FF07C
:1065C000FF324FF0FF331FF087FFB9E7D3F8843273
:1065D0001905CAD4204625F017FBC6E7D3F8843244
:1065E0001B05E1D42046FFF719FFDDE7A06800F5A1
:1065F0002670BDE8F8431FF033BF00BF56C003004C
:106600005AC003005FC0030068F90300014925F088
:106610000ABD00BF9EF60300F8B50F465168054657
:1066200016461C4611B11A4625F00AFDB3688BB117
:1066300021462846FFF758FD0821074A3B462846D1
:1066400025F088FBB168E21D21B12846BDE8F8407D
:1066500025F0F6BCF8BD00BF2B0104002DE9F04386
:106660000E460021044617460D4689B0304603AA5F
:1066700001F10108FFF728FC88B96DB127B13A464E
:106680000821204625F066FB0021304603AA01F1CF
:106690000108FFF719FC60B909B0BDE8F083006894
:1066A00010B1FAF751FF80B2854238BF0546414626
:1066B000DCE7D0F80090B9F1000F0FD099F8003066
:1066C00063B1476808212046CDE90059104B114AB3
:1066D00025F040FB27B96069FFF798FF4146D4E7F2
:1066E0000B4B204608210C4A25F034FB384625F098
:1066F00088FCAB1D9BB228B13A4649462046FFF7BD
:106700008BFFEBE71A463946204625F099FCE5E772
:106710000594040036010400C1F00300F7B50F68CA
:1067200005460E46D7B13846FAF70EFF84B2114B34
:10673000082128460093104A3B4625F00BFB716860
:10674000084625F05EFCE31C9BB248B10A46284689
:10675000316803B0BDE8F040FFF75EBF3C46E6E7B6
:1067600031B11A46284603B0BDE8F04025F068BCB8
:1067700003B0F0BD019404007FFE030010B507498B
:106780000446FAF7CFFE38B120460549FAF7CAFEAB
:10679000B0FA80F0400910BD0120FCE73D01040083
:1067A0004001040010B583680446D3F880329B068C
:1067B00003D50649406925F0AFFC5022A3680020AC
:1067C000DA871822A3689A8710BD00BF63C0030050
:1067D00008B5836908211B68024A24F060FE002086
:1067E00008BD00BF47010400F7B508210D4A054662
:1067F00024F055FE00230C4C0C4EB44203F101076B
:1068000002D3002003B0F0BD626A9BB20192A2687D
:10681000082100922846064A24F041FE30343B46C7
:10682000EBE700BF570104007CBA0300ACBA0300D9
:106830006F01040008B5024924F040FE002008BDA5
:10684000EC67040030B50446002585B0A2680DF160
:106850000E030121E06802F5B07225F0DBFCBDF803
:106860000E00A36850B103F5B073009308212B46C6
:106870002046044A24F013FE0135E7E783F860015F
:1068800005B030BD8001040010B5044624F04FFE71
:1068900008210346024A204624F001FE002010BDD4
:1068A000B13E0400022907B50DD1536801210193BF
:1068B0000C4B009313680C4A24F0F1FD6FF01500A7
:1068C00003B05DF804FB8368084AD3F880320821DE
:1068D00013F0020F064B08BF1346064A24F0DFFDF3
:1068E0000020EDE7930104008A0104002FF103006A
:1068F000676C0400A801040010B583680446D3F84F
:1069000080329A0603D50749406925F005FCA36843
:10691000D3F880329B0603D50349606925F0FCFB60
:10692000002010BD6AC003006FC00300F0B501294C
:10693000044685B00DD0536801210193604B6FF080
:106940001505009313685F4A24F0A9FD284605B099
:10695000F0BD8368D3F880329A0603D55A4940695E
:1069600025F0DAFB00256FF0F9012046FFF7A6FBC2
:10697000FA212046FFF7B8FBA0684FF48072294641
:1069800000F5B0708DF80B5033F024FD4F4960696D
:1069900025F0C2FB606924F0DDFD4FF47A76606873
:1069A000012203680DF10B011F6903ABB8470028F2
:1069B00009DB039B13BB013E4FF47A70B6B232F091
:1069C0000EFB002EEBD16FF08505A368D3F8803263
:1069D0009B0603D53E49606925F09EFB002DB5D08E
:1069E0005022A3680321DA871822A36820469A87D9
:1069F000384A24F054FD6FF00705A7E79DF80B20F7
:106A0000A3681B2A4FD093F860111B29C7D1522AC3
:106A100049D15A19002382F86031A66896F861219D
:106A20005B2A27D1022206F2611515F8010F1146E3
:106A30003B2802F1010292B21FD1FF29C3D00020EE
:106A400001F5B07116FA81F111F8015FFDB9FA286C
:106A5000074686F8605128BFFA27FA2B1A46A16824
:106A600028BFFA220028AED0002BACD0CF87A36875
:106A70009A87AAE786F86031A5E703EB83033038ED
:106A800000EB4300B2F5807F83B2CED19BE70132A9
:106A900000EB800092B2303D05EB4005B2F5807FFF
:106AA000A8B2D1D18FE72B440135ADB2092D83F8BF
:106AB00060217FF674AF0022A36883F8602182E72B
:106AC000930104008A01040075C0030008940400C7
:106AD00079C00300B901040008B5044823F0CCF8DC
:106AE000034823F0C9F8002008BD00BFB006040029
:106AF000E606040080B505460E461746984620F087
:106B0000CBFC034600F00AFD0446DFF8189042462D
:106B100049F8003039463046A84754F8090000F0DB
:106B200087FC00BF0800000008B50348034A0021A5
:106B3000121A25F0EAFB08BD602E002008A30020F1
:106B4000074808B5074A0849121A25F0E0FBBDE8D6
:106B500008400648064A0749121A25F0D8BB00BF6C
:106B6000000000205C2E002078940400000000202B
:106B700000000020789404002DE9F84305460C46F7
:106B800000AF002948D0DFF8B890D9F800305A0794
:106B900042D0D1E900016E468AB06A46A3684FF040
:106BA0000508DFF8A0C0CDE90713CDE905C042F81C
:106BB000108F00234FF421514846FCF7B7FDD9F858
:106BC0000030B5465B0727D0D4E903018AB06A4696
:106BD0006369DFF874C0CDE90713CDE905C042F859
:106BE000108F002348464FF42151FCF79FFDD9F840
:106BF0000030B54658070FD0E36901214846134AD3
:106C000023F03BFFD9F80030590705D0A3690121D3
:106C100048460F4A23F031FF012D0AD1EFF30583D7
:106C200007480268520704D00A4A2946103B23F05D
:106C300024FF214628461FF029F8BD46BDE8F88309
:106C4000B42800201407040043070400720704005E
:106C500081070400AF07040030BFFFF7FDBF00BF8E
:106C60002DE9F04105460B4EDFF82C80324606EB4D
:106C70000807CC1B2046094933F086FBA019424681
:106C80000021083C33F0A6FBC5F8C04007F108001E
:106C9000BDE8F0810000000008000000FCBF030018
:106CA00010B5334C2368580703D03249204625F0ED
:106CB0003BFB314B9B6A990157D523685A0703D098
:106CC0002E492B4825F030FB1E202B4B9B6ADB0105
:106CD00007D52368580703D02949254825F024FB08
:106CE0001F20254B9B6AD90207D523685A0703D07A
:106CF00024491F4825F018FB02201F4B9B6A1B03E9
:106D000007D52368580703D01F49194825F00CFB05
:106D10002120194B9B6A590307D523685A0703D0D2
:106D20001A49134825F000FB2220134B9B6A9B0352
:106D300007D52368590703D015490D4825F0F4FA03
:106D400023200D4B9B6ADA0307D523685B0703D02A
:106D50001049074825F0E8FA2420074A936A6FEAA9
:106D600003436FEA1343936210BD1D20ADE700BFDC
:106D7000B4280020C207040000ED00E0DA07040098
:106D8000ED07040007080400310804004F08040060
:106D9000740804008E080400F8B5364C06462368D3
:106DA0000D465B0703D03449204625F0BDFA334B2E
:106DB0009B6ADF065CD52368580703D030492D480D
:106DC00025F0B2FA11202D4B9B6A190707D52368CD
:106DD0005A0703D02B49274825F0A6FA1220274F3F
:106DE000BB6A9B0719D52368580703D02649214859
:106DF00025F09AFA7B6BBA6A11060DD52268520704
:106E000004D00121214A1B4823F037FE26B11B4A3A
:106E1000936A23F0800393621320184B9B6ADB076D
:106E200007D523685F0703D01949124825F07CFA7B
:106E30001420124B9B6A9E0607D52368580703D07F
:106E400014490C4825F070FA15200C4B9A6AD106AB
:106E500058BF9A6A9A6A920642BF5A6A22F400524E
:106E60005A629A6A42F0FF029A6200232B70F8BDC0
:106E70001020A8E7B4280020B908040000ED00E0C5
:106E8000CF08040002090400150904002D090400BC
:106E90004309040062090400F8B5374C064623682C
:106EA0000D465B0703D03549204625F03DFA344BAB
:106EB0009B6ADF0451D52368580703D031492E4817
:106EC00025F032FA17202E4B9B6A190507D5236847
:106ED0005A0703D02C49284825F026FA1820284FB5
:106EE000BB6A9B0519D52368580703D02749224858
:106EF00025F01AFABB6BBA6A11040DD52268520745
:106F000004D00121224A1C4823F0B7FD26B11C4AB7
:106F1000936A23F4004393621920194B9B6A5B0523
:106F200007D523685F0703D01A49134825F0FCF9F9
:106F30001A20134B9A6AD60511D52368590703D036
:106F400015490D4825F0F0F91B200D4A936A43F4CA
:106F50007F43936200232B70F8BD1620B3E79B6A32
:106F60009A04F2D523685B0703D00C49024825F048
:106F7000DBF91C20E9E700BFB428002091090400D8
:106F800000ED00E0A709040002090400B8090400AC
:106F9000D1090400E6090400010A040062090400A2
:106FA000F0B58BB0794B044600255E6800AF85F3E1
:106FB0001188BFF36F8F02F07F43B3F17F4F0AD187
:106FC00002F00C03082B14D1714803685A0709D04A
:106FD000704925F0A9F96E4803685C0702D06E4934
:106FE00025F0A2F900210846FFF7C6FD2C37BD4663
:106FF000F0BD13074CBF0C460125002CEBD000223E
:10700000C6F30803FA71DA1E092A00F29980DFE854
:1070100002F0058B8E879797979797915C4E336810
:10702000590703D05D49304625F07EF90023FB71F6
:10703000564BDA6A920708D53368580703D0584987
:10704000534825F071F9002337E0DA6A002A04DAA0
:1070500033685907F7D05349F2E7DB6A5A00F2D593
:1070600033685B0703D05049494825F05DF9474B29
:10707000A1695A6942F480725A61BFF34F8FBFF31E
:107080006F8F31F8022C596921F480715961BFF377
:107090004F8FBFF36F8F02F47F41B1F55F4F2AD15D
:1070A000D2B2022A27D13368580705D023680121BC
:1070B0003E4A374823F0E1FC2368FA79002A95D14B
:1070C00007F1080604F1200C324620686168083494
:1070D00003C264451646F7D17A6A002D52D0C2F336
:1070E000080121B96FEA52226FEA42227A621846F9
:1070F00007F1080178E79A6AD2B222B10120F91D9E
:10710000FFF74AFE0EE09A6A12F47F4F04D0012086
:10711000F91DFFF7C1FE05E09B6AB3F5803F92D3EE
:10712000FFF7BEFD0346C8E70020F91DE8E7002091
:10713000F91DEEE716480368590784D01C4980E71B
:107140001348026852073FF47EAF1A4A16F4F87FDC
:107150006E468AB0184918BF11466A46103B07931D
:107160004FF40073DFF854C0ADF82030144BCDE974
:1071700005C142F8103F00234FF41151FCF7D6FA35
:10718000B54660E76FF30802B0E700BF00ED00E02E
:10719000B4280020470A0400720A0400AE0A040062
:1071A000C50A0400E60A0400F40A0400130B0400F4
:1071B0002F0B04002E0A0400190A0400530B0400CC
:1071C00004000001064B5A6942F010025A615A69E4
:1071D00042F480625A615A6922F008025A6170478B
:1071E00000ED00E0EFF30880EFF3098101B572468E
:1071F000FFF7D6FE01BD00BF002080F31488BFF367
:107200006F8F002080F30A8880F30B88124880F388
:1072100008881DF03BFA002010490860BFF34F8F2B
:1072200000F032F8202080F311880D484FF0AA01B9
:107230004FF4006225F069F809484FF400614018E6
:1072400080F30988EFF314800221084380F3148847
:10725000BFF36F8F00F082F83806012094ED00E054
:10726000F8F80020002318460649D1F89020C2F310
:107270000722934200DB7047C1F89830C1F8A000A4
:107280000133F6E700ED00E010B572B6002484F398
:107290001388FFF7E7FF23464FF0FF300C4A03F156
:1072A00020010133102B42F82100F8D100234FF0C8
:1072B000FF30074A03F160010133102B42F821002F
:1072C000F8D162B6BFF34F8FBFF36F8F10BD00BF11
:1072D00000E100E01EF0040F0CBFEFF30880EFF3B5
:1072E0000980816911F8021C0229FFD001B572469C
:1072F00025F00FF801BD00BF00B2002807DB012315
:107300004109034A00F01F00834042F821307047D2
:1073100000E100E000B2002801F10101ACBF00F182
:107320006040064B4FEA4111C9B2ABBF00F5614066
:1073300000F00F0080F800131954704714ED00E0BE
:10734000044B054A23F07F039360BFF34F8FBFF3D5
:107350006F8F70470000000000ED00E008B5FFF7F8
:10736000EFFF074AD2F8883023F47003C2F8883060
:10737000FFF7DAFBFFF7E4FB00F0AEF81EF0D6FDF6
:1073800000ED00E042F8203C009B0B4942F81C3C19
:10739000019B21F0010142F8183C029B42F8081CB5
:1073A00042F8143C4FF0807342F8043C0023203A2A
:1073B0000266C0F8C4307047F56A0000044608B59C
:1073C0000E4B15469860D0F8C0200D4B0E461A6043
:1073D0001FF052FCD4F8B03083F30B882C4686F3B0
:1073E00009880020034B98472046002100220023F3
:1073F000014C204749C30200F56A00006063002089
:10740000606900201022014B1A61704700ED00E016
:10741000054BDA699B689A421FBF044A536843F0E0
:1074200080535360704700BF6063002000ED00E0B0
:10743000084B9B6883420BD1EFF3058343B1064BA6
:107440005A6842F080525A605A6A22F400425A62E4
:1074500032F06CBA6063002000ED00E001B532F05C
:107460002CFABDE8014019498A684FF040001044E9
:10747000EFF3098C80E8F01F202080F31288BFF31F
:107480006F8F134F4FF00066CA698A603E60D2F872
:10749000C000104C2060D2F8C4000023C2F8C430F1
:1074A00080F3118802F1400090E8F01F8CF3098806
:1074B00002F1000004B524F03FFFBDE8044001B52F
:1074C0001FF0DAFBBDE80140704700006063002058
:1074D00004ED00E0606900200023202040F20F123C
:1074E00010B5044CE1180133934281F80003F9D13F
:1074F00010BD00BF00E100E008B5EFF30583064AC8
:10750000103B02EBC30152F8330049688847BDE8DD
:107510000840FFF77DBF00BF60AD03000148006871
:1075200070470000606900201FB50121094B0A4A1D
:107530000A4800F01BF90023064A0393084B012177
:10754000019301A8D31A029300F01AF905B05DF86F
:1075500004FB00BF0000042000000020A0C90300BD
:10756000602E00200A7A0B6810B562F304031C46F3
:10757000CB68520923F01F0343EA4203044A43F055
:107580000103C2F89800C2F89C40C2F8A03010BDB8
:1075900000ED00E010B50C4B0446D3F89030C3F377
:1075A0000723013B98420BD9084803685B0704D0C6
:1075B00001212346064A23F060FA6FF0150010BD42
:1075C000FFF7D0FFFBE700BF00ED00E0A42800209C
:1075D0006A0B04002DE9F04F8946144606464FF029
:1075E0000008534D85B0C8452EDAD6F804A0BAF18C
:1075F000000F4BD0BAF11F0F1BD91AF01F0F18D173
:10760000D6F800B01BF01F0F13D1584624F0BFFE70
:1076100007460AEB0B00013824F0B9FE874217D069
:107620006FF01507434803685B070BD0424A3B469F
:1076300005E0404803685A0704D043463F4A012109
:1076400023F01BFA6FF01504204605B0BDE8F08F5B
:1076500017F1160FE6D0BC42E4DDC5F89870D5F8F6
:107660009C10C5F89870D5F8A03021F01F0143F0A8
:107670001F0BD6E900321A44994202F1FF3A1AD19F
:10768000D34507D13146F8B224F08AFE08F101084B
:107690000C36A8E73146C5F89870D5F89C30E0B2B2
:1076A00063F30402C5F89C2024F07AFE10F1160F53
:1076B000C8D0441CEAE7C5F89870D5F8A020013B73
:1076C00023F01F0302F01F021343D3453146E0B2FB
:1076D000C5F8A030E8D024F063FE10F1160FB1D049
:1076E000C5F89870D5F89C209DF808300BF1FF3B49
:1076F00062F304038DF80830D5F8A0309DF8082017
:107700005B0863F347128DF80820D6E90032134472
:10771000009323F01F035B44A3EB0A03013023F023
:107720001F036946C0B20393FFF734FFBEE700BFF3
:1077300000ED00E0A4280020B60B0400900B04002C
:107740000522044BC3F89420BFF34F8FBFF36F8F14
:10775000704700BF00ED00E0BFF35F8F0022024BD7
:10776000C3F89420704700BF00ED00E010B5034C53
:107770002278FFF72FFF207010BD00BF8B80002004
:107780002DE9F74F294D8A4606464FF00008AB46D3
:10779000274FD0451BDAD6F80490B9F1000F3FD03F
:1077A00031680846019124F0F2FD0199044609EB85
:1077B0000100013824F0EBFD84424FF014021D4B10
:1077C00008D002FB08F36FF015024BF8032003B05A
:1077D000BDE8F08F14F1160F2C60F8D01978A14293
:1077E000F5DD02FB08B0C7F89840C7F89840D7F815
:1077F0009C4000F10801007B64F304000871D7F895
:10780000A0000C79400860F347140C71D7F89C1065
:1078100021F01F016960D7F8A01021F01F01296134
:1078200008F1010814350C36B3E700BF6469002085
:1078300000ED00E08B800020F0B55349534DD1F8A6
:1078400090302C68C3F307239C4287B000F29980E4
:107850000020FFF781FF4E4BC1F8C030844216D1A3
:107860004C4D01A82C70FCF7F5F9002607464A4C50
:10787000B74213D100202B784349D1F89020C2F3AE
:107880000722934277DBFFF75BFF002046E0696841
:1078900001EB0011FFF766FE0130DFE701993001CF
:1078A00001EB0613DA682240B2F1807F52D00AD889
:1078B000B2F5001F34D0B2F5800F3ED0B2F5801F74
:1078C00012D00136D4E7B2F1006F43D0B2F1805F3D
:1078D000F7D15A689B680958013B22F01F00034406
:1078E00023F01F03012032E05A689B680958013BCE
:1078F00022F01F0003440120844623F01F0340EAC6
:107900004C10CDE902218DF8100002A928780593CA
:10791000FFF740FE00282ADA6FF0150007B0F0BD2F
:107920005A689B680958013B22F01F0003444FF03E
:10793000020C012023F01F03E1E75A689B680958F5
:10794000013B22F01F000344062023F01F034FF0E9
:10795000000CD4E75A689B680958013B22F01F00CD
:1079600003444FF0030C012023F01F03C7E72B78DB
:1079700001332B70A5E7C1F89830C1F8A00001339E
:107980007BE74FF0FF30C9E700ED00E0ACC9030032
:10799000AAFF44008B8000200000F0FFF0B587B004
:1079A00007460E4614460021102268461D4632F056
:1079B00011FD02238DF80230054B2A462146684608
:1079C000CDE90476019320F097FD07B0F0BD00BF2C
:1079D000D3C3020008B5024B1B689847002008BDBE
:1079E00078690020F8B50D46094F461EC0F1010424
:1079F000A3199D4201DC2846F8BD73780A2B02D1F9
:107A00000D203B6898473B6816F8010F9847EFE751
:107A100078690020034B044A1860937843F002030E
:107A20009370704778690020301D002008B5064922
:107A3000064821F00701C1F1005202F5802221F031
:107A400079FE002008BD00BF1B8B01207C6900204F
:107A500070B541690446867A0A4D59B1437ADB070D
:107A600006D4302303FB06539B6A1B689B68984728
:107A7000002363613020214600FB0650BDE87040C2
:107A800031F02EBD802C00203022024B02FB003052
:107A9000704700BF802C00203021827A064B01FB0A
:107AA0000233DA6A93F82230801A1B3323F003037F
:107AB000B0FBF3F0704700BF802C002038B53024B5
:107AC000827A064B04FB02339B6AD3E901240C60E3
:107AD0001568FFF7E1FF04FB005038BD802C002043
:107AE0002DE9F04385B00546684690461C46039153
:107AF00032F009FADDE90067EFF31189202383F3FF
:107B00001288BFF36F8F2B8C002B43D0EA8B9A42E5
:107B100025D90022002328461EF06EFC0446F0B151
:107B200089F31188BFF36F8F039B002B43D032463C
:107B30003B46684632F00CFA3021A27A264B2046AA
:107B400001FB02339B6A03A91B681D68DDE9002362
:107B5000A847606180BB2046FFF77AFF26E0298CAA
:107B60004B1E2B8489F31188BFF36F8F95F8223059
:107B7000EA8BEC6A1B3323F00303521A02FB034423
:107B8000154B164AEB1A1B115343A37295F822307A
:107B9000E372C9E789F31188BFF36F8F234642462A
:107BA00028461EF029FC04460028BDD100242046AA
:107BB00005B0BDE8F0836361012300252381039BA9
:107BC00029466382E27A656004F1180032F002FC13
:107BD00063692582E360EAE7802C0020ABAAAAAAA9
:107BE000F8B5002430260F4D00B9F8BD476800F104
:107BF0000802D2E8EF3F591EC2E8EC1FBCF1000FAB
:107C0000F7D1DBB2012BF0D1837AC46006FB0353BA
:107C100044605B6A13B198473846E5E7FFF718FF01
:107C2000FAE700BF802C002000B51622FFF776FC93
:107C3000024B1A504FF0FF305DF804FB0C000000BF
:107C4000132800B508D9FFF769FC0922074B1A5021
:107C50004FF0FF305DF804FB3022054B02FB003390
:107C6000D3E8AF3F002BEED00020F3E70C0000007C
:107C7000481D00203023434330B50D4908330B44E1
:107C8000D3E8AF2F92B1541ED3E8EF5F954204D1F1
:107C9000C3E8EC4FBCF1000FF6D1F1D1012A05D1B8
:107CA0003023584300230A180B50536030BD00BFE7
:107CB000401D002038B504461546FFF7C1FF0130CE
:107CC0000BD0094A59B1302303FB04235B688B4274
:107CD00005D0FFF723FC054B1D50002038BD302395
:107CE0005C431059FAE700BF401D00200C00000063
:107CF0002DE9F041184E90461F4600243546336862
:107D0000984202D1736899420BD00134142C06F1C9
:107D10003006F4D1FFF702FC17224FF0FF340F4B6F
:107D20001A502046FFF78CFF013012D0B8F1000F37
:107D300005D0302101FB04510C31C8F8001017B9EF
:107D40000120BDE8F081302303FB045520353D6060
:107D5000F6E70020F5E700BF401D00200C00000002
:107D600038B504461546FFF76BFF01300DD03023C0
:107D70006343074AD0184068086015B10C331344B8
:107D80002B6030235C43105938BD0020FCE700BF56
:107D9000401D002070B500254FF0FF334FF0FF323B
:107DA000184824F0CCFB184BD3E8AF2F82B1013533
:107DB000142D03F13003F7D1FFF7B0FB17224FF07A
:107DC000FF35124B1A500F4824F0BBFB284670BDFC
:107DD00030246C43D3E8EF0F0130C3E8E10F0029F2
:107DE000F8D10B4E331932515A609A6204F10C00EB
:107DF000304431F0A5FA04F12000304431F03DFD6B
:107E0000E1E700BF2C2A0020481D00200C000000E4
:107E1000401D00202DE9F0413024164644430F4A0E
:107E2000101911514660C362B6B1F368A3B1FFF7F0
:107E300075FB0B4F0C3450F807801319054640F2C0
:107E40000512304624F06CFBB8F15F0F04D0EB59FB
:107E50005F2B08BF45F80780BDE8F081401D00207A
:107E60000C0000002DE9F0410546FFF7E9FE431C38
:107E7000044621D030266E43DFF8488006F10C0717
:107E800047444FF0FF324FF0FF33384624F057FBA2
:107E900008EB06035A68946844B1DB6A58F8060098
:107EA00013F4404F0BD02946A0470446384624F02F
:107EB00048FB2846FFF7DEFE2046BDE8F081A047DC
:107EC000F3E700BF401D0020F0B5EFF3118420233D
:107ED00083F31288BFF36F8F036BDD0707D4FFF7BF
:107EE0001DFB0922464B1A504FF0FF3036E0B1F52A
:107EF000817F46D008D803292DD0042933D0FFF73D
:107F00000DFB5F223E4BEEE740F203139942F6D1A0
:107F1000D2E900329988CD070AD5D0E90A1529435C
:107F2000D98818BF41F00101D9801168143111605E
:107F30009988490723D5D0E90A51023571F1FF31FB
:107F400034BF01200020D98841EA8001D98013681C
:107F50001433136013E044F20200184084F31188D4
:107F6000BFF36F8FF0BD126826490A4204D0FFF7B5
:107F7000D5FA1622224BB6E70B40134303630020C9
:107F8000ECE79168D2E90053AA88D7071BD51A6895
:107F9000914204D1FFF7C2FA0C22194BA3E7012743
:107FA00010611A68567B67F3050656731E68B27B2C
:107FB00022F02002B2731E68F26822F4FE12F26010
:107FC0001A6814321A60AA885607D8D51A689142DE
:107FD000E0D01030106101201A68517B60F3050178
:107FE000517319688A7B22F020028A731968CA6863
:107FF00022F4FE12CA601A6814321A60BFE700BF8A
:108000000C000000FDBFFFFF002373B50546CDE95E
:10801000003331F036FC044648B1FFF77FFA0B22FB
:108020004FF0FF34194B1A50204602B070BD6A461B
:108030002846174901ABFFF75BFEEFF311862023BB
:1080400083F31288BFF36F8F2B6BDB070ED4FFF720
:1080500065FA09224FF0FF340C4B1A5086F3118851
:10806000BFF36F8F01981EF0D3FCDDE7094B0A4A7E
:10807000EB1ADB105A430121084822F0EAF90022EA
:1080800000232C63C5E90A23E8E700BF0C000000C9
:10809000F0C9030040370020B76DDBB60021002097
:1080A0002DE9F3411E460023072A04460D46CDE97B
:1080B00000330BD961B90E23FFF730FA4FF0FF34CC
:1080C0002F4A1350204602B0BDE8F0811623F3E793
:1080D000EFF311874FF0200888F31288BFF36F8FFA
:1080E000036B5B040ED5B047002846DA4342FFF726
:1080F00015FA4FF0FF34224A135087F31188BFF36B
:108100006F8FDFE731F0BDFB08B10B23EFE76A4665
:1081100020461C4901ABFFF7EBFD87F31188BFF345
:108120006F8FEFF3118788F31288BFF36F8F2946A3
:108130002046B04710F10B0F02460FD0D8B1FFF721
:10814000EDF94FF0FF340E4B52421A5087F311886D
:10815000BFF36F8F01981EF02BFCB3E787F31188F4
:10816000BFF36F8FDDE900104FF0FF324FF0FF33A8
:108170001EF084FCD5E70824E8E70824BDE700BF2B
:108180000C000000F0C90300014BFFF789BF00BFDE
:108190004BC50200014BFFF783BF00BFB9C502000A
:1081A0002DE9F34721F4804727F0020780468946EE
:1081B00057B1FFF7B3F91622214B1A504FF0FF3594
:1081C000284602B0BDE8F08701211E4801AA22F02E
:1081D000DAF8002804DAFFF7A1F90C22184BECE7D3
:1081E0003823019CDFF860A05C43FFF7D3FD051E38
:1081F00004EB0A0605DA0121019A124822F029F956
:10820000DCE749F001031034C6E90A8733635444BC
:10821000204631F0F1FF304631F0EEFFB8F1000FAB
:1082200003D0394630461FF04DFD002120461FF097
:1082300049FD002331462846044AFFF7EBFDBFE71E
:108240000C0000000021002040370020F0C903008E
:10825000002337B50D4609221349CDE90033FFF756
:1082600029FD0446E0B16A460F4901ABFFF740FD26
:1082700000984FF0FF324FF0FF331DF0FBFF082254
:1082800029462046094BFFF70BFF044600981EF0D5
:1082900063F801344FF0FF3018BF002003B030BD49
:1082A0004FF0FF30FAE700BFF0C90300B9C5020084
:1082B0001FB5CDE90023002309221349CDE902337C
:1082C000FFF7F8FC0446E0B10F4903AB02AAFFF741
:1082D0000FFD02984FF0FF324FF0FF331DF0CAFF41
:1082E000082269462046094BFFF7DAFE0446029849
:1082F0001EF032F801344FF0FF3018BF002004B0F8
:1083000010BD4FF0FF30FAE7F0C903004BC5020083
:108310002DE9F04F0026B146F3B0CDE9050108A8DC
:1083200014461D4631F0EFFDDDE90823DDE9057A4D
:10833000CDE902230EAB0B9304960DF13408BAF18C
:10834000000F22D1B9F1000F6ED0B5F1FF3F08BF89
:10835000B4F1FF3F65D04FF47A71A4FB010447F6F6
:108360001222002301FB0541F9F7C2F8069B3146B2
:10837000019000934FF48272059B049824F04CF90D
:108380000646304673B0BDE8F08F3868002844DBFD
:108390000DF1300B42465946FFF7E2FC07900028EA
:1083A0003BD0D8F800004FF0FF324FF0FF331DF004
:1083B00061FF72AB01930BAB009307993B464FF4FF
:1083C0008172DBF8000024F027F910F1780F0346E2
:1083D000079915D10023002208A831F094FDDDE9AA
:1083E0000834CDE90234002425462346D8F800009D
:1083F00007931DF0B1FF079B002B0EDA5B4234E0C0
:1084000010F1120FF2D1049B1BB90E46DBF80030BD
:10841000049300234FF00109E8E708370AF1FF3A17
:108420008DE74FF0FF30A1E7DDE9022308A831F026
:108430008FFDDDE9084522462B460BAF0DF13808CC
:1084400039683848A1EB08018910414340461FF0C4
:10845000E1FB00F10B020B2A06D840F68103D34062
:1084600013F00103049307D14342FFF757F82E4A54
:108470004FF0FF36135084E70025DDE905492E460D
:10848000C7F800800DF1340A0DF1300BB9F1000F7F
:1084900011D1002D3FF475AF002E3FF772AFDDE92B
:1084A000022308A831F054FDDDE908452B46254399
:1084B0002246C5D165E74FF000032068E38000281D
:1084C0002ADB52465946FFF74BFC18B92023E380BC
:1084D000013621E00790DAF800004FF0FF324FF04C
:1084E000FF331DF0C7FE0097234640F203120799A1
:1084F000DBF8000024F090F80790DAF800001DF097
:108500002BFF079B13F10B0F0AD0002B7FF476AFE4
:10851000B4F90630002BDBD1083409F1FF39B5E797
:10852000049DF9E7CDCCCCCC0C00000008B5244A62
:10853000244B1A6016F0A0FB4FF47A612248D0F861
:108540002436C3F30802C3F309434B4382F4807219
:108550001E49883201FB02334FF4FA215B00B3FB62
:10856000F1F201FB12331A49B3F57A3F28BF013209
:10857000C1F80429D0F820364FF47A60C3F308021A
:10858000C3F30943434342F21C5082F4807202F267
:10859000172200FB02334FF47A701B0AB3FBF0F290
:1085A00000FB12330020B3F5FA7F4FF0010328BF20
:1085B0000132C1F81C27C1F80009C1F8003608BD16
:1085C0000020A1077827002000C0FF00F82A0080C3
:1085D0000000125048B1054B054A1B68B3FBF2F38B
:1085E0005843044B43F00103184770477827002095
:1085F00040420F0080C003000268064B1A604268C8
:10860000054B1A608268054B1A600269044B1A60B8
:10861000704700BF94690020906900208C69002099
:108620009869002038B50025074C204630F088FEB8
:1086300004F11400013531F020F9052D04F1240472
:10864000F3D1002038BD00BF9C69002038B500245C
:10865000054D2846013431F010F9052C05F10C05C3
:10866000F7D1002038BD00BF506A002038B5002483
:10867000054D2846013430F063FE052C05F1140544
:10868000F7D1002038BD00BF8C6A00200B4B30B5FD
:108690001C4600250A4A191BB1F5806F01D900203C
:1086A00030BD506803F1D801C3E93620016003F5FD
:1086B000807303F8045C5160EDE700BF7837002059
:1086C00000220020F7B506460D461446124F3846E4
:1086D00030F0AFFCE0B1BB68314638461B68AAB247
:1086E0009847002802DB002003B0F0BD002CFBD12E
:1086F000AC42F8D22F1B042F28BF042730F046F9D4
:108700003A46019001A9301931F03EFE3C44EFE7B2
:108710006FF01200E8E700BF08AB030010B5094C8A
:108720000A44914200D110BD11F8013B584000F0BD
:108730000F03E35C83EA101303F00F00205C80EA70
:108740001310EEE70D9404007FB5124E124D4FF05A
:10875000FF334FF0FF32114801A91DF027FD0346FA
:10876000A8B12A685207F2D0012128460C4A22F00B
:1087700084F9ECE7236813B1019A934203D1D4E959
:10878000013101A898470C34B442F3D3DFE7054C1C
:10879000FAE700BF78BA03007C280020902B002065
:1087A0006D0C040078BA0300F0B517461E4685B07C
:1087B00001909DF82800DDE90C5423462C432A46FD
:1087C0008DF808008DF80910ADF80A70039608D0EE
:1087D000FEF7A4FE0E49D1F8D0400E4909588C424C
:1087E00001D1002213460C4801A930F069FD041E96
:1087F0000BDA0A48036813F0060F03D00221084A77
:1088000022F032F9204605B0F0BD0024FAE700BF9F
:10881000A063002008000000902B00207C2800208E
:10882000820C0400F8B590F8DC300446012B00AF50
:1088300004D0022B32D00020BD46F8BD026EB0F845
:10884000B83051681801B4F8DE2001EB0313095861
:108850009D881144AA1A96B23246206824F019FD68
:10886000031E21DCE7D0164802685207E3D06C46AD
:108870008AB0144A089305924FF40073124AADF877
:108880002430CDE906266A46104B42F8103F0023FB
:108890004FF43151FAF74AFFA546CCE7B0F8DE2095
:1088A000416B058F1144D5E7B4F8DE2013449BB229
:1088B0009D428CBF00200120A4F8DE30BCE700BF41
:1088C00098280020BA0C0400D60C04000500000112
:1088D000F8B50D46044600AF002850D0026E002ABD
:1088E0004DD0C9B12B480129036803F0060348D1D4
:1088F00093B16E4688B013686A462749C2E90513EA
:108900004FF400739383254B42F8103F00234FF43C
:10891000E451FAF70BFFB546236E5B691BB129469C
:10892000204662689847D4F8202100233AB1B4F871
:108930002821012A9CBFC4F82031A4F82431C4E9BD
:1089400013332366A36504F1780030F050FF04F17F
:10895000E00030F001FF04F1F00030F048FF04F1D6
:10896000BC03D3E8EF1F21F00101C3E8E21F002A96
:10897000F7D184F8C05004F1C4001DF071FDBD466C
:10898000F8BD002BC8D06E4688B013686A4604490B
:10899000B4E700BF98280020DF0C040003000001AA
:1089A000EB0C04002DE9F04FA0F59674A0F58E7144
:1089B00005462022206885B024F085FC002840F37D
:1089C0004C814FF0000847462086228E1FFA88F31C
:1089D0009A4205D8284605B0BDE8F04F1DF03ABFD1
:1089E00014FA88F31A7C0023B4F84010DEB28E42E9
:1089F00013D3E389A189994217D19948036813F0E9
:108A0000060F03D0974A022122F02EF8E7816787EC
:108A1000A4F84A70C4F8207104E0E06B0133805D73
:108A20008242E3D108F10108CFE7B4F84A00B4F874
:108A30004810884206D18A48036813F0060FE5D033
:108A4000894AE0E7A168CA54E389B4F838B05E1CEB
:108A5000B6B25E450093E68170D3D4F80890A6EBD9
:108A60000B0A5A46616B09EB0A0031F0BFFC002883
:108A700064D15E45CAD0D4F820316BBB4FF0140EE0
:108A800009F80A30A5F1D600C5F1C80C002230F86B
:108A9000026F91B2B14204D301339BB2032BB5D024
:108AA000F4E75CF810100EFB021191F8049001320B
:108AB000B9F1000FEDD1A4F828316C4A636CC4F809
:108AC00020111A60636CA2685A600223A4F84A302D
:108AD000204623F05EFE99E7B4F82631002BF7D04C
:108AE000626CB4F84A10AAEB030A09EB0A0342F8D5
:108AF0002130228FE3899B1AA268D054B4F84A30FF
:108B00000133E3E7626B0133515CA268324412F82F
:108B1000012C8A4286D0D9B25945F3D355F80C2C92
:108B2000A5F5967362B9C5F1C801A5F1D60A0391FE
:108B30003AF8021F4FF0000E029168E00023EAE7C6
:108B4000002092F80CC081B261456BD30021B3F8CC
:108B5000262100297FD0B3F84AC0586C002A6DD175
:108B6000424A40F82C20B3F84A200132A3F84A20A8
:108B70000022A3F8262155E71420039951F81A1072
:108B800000FB0E1999F804108E4201913DD14FF06F
:108B9000000C9968DDF804B01FFA8CF0834522D8E8
:108BA000A4F82821009AA389023292B29B1A0B449E
:108BB0001846A4F82421C4F82091013A31F0E4FBCE
:108BC000B4F84A10626C42F82100A289A3681344E9
:108BD000002203F8012CB4F84A30A4F8262101330E
:108BE000A4F84A301EE7D9F8000011F80CB010F8CC
:108BF0000C00834506D099F80DB0BBF1000F04D0EE
:108C00003F2802D10CF1010CC4E70EF1010E0298CD
:108C10001FFA8EF18842AFD8013292B2032A3FF494
:108C200001AF85E7916811F800E09968013031449F
:108C300011F8011C714586D1012188E79968B21AA3
:108C4000013A114440F82C10D9899A680A4400214D
:108C500002F8011C87E701328BE705B0BDE8F08F11
:108C600098280020F90C0400100D0400EC670400A3
:108C700038B50D4604464FF4A072002131F0AAFB2E
:108C80002B6863606B68A3602B89A381EB696364C5
:108C90002B8CA4F84830EB6863632B7C23876B69CB
:108CA000E3632B7EA4F840306B6A63652B8D00254F
:108CB000A4F85C3004F1BC03D3E8EF2FC3E8E15F14
:108CC0000029F9D10122294604F1C40030F05EFCEC
:108CD00004F596700E4930F004FD04F168000D496A
:108CE00030F0FFFC04F178000B4930F072FD04F124
:108CF000A8000A4930F0F5FC04F1E000084930F022
:108D0000F0FC04F1F000074930F063FD284638BD5F
:108D1000A589000005C8020025C7020015C702008A
:108D20005BC8020083C70200024608B51368084604
:108D30008B4207D000231160D3815387A2F84A30B9
:108D4000C2F82031024924F07EFA002008BD00BF9D
:108D5000FDC6020070B5036806460D46A3B349B3CD
:108D60004B683BB30A8912B91A498B4222D1298A2E
:108D700009B9E968D9B903EB02129A421DD106F18B
:108D8000BC02D2E8EF3F43F00101C2E8E01F002837
:108D9000F7D113F001041AD106F1C4001DF0C2FB93
:108DA000756606F168001DF055FD204670BD0A4845
:108DB0008142E0D06FF01500F8E7998811B9D968C1
:108DC0000029F7D01033D8E74FF0FF30EEE76FF00F
:108DD0000F00EBE700CA030000CA030010B5044609
:108DE00018220021043031F0F5FA014B236010BD48
:108DF000EC67040038B50446037809480D46037053
:108E0000637843706278012A04D95208A11C0230A9
:108E100031F0BAFA637802485B0802332B8038BD20
:108E20008C80002010B504460648036813F0060F36
:108E300003D00221044A23F06BFE00232374E36471
:108E400010BD00BF9C2800202F0D040001780246B1
:108E5000CB0705D563294FEA910305D8032B01D829
:108E600000207047204905E0203303F03F03182B12
:108E7000F6D81E4921FA03F3D807F1D55378D9075C
:108E8000EED5072BECD8580813789B08202B17D069
:108E900009D8082B19D0142B20D0042B22D0B0FADB
:108EA00080F040097047342B1AD0382B13D0242B74
:108EB000F5D1012818BF08280CBF012000207047F9
:108EC000082814BF002001207047013802288CBFF9
:108ED00000200120704702380128F8E70228F0E757
:108EE00000F07D000128ECE71001110111011101D2
:108EF00073B5044600F12C064FF0FF324FF0FF33FC
:108F000030460D4623F054FEA38CA28BD21AA36ADE
:108F10009B1A9BB20A2B0ED8304623F0C4FE0D4894
:108F2000036813F0060F03D002210B4A23F0F0FD73
:108F3000002002B070BD2A896846696823F0B3FD3D
:108F40002946204623F051FE304623F0ACFE012096
:108F5000EFE700BF9C2800203D0D040070B590F89D
:108F60006630054686B0A0F58C74002B58D0D4E945
:108F7000580123F089FD002852D0237B022B3AD1DF
:108F80000321204623F091FE94F880616EB1042104
:108F9000204623F08AFE94F87F31002B40D02068D1
:108FA00006B0BDE8704024F0B7B940F243130DF1AC
:108FB000020101A801938DF80860FFF71BFFA37B56
:108FC0000490C3F340038DF80D304EF60173ADF8F5
:108FD0000E30BDF80230204603A9ADF814308DF8EC
:108FE0000C60FFF785FF002328460E4A06B0BDE857
:108FF00070401DF0D7BC032B12D10B48036813F04F
:10900000060F03D00221094A23F082FD20460221E7
:1090100023F04BFE204606B0BDE8704023F0AEBD05
:1090200006B070BDB4C404009C280020510D04009B
:1090300070B5B0F848500446052D86B00BD91948D4
:10904000036813F0060F2BD00221174A06B0BDE8C3
:10905000704023F05DBD006C616C03AB03C3A06C7A
:1090600001AE1860616C2A46304631F08DF99DF8EA
:10907000040023F0F9FC00F0FD008DF8040003A9C2
:1090800020460496ADF81450FFF732FF40B905486A
:10909000036813F0060F03D00221034A23F038FDC2
:1090A00006B070BD9C2800207D0D04008B0710B514
:1090B000044601D5FFF7BCFF237B072B0CD0022B06
:1090C0000FD01048036813F0060F19D0BDE8104008
:1090D00002210D4A23F01CBD2046BDE8104023F0BC
:1090E000ECBD2046072123F0E0FD0323637304F168
:1090F000E80040F63542BDE8104000231DF01ABCE0
:1091000010BD00BF9C280020A00D040010B504462F
:1091100086B0002843D094F8302050F85C0C032A25
:1091200017D1437B0133DBB2032B437318D91D489E
:1091300003685B0706D034F8603C012100921A4AAC
:1091400021F0A5FCA4F1880006B0BDE8104023F092
:10915000E1BC022A23D1032384F830300023437377
:1091600034F8603C03A98DF80C3054F85C3C9B7BD0
:10917000C3F340038DF80D3044F20133ADF80E30E7
:1091800000230493ADF81430FFF7B2FE40F63542E9
:109190000023204606B0BDE8104023F00BBD06B00A
:1091A00010BD00BF9C280020B60D040030B5044659
:1091B00087B0002853D050F82C5C284623F0A3FD3C
:1091C00040B942F29F420023204607B0BDE830403C
:1091D00023F0F0BC94F8601001291BD154F82C2C1A
:1091E000537B0133537354F82C3C5B7B032B1DD909
:1091F0001C4803685B0706D034F8303C0322009219
:10920000194A21F044FCA4F1580007B0BDE83040F1
:1092100023F080BCB4F8603023F49F6323F007038D
:1092200043F00103A4F8603000236B7334F8303C42
:1092300054F82C0C8DF80C30837B03A9C3F3400346
:109240008DF80D3042F60173ADF80E300023049313
:10925000ADF81430FFF74CFE40F63542B3E707B0E7
:1092600030BD00BF9C280020DC0D040070B5044612
:1092700098B310F8AC1CA0F1B805012914D110F86E
:10928000AB3C0133DBB2032B00F8AB3C19D91348DC
:1092900003685B0703D00323114A21F0EEFB284645
:1092A000BDE8704023F009BD0121284623F0FDFCF4
:1092B00014F8AA3C43F0020304F8AA3C002304F883
:1092C000AB3C28460749FFF713FE2046BDE8704037
:1092D00040F63542002323F06DBC70BD9C28002071
:1092E000010E040000CA03001FB5037B0446042BD3
:1092F00037D1062123F0D9FC94F87F31D3B14FF058
:10930000FF334FF0FF32206823F067FF031E11DAAE
:1093100024480268520703D00121234A21F0ADFB03
:109320000021204623F0C1FC0121204623F0A1FBAF
:10933000012019E094F8803123B10221204623F066
:10934000B4FC10E00023194A684630F0DCFDDDE98A
:109350000023C4E9562305221549206823F099FF0C
:10936000E6E7062B02D0002004B010BDD0E956017C
:1093700023F08AFB58B10B4803685B0703D0012137
:109380000C4A23F0C5FB204623F097FCD0E7237C52
:10939000012BD2D0F92301228DF80F300DF10F01EE
:1093A000DBE700BF9C280020290E0400B4C40400A1
:1093B0001D9404004E0E04002DE9F04F044685B0C4
:1093C000A0F15C094FF0FF334FF0FF3200AFA0F186
:1093D0008808484623F0ECFB14F87C3C032B04D0AF
:1093E000052B02D0404623F0C9FBA4F1700AA4F17A
:1093F000660B404634F8666C34F86A5CFFF774FF1D
:10940000786030B1484623F04EFC1437BD46BDE8C5
:10941000F08FAE423ED034F8662C34F86A3C5946A0
:109420009B1A9BB207F10C02504621F0CFF9F96864
:109430000246054654F8880C23F02BFF061E21DA5D
:109440007A685946504621F0F7F9721CDAD01B4869
:1094500002685307D6D06C468AB06A464FF4007350
:109460001749ADF824300591164B17490896CDE9F8
:10947000061542F8103F4FF431517B68FAF756F960
:10948000A546BFE732465946504621F0D5F9AE42CF
:10949000AFD2B7E714F87C3C052B0AD10421404633
:1094A00023F003FC94F8F7301BB154F8880C23F038
:1094B00033FF404623F055FBA4E700BF9C28002063
:1094C000BA0C040005000001D60C04002DE9F04F91
:1094D000A0F1580691B0044602AF304623F04EFB8F
:1094E000DFF8609254F8443CB4F81C21D4F8181109
:1094F000D21A194454F8580C23F0E5FE031E0CDC74
:1095000007D090480268520703D001218E4A21F00B
:10951000B4FA3C37BD46BDE8F08F54F8448C434460
:1095200044F8443C54F8442CD4F81801424514F84B
:10953000483C08DC012B00F20D84002344F8443C35
:1095400044F80C3CCEE710F8085000EB08020A2B58
:109550001CD8DFE813F00B001E004B001B005D0061
:1095600081009400BA00C500D30001010023F92D49
:1095700044E9063344F8103C24F8083C44F80C3C19
:1095800004D1012304F8483C24F8083C08F1010800
:10959000C8E7F92D2AD134F8083C013324F8083CF7
:1095A00014F84C3C042B0ED134F8083C032B12D990
:1095B000F923012254F8580C07F12C0187F82C30BC
:1095C00023F067FE07E0022B05D1D6E9560123F010
:1095D0005BFA0028E8D114F84C3C062BD6D10022C7
:1095E000002304F130001DF0DDF9CFE74FF0010357
:1095F00024F8083CC5F3400304F8173C4FF004037B
:10960000AD0844F80C8C04F8185C04F8483CBDE73D
:1096100034F8083C013324F8083CC5F3001305F086
:10962000EF050F2D04F8163C04F8155C09D825B198
:1096300048F22A23EB40D9070AD43046FFF7F2FB61
:10964000A4E7632D04D005D82F2D01D0432DF4D1EC
:109650000523DAE7EF2DFAE734F8083CEA0703F1CF
:10966000010324F8083C4FEA550324F8103C01D4C8
:109670000623CAE70BB90923C7E70723C5E734F870
:10968000083C013324F8083C34F8103C43EAC51385
:109690007F2B24F8103C09D9D9F800305B07CCD0D7
:1096A00001212A4A274823F033FAC6E7B4F81C21DF
:1096B0009342E2D9D9F800104D07BED001210092A3
:1096C0002048234A21F0E3F9B7E734F8103C1BB1F6
:1096D00014F8153CEF2BB0D1082344F8142C94E770
:1096E00054F80C2C34F8103C134434F8082C134470
:1096F0009845FFF64BAF092304F8483C54F80C1C7E
:1097000034F8082C0144FF20FFF708F814F8152C52
:10971000EF2A0DD1C343DBB29D4211D0D9F800200E
:1097200012F0060F89D0022148460A4A0095C9E77F
:1097300034F8102C54F8141CFEF7F0FFC343EAE78A
:109740000A2362E79C280020E30F04006B0E04004C
:109750007B0E0400B90E0400F92D7FF46EAF14F8EF
:109760004C3C03F0FD03042B03D10221304623F0CF
:109770009CFA14F8183C14F84C2C002B40F0BC81D7
:10978000022A08D114F84A3C14F8171CC3F340030A
:10979000994200F08D8014F8153C632B3DD01FD802
:1097A0002F2B00F05381432B00F07681C5480268CF
:1097B00012F0060F7CD06D468AB002AAC2495161F0
:1097C000C249C2E906134FF400731384C04B42F838
:1097D000103F00234FF41251F9F7A8FFAD4667E0A0
:1097E000EF2BE3D1012A63D954F814AC34F810BC40
:1097F00007F114005A46514623F055F907F11400B9
:10980000FFF724FB80BBAF48036813F0060F4FD06F
:10981000B04A022123F07CF94AE0012A48D1022112
:10982000304623F042FA14F84A3CA4F12C0543F0E8
:1098300002034FF0FF32284604F84A3C4FF0FF3352
:1098400023F0B6F914F84A3C284643F0010304F823
:109850004A3C23F028FA04F160002FF0C8FF0021F1
:10986000304623F006F923E0397D88074FEA91035B
:1098700020D4102B05D0302B1AD13046FFF716FC20
:1098800016E0A4F12C054FF0FF334FF0FF322846CD
:1098900023F08EF90421304623F007FA284623F0FE
:1098A00002FA94F827311BB154F8580C23F034FD18
:1098B0000023AAE6282B00F0868030D8102B00F079
:1098C000B180182B00F09880A4F1180307F12C0543
:1098D00093E8070085E8070007F11C005A46514647
:1098E00023F0E1F807F11C00FFF7B0FA00288AD056
:1098F00040F211337B62002387F828303B7F07F169
:10990000120107F1240087F82630FFF773FA7B8AEB
:10991000386329463046BB86FFF7EAFAC8E7302BA2
:10992000ABD0382BD0D13046FFF782FB7B7D5B0874
:109930009A1E012A09D96348026812F0060FB7D0AF
:109940000221654A21F099F8B2E7B968FA7DBB7D3A
:1099500002F0CF0201F030010A4354F8545C9B0836
:109960003A72002DA4D0298D994201D02D68F8E7D4
:1099700002F00A02B2F1080018BF012095F8B930D0
:1099800003F00101884205D0082A14D043F00103F6
:1099900085F8B93095F8B930590789D495F8B820C9
:1099A000022A85D143F004032946304685F8B930B0
:1099B00023F077FA7CE723F0010385F8B930281DFE
:1099C00023F0E5FCE6E7A4F12C054FF0FF32284632
:1099D0004FF0FF3323F0ECF814F84A3C284643F0EC
:1099E000010304F84A3C23F05EF93046FFF720FB00
:1099F000304623F0B6F85BE7A4F12C054FF0FF32B8
:109A000028464FF0FF3323F0D3F814F84A3C284699
:109A100023F0010304F84A3C23F045F93046FFF7F0
:109A200007FB45E7A4F12C054FF0FF324FF0FF3361
:109A3000284623F0BDF80521304623F036F930469C
:109A4000FFF7F6FA284623F02EF931E7022A3FF411
:109A50002FAF072A3FF42CAF14F84A3C022123F021
:109A6000020304F84A3C304623F01FF9A4F12C0508
:109A7000304623F08AFA28464FF0FF324FF0FF338A
:109A800023F096F814F84A3C284643F0010304F802
:109A90004A3C23F008F9E2E6304623F076FA14F85F
:109AA0004C3C072B09D0022B1AD00648036813F050
:109AB000060F3FF4FDAE094AABE6304623F0FDF851
:109AC000F6E600BF9C2800200F0F04005456040047
:109AD00004000001DE0E0400EE0E0400A00D0400E0
:109AE0003046072123F0E1F840F63542002304F127
:109AF00090001CF01FFFDBE6022A7FF4D9AE54F879
:109B0000545C65B9AB48026812F0060F03D002211D
:109B1000A94A20F0B2FF304623F04EFAC8E62A8D5B
:109B20009A4201D02D68ECE714F8151C432900F087
:109B3000FB8021D80F2900F09F802F2900F0D080D2
:109B40009C48026812F0060F3FF4B2AE6D468AB030
:109B500002AA13624FF40073DFF860C29384C2F864
:109B600014C0974BDFF85CC2C2E906C142F8103F4F
:109B700000234FF432512FE663296DD0EF29DFD156
:109B800095F8B830022B7FF493AE95F8B930D5F83C
:109B90002CA0C3F3400305F1440B4FF0FF325846AD
:109BA000FB604FF0FF3323F003F8DAF84410BAF803
:109BB000482005F1300020F058FE7860584623F028
:109BC00072F8BAF848107B688B421ED27948026856
:109BD000520714D0EB468AB0B5F828C002AACB1AB7
:109BE000C2E907310523DFF8E0E1C2E905EC42F8FC
:109BF000103F00234FF42151F9F798FDDD4695F809
:109C0000B93043F0020385F8B930AA8FAB8E9B1AA6
:109C10002A6C9BB2D21A1F2A0FD86648036813F029
:109C2000060F04D02B8D0221684A20F026FF95F8FC
:109C3000B93043F0020385F8B93095F8B930FA68C5
:109C4000C3F34003934203D02946504623F029F939
:109C5000281D23F090FB2BE6EA6A937B92F84120C3
:109C6000C3F340039A427FF423AE95F8B830012B3A
:109C700006D0032B7FF41CAE284622F04BFF17E6DC
:109C80000223281D85F8B83023F059FB05F1440A5A
:109C900005F158002FF0ABFD4FF0FF324FF0FF33CE
:109CA000504622F085FF00235046C5E90D33EB6393
:109CB00022F0F9FFE86A837B13F0020309D02946FA
:109CC00023F0EFF895F8B93043F0040385F8B93084
:109CD000EEE595F8B92063F3820285F8B920E7E54F
:109CE000E86A23F052F995F8B830022B3FF4E0AD62
:109CF000B5F8B830281D23F49F6323F0070343F021
:109D00000203A5F8B83005F1440A23F018FB4FF020
:109D1000FF3350464FF0FF3222F04AFF00235046F7
:109D2000C5E90D33EB638EE6D5F82CA0504623F041
:109D30002CF995F8B830022B05D0BAF1000F3FF49A
:109D4000B7AD5046E8E60023281D85F8B83023F06B
:109D500006FBADE5062A7FF7C5ABB4F81C1154F835
:109D60000C3C85398B42FFF6BDAB00EB0308D21AE1
:109D7000414654F8145C30F014FB54F8443C54F859
:109D80000C2C9B1A44F8443C002344F80C3C54F837
:109D9000143C002B3FF4A6AB14F8483C072B81BFC2
:109DA000D4F81831A5EB08055B1944F8143CFFF70B
:109DB00099BB00BF9C280020280F0400BA0F0400A4
:109DC00005000001DE0F0400510F04008D0F040098
:109DD000F0B50C4605468DB068460022002330F0F1
:109DE00092F8DDE900670FCC0DF1080CACE80F002C
:109DF0000FCCACE80F0094E803004FF4C8728CE875
:109E000003000021284630F0E5FA05F5B474C5E9F1
:109E1000566702AE0FCE0FC40FCE0FC496E80300F4
:109E200084E80300D5F87831B5F87C21AB61AA62EB
:109E300005F12C002FF084FA05F1580010492FF09D
:109E4000C8FC05F188000F492FF0C3FC05F1B800EC
:109E50000D492FF0BEFC05F1E8000C492FF0B9FCCC
:109E60000B4905F58C702FF0B4FC05F5A47030F0AB
:109E70002EFA002128460DB0BDE8F04022F015BFB3
:109E8000CD940000B99300006D920000DFCF020076
:109E90005D8F000070B50C46064615460021C022B5
:109EA000204630F097FAE6622B7823856B682A8982
:109EB0002363226404F14400251D2FF041FA0E4A69
:109EC0002146284623F081F90C4904F158002FF06F
:109ED00080FC0B4904F188002FF07BFC0022E36A30
:109EE00084F8B82022609A681AB9C3E90144284668
:109EF00070BD14609C60FAE70CCA0300AD910000CD
:109F00000D91000038B5044625680846CDB921609A
:109F10002246C4E907550C496562257423F093F97C
:109F2000EFF31182202383F31288BFF36F8FA37B9B
:109F300043F00403A37382F31188BFF36F8F2846A5
:109F400038BD6FF07700FBE7B9CB02002DE9FF4188
:109F5000044630F85C2C50F8641C50F8580C23F080
:109F6000B2F9071E40F3F0800026DFF8E48154F8D0
:109F7000643C9D5D14F8543C062B27D8DFE803F0C1
:109F8000323F494E74D5040014F8532C531C18F872
:109F90000220DBB2AA4204F8533C20D10E2B15D18B
:109FA0006C48036813F0060F03D002216A4A20F0C0
:109FB0005BFD002304F8543CA4F16803D3E8EF1FD1
:109FC00041F00201C3E8E21F002AF7D10136B7428F
:109FD000CDD1204604B0BDE8F0411CF03BBC0023CD
:109FE00004F8543C0D2D06D1062304F8543C0123FB
:109FF00004F8533CEAE77E2DE8D1012306E07E2DEC
:10A00000E4D00D2DF0D0FF2D26D1032304F8543CCD
:10A01000DCE7032385F0200504F8543C7D2D01D1B5
:10A020000223F3E7032D17D100220023CDE90023FB
:10A0300000234FF480711A4654F8700C0DF0F0FCB8
:10A0400044F8500C50B94348036813F0060F03D08E
:10A050000221424A20F008FD0023D7E7042304F838
:10A06000543C27F0DAFBB1E77E2D54F8500C23D195
:10A07000022127F0B7FB54F8502C92F83F3043F000
:10A08000400382F83F3054F8501C54F8700C24F010
:10A0900063FE00280CDA2F48036813F0060F03D084
:10A0A00002212F4A20F0E0FC54F8500C27F029FB45
:10A0B000002344F8503CA0E727F04DFB012802465E
:10A0C0001CD100200021CDE900014FF4807154F82B
:10A0D000500C0DF057FC002810DA1E48036813F0EE
:10A0E000060F03D01F4A022120F0BEFC54F8500C8A
:10A0F00027F007FB002344F8503C87E77D2D01D172
:10A10000052383E7012254F8500C0DF10F018DF85F
:10A110000F5027F059FD0028BFF658AF0D480368CF
:10A1200013F0060FE2D0104ADDE7012254F8500C7C
:10A1300085F020050DF10F018DF80F5027F044FD3B
:10A140000028EBDB042361E704B0BDE8F08100BF29
:10A1500007100400A028002016100400321004008C
:10A1600056100400751004008C1004002DE9F74F00
:10A17000044650F8380C38B900220023A4F11C0022
:10A180001CF03AF944F8380C34F82A2C34F8263C00
:10A190009A420CD1002324F8283C24F82A3C24F8C5
:10A1A0002C3C24F8223C24F8243C24F8263C0028AB
:10A1B00000F01D8114F83C3C13B9012304F83C3C29
:10A1C00034F8242C34F82C3CA4F130099B1A54F8B0
:10A1D000202CA4F12C0A9BB2D31A514601AA48465E
:10A1E00020F0F4FA804654F8600C019D23F03FFD06
:10A1F0004FF0000B0746C34580F0E58014F83C2C77
:10A20000A8EB0B06013A032A00F2DD80DFE802F03A
:10A210000228A4AC032E40F2D68054F8380C27F064
:10A22000FCFA7E227D2005F80B20FF2205EB0B01B6
:10A230004A70887023210BF10302A95443F6E352BC
:10A2400024F8342C54F8382C0BF1040B92F83F20EE
:10A2500012F0400F14BF0322022204F83C2CCAE77C
:10A26000032E40F2B08054F8382C92F83F20C2F30D
:10A27000C202012A3FD0022A3FD07248026812F07F
:10A28000060F03D00221704A20F0EEFB00260022C8
:10A290000DF103018DF8032034F8340C012222F073
:10A2A000FDF9F6B201220DF1030124F8340C8DF80A
:10A2B000036022F0F3F917F001011CBF7D22202179
:10A2C00024F8340C1CBF05F80B200BF1010B05F82A
:10A2D0000B10384631460BF1010223F0A6F828B1E5
:10A2E0007D2186F02006A9540BF1020202F1010B38
:10A2F000AE540322B1E72126C9E75726C7E7012E4E
:10A3000061D901220DF1020154F8380C27F0F6FA58
:10A310009DF802200DF103018DF8032034F8340C70
:10A32000012222F0BBF99DF8022024F8340C1146DA
:10A33000384623F07AF850B14FF07D0382F02002C6
:10A3400005F80B30013E8DF802200BF1010B05F8EA
:10A350000B20013E0BF1010B54F8380C27F041FBA8
:10A360000028CCD1042278E7042E2CD934F8342CE0
:10A370003846D24392B25FFA82F824F8342C414630
:10A38000120A23F052F830B17D2188F0200805F838
:10A390000B100BF1010B1146384605F80B800BF141
:10A3A000010623F042F828B17D2182F02002A95550
:10A3B0000BF10206AA557E2206F1020B2E447270A2
:10A3C000002204F83C2C5A465146484620F034FA04
:10A3D00014F83C3C5BB954F8380C27F092F9002291
:10A3E0000023A4F11C001CF007F844F8380CA4F179
:10A3F0003007A4F1260806E02A464146384620F0F8
:10A400001BFAB5421AD334F8262C34F82A3C9A4267
:10A4100014D09B1A41469BB201AA384620F0D6F9C7
:10A4200001990246064654F8480C22F032FF051EF8
:10A43000E2DA00224146384620F0FEF903B0BDE8DA
:10A44000F08F00BFA02800209E100400024638B5FF
:10A45000084602F10804D4E8AF5F15F0010512D1F7
:10A4600091611577094922F0EEFED4E8EF3FC4E888
:10A47000E25F002AF9D1D4E8EF3F43F00103C4E8DA
:10A48000E23F002AF7D1002038BD00BFE1D402002E
:10A4900038B50025046904F10803D3E8EF2FC3E8B9
:10A4A000E15F0029F9D12369A28AC4E90C3522644D
:10A4B00004F16000C4E90E5506492FF012F906496F
:10A4C00004F170002FF00DF904F144002EF0B5FFF7
:10A4D000284638BD6DA100004D9F000038B50D46DF
:10A4E00004464FF4847200212FF074FF2B680E494C
:10A4F00023606B6804F1300063602FF06AF904F1A7
:10A5000060000A492FF0EDF8204600F0ABF908B9D9
:10A51000002038BD2946204600F0B6F90028F7D1C2
:10A5200004F10800F5E700BFB3D50200ADD5020085
:10A53000F8B5436F04469A4228BF1A4600AF006F31
:10A5400015462FF021FF2068216F83682A465C683A
:10A55000114BA0470446E0B1104803685B0715D0D3
:10A560006E468AB00E4A0F4B05920F4A0894CDE909
:10A5700006254FF40072ADF824206A4642F8103FD9
:10A5800000234FF43151F9F7D1F8B5462046BD46C6
:10A59000F8BD2C46FAE700BF40420F00902800208B
:10A5A000BA0C040005000001BD1004002DE9F843B9
:10A5B00000F170080546404623F02CF8814600283B
:10A5C00045D0286820F073FB041E0BDA214803688D
:10A5D0005B0704D0012123461F4A20F04EFA204693
:10A5E000BDE8F883686810B1012122F0FDFF002763
:10A5F00005F18806D6E8EF3FC6E8E27F002AF9D1E8
:10A60000D6E8EF3F43F00103C6E8E23F002AF7D166
:10A61000D5F80021286809F10409043A83684946FD
:10A62000DC684FF47A73A047041E0ADA49464046B4
:10A6300022F0C5FFD6E8EF3FC6E8E27F002ACED081
:10A64000F8E705F1080022F07AFE3C46C7E76FF014
:10A650000B04C4E790280020D610040038B5044647
:10A6600000F18805D5E8EF3F23F00102C5E8E12FAE
:10A670000029F7D1D90702D40024204638BD20682C
:10A6800083689B689847D5E8EF3F23F00402C5E84C
:10A69000E12F0029F7D15A0702D4206822F0B7FF32
:10A6A000606810B1002122F09FFF20680022002383
:10A6B00020F025FC041EDFDA044803685B07DCD0C9
:10A6C00001212346024A20F0D8F9D6E7902800203D
:10A6D000F2100400F0B50B780E46144685B002F176
:10A6E0008805062B11D8DFE803F0042260395A9060
:10A6F000A700D5E8EF3F23F00203C5E8E23F002AB8
:10A70000F7D104F160001CF0A5F8D5E8AF3FD907F8
:10A710000BD4D5E8AF3F5A0707D4D5E8AF3F9B0726
:10A7200003D404F178001CF095F805B0F0BDD5E82D
:10A73000AF3FD90709D54648036813F0060F04D088
:10A74000B3680221434A20F098F9D5E8EF3F23F09F
:10A750000203C5E8E23F002AD3D0F6E704F1700710
:10A76000384622F057FF06460028CED02068D4F89D
:10A770000021836804361B693146043A9847034632
:10A780000028C2D032480268520703D00121324A61
:10A7900020F073F93146384622F011FFB5E74968D9
:10A7A0000029B2D004F17000F6E74B68002BACD062
:10A7B000D4F89820D4F800119B1A043BB3FBF1F3B2
:10A7C00001FB0323D3E8EF1F0131C3E8E21F002A96
:10A7D000F8D1D6E9013213440293F36803930023BE
:10A7E000002202A904F1AC002EF06AFD0346E0B19C
:10A7F0001748026812F0060F05D0F2680221009295
:10A80000164A20F044F97168CCE7D5E8AF3FDE077F
:10A810007FF57BAFD5E8EF3F43F00402C5E8E12FB9
:10A820000029F7D158073FF570AF0022002304F14B
:10A8300030001CF07FF868E70548036813F0060F46
:10A840003FF463AF0B790221054A20F016F95CE76B
:10A85000902800200F1104002B1104003F11040068
:10A860006211040008B50246006883681B682BB1BA
:10A8700004499847B0FA80F0400908BD6FF05700CE
:10A88000F8E700BFD5A60000F8B50327CA6880F82E
:10A890000471CB680D460C210446B3FBF1F001FBBB
:10A8A0001033D21A92FBF7F2C4F800213B46A96894
:10A8B00004F18C002EF092FC0646B0B908223B460B
:10A8C00004F1E80104F1AC002EF0E6FC2B69084924
:10A8D00023676B6904F1780063672EF002FF21465D
:10A8E000044A04F1080022F070FC3046F8BD00BFB5
:10A8F000B9D502002CCA0300004870479C270020ED
:10A9000030B50E4A0E4B1168928893B003F14005A2
:10A910009A80196002AA144618685968083303C45B
:10A92000AB422246F7D14023002200934FF48070BF
:10A93000044902AB0BF0C0FF13B030BDA0110400FE
:10A940009C270020000050F02DE9F04105460E46FE
:10A950001746134CDFF84C80444508D3FCF7DEFD66
:10A960006A22114B1A504FF0FF30BDE8F081236886
:10A97000AB4200D08BB93A4631462846A368984787
:10A9800058B1FCF7CBFD0022074B3146C2503A4686
:10A990002846E368BDE8F04118471034DCE700BF03
:10A9A0006CB803007CB803000C00000073B50D46C2
:10A9B0001646694601AAFDF7D3F90446B0B1009BDB
:10A9C0005B69DBB14FF0FF324FF0FF33019822F0AB
:10A9D000BEFE009B2046324629465B6998470446E6
:10A9E000019822F0B6FE204602B070BD0923FCF7A4
:10A9F00095FD034A4FF0FF341350F4E75F23F6E769
:10AA00000C00000073B50D461646694601AAFDF715
:10AA1000A7F90446B0B1009B9B69DBB14FF0FF3250
:10AA20004FF0FF33019822F092FE009B2046324601
:10AA300029469B6998470446019822F08AFE2046E1
:10AA400002B070BD0923FCF769FD034A4FF0FF34E3
:10AA50001350F4E75F23F6E70C0000002DE9FF41F7
:10AA60000D46164602A903AA1F46FDF779F90446CA
:10AA7000E8B1029B5B6A13B34FF0FF324FF0FF3334
:10AA8000039822F064FE0B9B204601930A9B3246FA
:10AA90000093029B2946D3F824803B46C0470446D6
:10AAA000039822F056FE204604B0BDE8F081092349
:10AAB000FCF734FD034A4FF0FF341350F3E75F23F4
:10AAC000F6E700BF0C0000002DE9FF410D461646D9
:10AAD00002A903AA1F46FDF743F90446E8B1029B09
:10AAE0009B6A13B34FF0FF324FF0FF33039822F00D
:10AAF0002EFE0B9B204601930A9B32460093029B3D
:10AB00002946D3F828803B46C0470446039822F0E4
:10AB100020FE204604B0BDE8F0810923FCF7FEFCCE
:10AB2000034A4FF0FF341350F3E75F23F6E700BF0B
:10AB30000C0000002DE9FF410D46164602A903AAAC
:10AB40001F46FDF70DF90446D8B1029BDB6A03B33B
:10AB50004FF0FF324FF0FF33039822F0F8FD0A9BCD
:10AB600020460093029B3246D3F82C8029463B4670
:10AB7000C0470446039822F0ECFD204604B0BDE82F
:10AB8000F0810923FCF7CAFC034A4FF0FF3413504D
:10AB9000F3E75F23F6E700BF0C0000002DE9FF415B
:10ABA0000D46164602A903AA1F46FDF7D9F804462A
:10ABB000D8B1029B1B6B03B34FF0FF324FF0FF3352
:10ABC000039822F0C4FD0A9B20460093029B324664
:10ABD000D3F8308029463B46C0470446039822F00C
:10ABE000B8FD204604B0BDE8F0810923FCF796FCCF
:10ABF000034A4FF0FF341350F3E75F23F6E700BF3B
:10AC00000C00000070B506461D460C4609B10C2A22
:10AC100007D0FCF783FC1622174B1A504FF0FF3079
:10AC200070BD0B68002BF4D08868C0B122F09BFD8A
:10AC300038B996F9BC00002815DC09F075FB00282E
:10AC4000E7D09DB1002221460DF024FC00280346E8
:10AC500010DAFCF763FC084A5B421350DEE7081D7C
:10AC600025F018F9E2E722F07EFDE8E721460DF035
:10AC70004DFCEBE70020D3E70C00000070B5064662
:10AC80001D460C4609B1142A07D0FCF747FC1622D2
:10AC9000194B1A504FF0FF3070BD0BF0C9FC102259
:10ACA000014620462FF0A2FB0028EED0206922F0BA
:10ACB0005AFD70B996F9BC00002807DC09F034FB96
:10ACC00038B9FCF72BFC02220B4BE2E722F04BFDDC
:10ACD000F6E7214655B10EF069FC0028034608DA74
:10ACE000FCF71CFC044A5B421350D3E70EF09AFCBD
:10ACF000F3E70020D0E700BF0C000000F7B50746DF
:10AD00000E461446FDF746F8051E18DB3CB97B1EBF
:10AD1000012B04D8022E17D0012E08BF0624F1B251
:10AD200001ABA2B2B8B20CF063F9061E0EDA2846E7
:10AD300021F009FCFCF7F2FB104B76421E504FF05D
:10AD4000FF35284603B0F0BD1124E8E70023019841
:10AD50004360036774302EF070FB019890302EF042
:10AD60008CFD062C02D1019825F0E3FC4FF4404302
:10AD70002846034A0199FDF74DF8E2E70C00000070
:10AD80003CCA03002DE9F04389B0DDE910980C4678
:10AD900058EA090105464F46129E13D014F1690F77
:10ADA00002D014F10B0F0DD168462FF0D1F8DDE978
:10ADB000002313430ED114F1690F14BF6FF0680420
:10ADC0006FF00B04FCF7AAFB364B64421C504FF0AB
:10ADD000FF304CE0B8F1FF3F08BFB9F1FF3F0FD0A3
:10ADE0004FF47A71A7FB0107002347F6122201FBFB
:10ADF0000871F6F77DFB3368834294BF336030609F
:10AE0000D5F8980008B11BF0A7FA693432D0B5F82C
:10AE1000BA3003F0C003402B2CD195F9BC0022F0CE
:10AE2000A2FC28462AF068F800220346022103A863
:10AE30002FF0B4F947F6122740F2E73000213468CA
:10AE40004FF47A720023E4FB0701F6F751FB024648
:10AE50000B46012103A81CF0DDFE33685B00642B68
:10AE600028BF64233360D5F8980098B9002009B052
:10AE7000BDE8F08347F6122740F2E730002134683E
:10AE80004FF47A720023E4FB0701F6F731FB2EF052
:10AE900051FEE2E74FF0FF324FF0FF331BF0EAF9CB
:10AEA000E4E700BF0C00000040F205139942F7B53B
:10AEB000044600F0EC80B1F5837F58D2B1F5817F74
:10AEC00000F0868009D803296FD0042974D0FCF7DC
:10AED00025FB5F22824B1A5064E040F20313994233
:10AEE000F5D1D2E90056AB88DB070ED53368DB68B5
:10AEF00013F4EE1F02D1036FDF0703D5EB8843F095
:10AF00000103EB80336814333360AB8858071FD5D7
:10AF1000B4F8BA3003F0C003402B40F0B38094F98A
:10AF2000BC0022F020FC3368DB6813F4FE1F0CD059
:10AF3000236FD90709D4B4F8BA30C3F34103022B05
:10AF400002BFEB8843F00403EB80336814333360B3
:10AF5000236F5A0742BFEB8843F00803EB80236F4F
:10AF6000DB0733D5EB8843F01003EB802EE045F28E
:10AF70001B43994200F0918045F22143994200F031
:10AF80008A8045F211439942A1D1B0F8B8301568D2
:10AF9000062B00F08F806FF05E03FCF7BFFA504A7B
:10AFA0005B4213504FF0FF3004E090F87000C0F3A4
:10AFB0004000800303B0F0BD1268036F550402D552
:10AFC00043F0020301E023F0020323670020F1E7CE
:10AFD000D2E900158B889768D8071BD52B689F424C
:10AFE00002D16FF00B00E5E7042004F174021A614E
:10AFF0002B685A7B60F305025A732A68937B23F00F
:10B00000200393732A68D36823F4FE13D3602B685C
:10B0100014332B608B885A072CD5B4F8BA3003F060
:10B02000C003402B02D06FF07700C3E794F9BC0057
:10B0300022F099FB2E68B742D3D0B4F8BA3020463C
:10B04000C3F34103012B1AD129F059FF02213061CA
:10B050002B685A7B61F305025A732A68937B23F0AD
:10B06000200393732A68D36823F4FE13D3602B68FC
:10B0700014332B60236F13F0050FA7D0D3E729F00B
:10B080003BFFE3E7EB8843F00403EB8060E71368E2
:10B09000C0F898309AE7036F92E7002314681946C6
:10B0A0001A4622F0A4FB6FF00043984294BF206040
:10B0B00023608BE7B0F8BA30C3F34103032B02D10E
:10B0C0006FF0150369E701A929F0F9FE031EFFF6E9
:10B0D00064AF019B002BFFF660AF2B6076E700BFEB
:10B0E0000C00000037B5002B0546069C1CD10093D0
:10B0F0000022002313490CF095F805F174002EF09E
:10B100009CF905F190002EF0B8FB04F1740029467B
:10B110002EF0D3F9284625F00CFB04F1900003B083
:10B12000BDE8304022F03EBB0ADA5B426360236F29
:10B1300043F00403236704F174002EF08BF9ECE76D
:10B1400003B030BDE9D8020013B50021B0F8BA3021
:10B150000446C3F34103032B4FF000024FF00003FA
:10B16000009119D125F09CFF04236360236F2046D2
:10B1700043F00403236722F017FB20460CF02AF863
:10B18000031E06DAFCF7CAF9054A5B4213504FF07A
:10B19000FF33184602B010BD0CF044F8E4E700BFDE
:10B1A0000C00000037B505460C4611BBB0F8BA30AC
:10B1B0000022C3F34103032B00914FF000030DD194
:10B1C00025F06EFF031E0CDAFCF7A8F90E4A5B426D
:10B1D00013504FF0FF34204603B030BD0CF022F87E
:10B1E000F0E72B6F284643F001032B6722F0DCFACF
:10B1F000F1E74C1EFCF792F9012C94BF862216222F
:10B20000014B1A50E5E700BF0C00000013B50446DF
:10B2100025F0C8FA031E07DAFCF780F90D4A5B42F5
:10B2200013504FF0FF3007E0B4F8BA30C3F3811386
:10B23000023B012B02D9002002B010BD636800223E
:10B2400000932046002304490BF0ECFF031EF2DAC2
:10B25000E2E700BF0C000000E9D802002DE9F0434E
:10B26000B0F8BA309146C3F38112032A04468846E7
:10B2700085B007D1FCF752F95F222D4B1A504FF0E1
:10B28000FF3037E0C3F34103022B32D0012B056FAF
:10B2900009D1FCF743F915F0040F254B01D0626882
:10B2A000ECE77822EAE715F002051BBF002600272D
:10B2B0000027204D08BF204E012A43681DD100936E
:10B2C000002200231D490BF0ADFF002805DA4342A0
:10B2D000FCF724F9164A1350D1E763684A460293F3
:10B2E00041462B462046CDE9006725F0DAFD0028CF
:10B2F000EDDB002005B0BDE8F08302934A462B4603
:10B30000CDE9006725F0CDFD031E03DAFCF706F951
:10B310005B42DFE7236FDB07EBD463680022009317
:10B320002046002305490BF07DFF031EE1DAEDE71F
:10B330000C0000007BD90200366E0100E9D8020043
:10B3400013B5B0F8BA30044603F0C003C02B08D1DF
:10B35000FCF7E4F85F220D4B1A504FF0FF3002B0BB
:10B3600010BD25F06BFD031E05DAFCF7D7F8074A80
:10B370005B421350F1E70023002220460449009469
:10B3800025F08EFE031EF0DB0020E8E70C00000035
:10B39000E5B000002DE9F04F16460A224FF0FF38C5
:10B3A0004FF0FF398FB00B925A0604460D46CDE997
:10B3B0000C89189F03D4036F13F0020328D00022D6
:10B3C0000023CDE90C2308A82EF09DFDDDE90C2318
:10B3D000DDE9088908A82EF096FDDDE90823CDE90E
:10B3E0000623236FDB071AD46368002200932046EC
:10B3F000002327490BF016FF031E10DAFCF78EF826
:10B40000244A5B4213504FF0FF300FB0BDE8F08F7D
:10B410000CAA05210CF0B6F800231F4AD3E74FF021
:10B42000000A0DF12C0B6168DDE90C2337B3CDE97F
:10B430000223199B0491009332463B46294620463D
:10B44000CDF804A025F0BEFE0028DEDADDE90C23ED
:10B450000146CDE90023204642464B46CDF808B0D0
:10B46000FFF790FC0130CED0DDE9062308A82EF0CE
:10B470006FFDDDE90823CDE90C23D4E7CDE90023F6
:10B4800002913B4632462946204625F03AFEDBE74C
:10B49000E9D802000C000000B4C404002DE9F04714
:10B4A0004FF0FF3315464FF0FF328CB0CDE90A2341
:10B4B0000A236A0604460E46099303D4036F13F069
:10B4C000020339D000220023CDE90A23002706A871
:10B4D0002EF019FDDDE90A23DDE9068906A82EF024
:10B4E00012FDDDE90623CDE904230DF1240ADDE98F
:10B4F0000A233146CDE90023204600232A4602973D
:10B5000025F03BFE00281EDADDE90A230146CDE9DD
:10B51000002320464B464246CDF808A0FFF732FCF8
:10B52000431C10D0DDE9042306A82EF011FDDDE94F
:10B530000623CDE90A23DAE70AAA05210CF022F84E
:10B540000023024AC2E70CB0BDE8F087B4C404008F
:10B55000F7B5B0F8BA30044603F0C003C02B0E466E
:10B56000174609D1FBF7DAFF5F22294B1A504FF03B
:10B57000FF35284603B0F0BD036F5A0704D5FBF72B
:10B58000CDFF6268224BF1E79B0710D44FF0FF33E9
:10B590004FF0FF326946CDE9002322F019FA031E6D
:10B5A00005DAFBF7BBFF1A4A5B421350DFE70022C4
:10B5B00004F1740000231AF01FFF044620B9FBF7C2
:10B5C000ADFF0B22124BD1E728F0A3FFFCF7E2FB03
:10B5D000051E06DA204622F0E7F820460BF0FAFDB9
:10B5E000C5E73A463146204622F0BFF840B128462A
:10B5F00020F0A9FFFBF792FF8622054B1A50E9E7DE
:10B600004FF4404321462846024AFCF703FCB0E7CA
:10B610000C0000003CCA03002DE9F04F8FB09A46A1
:10B62000DDE9196B4FF0FF3302924FF0FF32CDE9A5
:10B630000423189B0D465906074603D4036F13F0E5
:10B64000020330D000220023CDE90423189B07F128
:10B65000740413F00203009339D0DDE90489102249
:10B66000002109A82EF0B6FE04230D948DF8313088
:10B6700001214B46424609A81CF0CCFA00F10B010F
:10B680000B29034619D840F68102CA40D20714D5C7
:10B6900020462DF057FF0446F8B9FBF73FFF0B2279
:10B6A000964B1A500EE0042104AA0BF06BFF3846AB
:10B6B00004A922F08DF9031EC8DAFBF72FFF8F4A89
:10B6C0005B4213504FF0FF300FB0BDE8F08FDDE963
:10B6D000042320461AF090FEDDE7D0E90398002EFF
:10B6E00000F09380BBF1000F00F08F80DBF80020AA
:10B6F000B7F8B8300392019326F08FF894F83F30F2
:10B70000039AC3F3C203338094F83F30C3F3C203F8
:10B71000012B30D100201423072ACDE9090363D976
:10B72000204609A926F06BFA074610B96FF06803A6
:10B7300025E020460A9926F0CBF80028F6D12046CD
:10B7400094F8421026F0C4F80028EFD1FB6873602B
:10B750009DF80430B71C112B49D107AB099308237E
:10B7600009A90A93204626F04AFA0028DED0038869
:10B770003B80002303E0022B11D06FF08503C4E966
:10B780000398002B3BD05B42FBF7C8FE5B4A13508B
:10B79000009B002B96D1204625F0B3FF92E70021B5
:10B7A0002823172ACDE909131ED9204609A926F016
:10B7B00026FA07460028B9D020460A9926F088F8CC
:10B7C0000028B3D12046B4F8421026F081F80028B2
:10B7D000ACD107F10803321D183753F8041BBB42E4
:10B7E00042F8041BF9D1B3E76FF01503C7E7062B46
:10B7F000C3D109AB0793142307A90893B2E7338891
:10B80000012B0DD10823CBF80030002D44D0EB687C
:10B810000BB1AB6843B9FBF781FE0C22374B40E715
:10B82000022B69D11823EEE7204626F0DAF85045BE
:10B83000074628BF57460646BB460023BBF1000F0C
:10B840000FD1564503D9AB6943F02003AB612A6998
:10B85000002A4CD0696971B30F2946D8C5F814B0D5
:10B8600029E0AA68D158D01821B9FBF757FE162253
:10B87000224B16E7426820465A4528BF5A46029393
:10B88000019226F03BF8029B019A083308B1692324
:10B890007AE7ABEB020BD1E7204626F0A2F882450F
:10B8A000574628BF074606463A462046029926F0E4
:10B8B00025F80028EBD1009BDBB9204625F021FFBD
:10B8C000189B13F0200F0CBF38463046FCE60733B8
:10B8D00023F007000346103313448B428344BDD842
:10B8E00002441368002BF2D1B8E71144F9E76A610A
:10B8F000E1E7C4E90398E3E7862345E70C0000008D
:10B900002DE9F04F90461C464FF0FF324FF0FF33C9
:10B910008DB0CDE90823B0F8BA300546DF070E46F2
:10B92000DDF858A00ED5C3F34103022B0ED08023BF
:10B93000FBF7F4FD4FF0FF345A4A135020460DB088
:10B94000BDE8F08F0923F3E78623F1E71AF0400FF3
:10B9500002D1036F990715D500220023CDE90823F2
:10B96000002CEBD0DDE90879CDE905840AF4807B71
:10B97000AEB1B8F1000F12D1F3685BB96FF01500EA
:10B980004342D5E713F00503EAD1042108AA0BF0DE
:10B99000F9FDE5E7B3681A685B68059207934FF015
:10B9A0000008CDE90A7902A8DDE90A232EF0ABFAF6
:10B9B000DDE90234CDE900344446069B93B36B6F56
:10B9C000E3B92B6F5A0707D564BB6868404200286B
:10B9D00020EAE07403DAD3E7DB070FD514BBDDE917
:10B9E0001712284621F0C1FE0028ADD11AF0020F2F
:10B9F000A4D12146284625F00FFC9FE757EA09030A
:10BA000012D1D6B95346284606AA05A921F0EFFE61
:10BA1000231850EA030443D157EA09071AD0BBF1AF
:10BA2000000F35D12046D2E728460AA9CDE90A7988
:10BA300021F0CEFF0028E4DAC9E75346284607AADA
:10BA400005A921F0D4FE044450EA040305D157EAC5
:10BA5000090302D16FF00A0092E7B2684FEAC80307
:10BA600052F83810014405910699091A0691079970
:10BA70000029D4D1F16808F101088845D2D00833F3
:10BA8000D118D2584B68059207930AB1002BD4D134
:10BA9000DDE900230AA82EF05BFADDE90A798CE7DC
:10BAA0001C46BCE70C000000F0B585B01C46DDE983
:10BAB0000A6713460AB3B0F8BA20C2F38112951E82
:10BAC000012D08D80A46CDE9016700210094FFF74F
:10BAD000A3FD05B0F0BD012A07D10A46CDE90167F3
:10BAE00000210094FFF70CFFF3E7FBF717FD862218
:10BAF000034B1A504FF0FF30EBE71046E9E700BF69
:10BB00000C000000F0B5B0F8BA3085B0C3F3811C6A
:10BB1000644699B18E68D6B100231D46CF680436BD
:10BB2000AF4218D1023C012C1AD80C1D02940C68AB
:10BB3000CDE900240022FFF76FFD06E01623FBF796
:10BB4000EDFC0D4A13504FF0FF3005B0F0BD0C2353
:10BB5000F5E78623F3E756F835E001357344DFE770
:10BB6000BCF1010FF5D10C1D02940C68CDE9002445
:10BB70000022FFF7C5FEE8E70C00000073B50E4693
:10BB8000062E1C4605461146069B60D008DC002E9A
:10BB90006CD0012E24D0FBF7C1FC6D226F4B40E02E
:10BBA000292EF8D1182A00F3B5800F2AF3DDA2F16F
:10BBB00010010829EFD801A252F821F037BD00008A
:10BBC0003DBD00004FBD000055BD000097BB00000B
:10BBD00097BB000097BB000097BB000029BD000089
:10BBE0000F2A31D00ADC032A20D0042A12D0022ADC
:10BBF000D1D1224609210BF0C5FC2DE0262A20D008
:10BC0000272AC8D11B68042B07D1B0F8BA30C3F378
:10BC1000C20309E01B68042B05D0FBF77FFC16224A
:10BC20004E4B1A501FE04368236007E0B0F8BA207B
:10BC3000C2F381121B68042BEFD12260002002B0F6
:10BC400070BDB0F8B820F5E722460A21D3E7012AF3
:10BC5000A1D1224629F00CF9031EEFDAFBF75EFCB6
:10BC60003E4A5B4213504FF0FF30E8E70F2A58D0AE
:10BC700008DC022A17D00E2A46D0012A8BD1224690
:10BC80000821B8E7212A3CD0222A40D0202A82D19C
:10BC9000B0F8BA20C2F3C202012A07D0FBF73EFC7B
:10BCA0006A222E4BBDE722461021A4E704221B681E
:10BCB00001920CB1934205D0FBF730FC1622274BC2
:10BCC0001A500BE001AB6A4613210BF05BFC031E1C
:10BCD00008DAFBF723FC214A5B4213504FF0FF3692
:10BCE0003046ACE7009808B92060F9E723F067FE1A
:10BCF00020B9FBF713FC0222184BE1E743682360ED
:10BD0000EEE722460D2176E72246142173E722460C
:10BD1000172170E7432AB2D0482A09D03E2A7FF47F
:10BD20003AAF2246192166E722461421284662E7E7
:10BD3000224611215FE722460F21F7E7B0F8BA202B
:10BD4000C2F3C202022AA9D122461321EEE72246FB
:10BD50000E21EBE722461621E8E700BF0C000000A9
:10BD60007FB50E46062E114605461C46089A00F081
:10BD7000AA8009DC002E00F0B080012E28D0FBF74D
:10BD8000CDFB6D229D4B3CE0292EF8D11A2900F302
:10BD900008810F29F3DD10390A29F0D801A353F8DF
:10BDA00021F000BFC9BF0000D1BF0000D9BF000013
:10BDB000F5BF0000E1BF0000F1BF00007FBD000043
:10BDC0007FBD0000B9BF00007FBD0000DFBD0000E7
:10BDD0000F291ED006DC022915D00D29CFD1002055
:10BDE00004B070BD142918D01929C8D1B0F8BA30E0
:10BDF000C3F3C2010139012939D9FBF78FFB6A224C
:10BE00007E4B1A5049E01346092122460BF0CCFA2A
:10BE100060E013460A212246F8E7102A04D0FBF717
:10BE20007DFB1622754BECE7D3E9003653EA060298
:10BE3000A16800D1B9B17248A3FB003200FB062211
:10BE4000C8171F3140F100005B1842EB00025B098C
:10BE500043EAC2635209CDE90232082304210DEB03
:10BE600003022846D2E74FF0FF331A46F3E71AB130
:10BE7000002CD4D0217821B923F40073A5F8BA306E
:10BE8000ADE7082ACBD120460AF030F8031E07DAC6
:10BE9000FBF744FB594A5B4213504FF0FF309FE7DA
:10BEA00021F061FC20B9FBF739FB1322534BA8E7C3
:10BEB000B5F8BA3043F40073A5F8BA3009F01AFCAB
:10BEC00085F8BC008BE701297FF459AF1346224661
:10BED00028F0A2FF031E82DADAE724293FF74FAFEA
:10BEE0001F290ADC02294AD00F2961D001297FF4D9
:10BEF00046AF13460821224688E7A1F12103032B10
:10BF000003D8DFE803F0384A4048002301931CB10E
:10BF10000C2A0AD0082A20D0FBF700FB1622374B48
:10BF20001A504FF0FF3630465AE7A068A8B121F00A
:10BF30001AFC0190019808B109F0DCFB042302907F
:10BF40001321284602AA0BF02FFA031EEBDAFBF7A7
:10BF5000E5FA2A4A5B421350E3E76368002BE9D015
:10BF600001A9201D23F048FD0028E3D1FBF7D6FAF4
:10BF70000222224BD4E713460D21224671E71346D5
:10BF80001021224642E701232146284604B0BDE89D
:10BF90007040FEF737BE0023F6E71346172122460E
:10BFA0005FE74329A5D048290AD03E297FF4E7AEB0
:10BFB00013461921224629E713461421224650E749
:10BFC00013461121224621E713460F21224648E756
:10BFD00013461321224644E713460E21224640E72A
:10BFE00001232146284604B0BDE87040FEF746BE56
:10BFF0000023F6E713461621224632E70C00000024
:10C0000040420F00F0B51446B0F8BA200D46C2F316
:10C0100081110329034687B008D1FBF77FFA5F221D
:10C02000274B1A504FF0FF3007B0F0BD05B124B9CF
:10C03000FBF774FA1622224BF3E7D00504D4FBF782
:10C040006DFA80221E4BECE7012903D1C2F34102B5
:10C05000022AF4D19A8D012A12D1ADF80020DA8D8E
:10C060001B6BADF8022022686946082A28BF082207
:10C07000284601932EF088F9082300202360D3E797
:10C08000022AD5D10021ADF80020DA8D0591ADF856
:10C09000022001AF03F1300240333E461068516880
:10C0A000083203C69A423746F7D122686946182AF1
:10C0B00028BF182228462EF067F91823DDE700BFB5
:10C0C0000C000000F0B5038C0E46012B044615460B
:10C0D0004FF0000189B014D1436ACDE902115BB37E
:10C0E000082301AA01930DEB030125F0ABF8031E11
:10C0F00015DA5B42FBF712FA134A13504FF0FF3088
:10C1000018E0022B1AD1182702A83A462EF062F93D
:10C11000636A8BB12046019701AA02A9E5E7019C59
:10C120002A683046A24228BF224602A92EF02CF9E6
:10C1300000202C6009B0F0BD1623DBE7FBF7EEF919
:10C140001622014B1A50D9E70C000000F8B505463D
:10C150000E46054C054FBC4200D3F8BD2046314683
:10C16000A8470C34F7E700BFECB80300F8B80300A9
:10C170002DE9F84305460C46904699464FF0FF33AB
:10C180004FF0FF3234481AF075F8344B1B78EBB996
:10C190004FF0FF324FF0FF332F4931481AF06EFC59
:10C1A000304B9D4251D3304B9D424ED26CBBB9F1C6
:10C1B000010F30D114224FF400416B689C4217DA12
:10C1C0002B6802FB043301341981F6E7032BE7D017
:10C1D0006FF0040413E000FB03F12A6801330A4402
:10C1E00056602A680A4417816A689342F3DBA4B94F
:10C1F0001E49012200230868FCF75AF8002416485B
:10C200001AF0AAF82046BDE8F883002314204FF066
:10C21000FF360027E8E72346F8E7424518DB00270A
:10C220004FF0140CB845E3DD0CFB07F22E6804EB6D
:10C23000C7031644043693E8030086E803002B681E
:10C2400001371344C3F80C90ECE76FF00104D6E714
:10C250006FF00B04D3E700BF402A0020918000203C
:10C26000742C0020ECB80300F8B80300F06A00203A
:10C270002DE9F04F5D4BDFF8789185B0A9EB030213
:10C280000B2A40F2AA8000274B4507F101083ED354
:10C29000B8F1140F00F2A1800021564D0846C5F8F0
:10C2A000A080FBF77DFF041E534EC0F29180032354
:10C2B000337052481AF0ACFB01234FF0140A2C6083
:10C2C000AB804FF0FF324FF0FF334D4819F0D2FFF3
:10C2D000DFF818B1CB454AD349481AF03DF84FF082
:10C2E000FF324146434820F0A6F9002870DD4FF0A8
:10C2F000010B404CBB453CDDB5F90630002BEED0C0
:10C30000286802A9FBF7A4FF0023EB80D9E79A680D
:10C310000C33C2F8008053F8082C1744B4E7DBF85C
:10C3200000400AFB0344606800280DDBB4F90810E4
:10C3300011F5004F08D1019321F00DFA4FF0FF32B3
:10C340000021019B62602181DBF80810096803EB82
:10C35000010C05EBCC0CD4E901018CE8030001339E
:10C36000DBF804109942DADC0BF10C0BB2E7002386
:10C37000F6E7D4F808C0BCF1000F25DBB4F90E30A5
:10C38000002B21DD194B0AE01A680AFB0022D2F8C3
:10C3900004E0F44508D001308842F5DB0C334B450E
:10C3A0008FD200205968F7E71361131DD4E9020109
:10C3B00083E803004FF0FF31A3681046A1600193AA
:10C3C00021F039FB019BA3600BF1010B083491E7CD
:10C3D0000223337005B0BDE8F08F0122064B1A70BE
:10C3E000064805B0BDE8F04F1AF012BBECB80300E8
:10C3F000F8B80300F06A002091800020742C00201F
:10C40000402A002000B589B000220023CDE9062390
:10C4100000230E22CDE90133CDE9032300934FF42D
:10C420009662054B054906481AF09EFC054909B07D
:10C430005DF804EB1AF04EBB71C2000008C000208A
:10C44000483D0020A711040037B504460D4661B9E8
:10C4500038B10321194A1FF022F86FF0150003B01C
:10C4600030BD16481DF008FCF7E70A22284601A94E
:10C470001BF04EFE019B1B7873B144B12B46032188
:10C4800020460F4A1FF00BF86FF00100E7E729463E
:10C490000B481DF0F1FBF7E7FF28E0D944B1034654
:10C4A00003212046074A1EF0FAFF6FF02100D6E76D
:10C4B000014604481DF0E0FBF7E700BFBA11040095
:10C4C000D7110400E911040004289ABF024B53F865
:10C4D00020000248704700BF90CA0300FB1104000F
:10C4E0000130C0B203289ABF024B53F82000024823
:10C4F000704700BF80CA03000A1204002DE9F3410F
:10C500001F46038C04460D461646DDF82080042B9A
:10C5100058D8DFE803F04B2A03535500416AF1B1C4
:10C52000022009F029FF628C034652BA92B20092AF
:10C5300031462846274A1BF09DFD022004F13001B8
:10C5400009F01AFF0346E28D52BA92B20892214ACC
:10C550004146384602B0BDE8F0411BF08BBD314684
:10C5600028461D4A1BF086FDE7E7416AC1B101205C
:10C5700009F002FF628C034652BA92B20092314631
:10C580002846164A1BF076FD012004F1300109F01F
:10C59000F3FEE28D034652BA92B208920F4AD7E7F1
:10C5A000314628460C4A1BF065FDEDE70C4A314642
:10C5B000284602B0BDE8F0411BF05CBD094AF6E731
:10C5C000094AF4E731462846084A02B0BDE8F0417E
:10C5D0001BF050BD1A120400221204002E12040097
:10C5E000341204003E120400481204004F120400EA
:10C5F00048B103685A68074B9A4204D109B1064B07
:10C600000B600648704709B905487047054B0B6039
:10C61000FAE700BFE02D002074120400C4470400B4
:10C620005A1204006912040007B550B1084B0221E8
:10C630000093084A084B1EF032FF002003B05DF85B
:10C6400004FB034A044903481DF016FBF5E700BF4D
:10C650002313040005130400E612040007B548B1D3
:10C66000084B02210093084A084B1EF018FF03B044
:10C670005DF804FB034A0549034803B05DF804EB89
:10C680001DF0FABAAD130400051304005F13040093
:10C6900007B550B1084B02210093084A084B1EF021
:10C6A000FEFE002003B05DF804FB034A0449034882
:10C6B0001DF0E2FAF5E700BF5F1404000513040063
:10C6C00005140400002310B586B004460393002827
:10C6D00048D00821354A1EF0E2FE03AB344804A9D5
:10C6E000059304940BF014F8039B002B45D1002C08
:10C6F0003CD0082120462F4A1EF0D1FE08212046BA
:10C700002D4A1EF0CCFE00232C4804A903930BF005
:10C71000E7FC039B002B3AD1002C31D008212046A6
:10C72000274A1EF0BCFE08212046264A1EF0B7FE0E
:10C730000023254804A903930DF058FA039B002B0E
:10C7400031D13CB308212046204A1EF0A8FE204BE0
:10C750000221009320461F4B1F4A1EF0A0FE00201E
:10C7600006B010BD11481DF087FAB6E711481DF05C
:10C7700083FA11481DF080FAC5E7002CBED1F8E716
:10C780000F481DF079FA0F481DF076FAD0E7002C1B
:10C79000C9D1F8E70D481DF06FFA0D4A0D490E4852
:10C7A0001DF06AFADBE7002CD1D1F6E70816040089
:10C7B00089C900004A1604005A16040069C800001E
:10C7C000A5160400C4160400DDC7000011170400FC
:10C7D0004217040025170400051304002DE9F04F4B
:10C7E0000446D1E900B88BB028F006F8D4F80490DC
:10C7F0000746B9F82250B9F82E606DBAABB276BAD6
:10C80000D4F88452D4F890A294F880020993B6B276
:10C81000BBF1000F17D00EF061FF099BCDE9057049
:10C82000CDE90093082123465846CDE9035A0D4A25
:10C8300002961EF034FED8F800300133C8F80030FC
:10C840000BB0BDE8F08F0EF049FF4A46CDE903700A
:10C850002146CDE9015A099B024800961DF00CFAC9
:10C86000E9E700BF501704002DE9F0470446D1E97D
:10C870000087A2B014AE3522002130462DF0AAFD6B
:10C88000A38B06AD032B61D8DFE803F0593E025EAF
:10C8900004F12001022009F06FFDE28B034652BA39
:10C8A00092B2352100922846314A1BF0E3FB022068
:10C8B00004F1080109F060FD0346E28852BA92B221
:10C8C00000922B4A352130461BF0D4FB3B68D4F84C
:10C8D00034A0A08BB4F8401003F10109B8F1000FA7
:10C8E0003AD009F0F7FB4B46CDE901A008214046BC
:10C8F000CDE903561F4A00941EF0D1FD3B68013379
:10C900003B6022B0BDE8F08704F12001012009F06E
:10C9100033FDE28B034652BA92B23521009228468B
:10C92000154A1BF0A7FB012004F1080109F024FDC2
:10C93000E288034652BA92B200920F4AC2E70F4908
:10C940002846F4F7F9FDC1E70D49F9E735212846F6
:10C950000C4A1BF08FFBB9E709F0BCFB5346009073
:10C9600022464946CDE9015602481DF085F9C5E742
:10C970001A120400771704002E1204003412040067
:10C980003E1204004F1204002DE9F0433525D1E991
:10C9900000970446A5B016AE2A46002130460DF198
:10C9A00020082DF017FD2A462046009533464146C3
:10C9B000FFF7A4FD3D6894F9BC000135B9F1000F03
:10C9C00034D007F027FC08F095FEB4F8BA30C3F372
:10C9D000C202022A26D0012A14BF20223422C3F325
:10C9E0008113013B022B96BF27492023CB56B4F875
:10C9F000B810112918D0062914BF20215421CDE9DF
:10CA00000331CDE901022B4608214846CDE90586D0
:10CA10001E4A00941EF043FD3B6801333B6025B085
:10CA2000BDE8F0833622DAE75521E8E707F0F2FBAC
:10CA300008F060FEB4F8BA200346C2F3C20102292E
:10CA40001ED0012914BF20213421C2F38112013AE2
:10CA5000022A96BF0E4820228256B4F8B800112848
:10CA600010D0062814BF20205420CDE901200091C9
:10CA700022462946CDE9038604481DF0FDF8CBE7A0
:10CA80003621E2E75520F0E72294040092170400D3
:10CA90002294040007B550B1084B02210093084AC4
:10CAA000084B1EF0FCFC002003B05DF804FB034AB9
:10CAB000044903481DF0E0F8F5E700BFFB17040048
:10CAC00005130400E917040007B550B1084B022113
:10CAD0000093084A084B1EF0E2FC002003B05DF80A
:10CAE00004FB034A044903481DF0C6F8F5E700BFFC
:10CAF0001B180400051304000218040007B550B108
:10CB0000084B02210093084A084B1EF0C8FC002085
:10CB100003B05DF804FB034A044903481DF0ACF878
:10CB2000F5E700BFEF19040005130400DD19040048
:10CB30007FB5566804465EB930B10321554A1EF0F0
:10CB4000AEFC6FF0070091E052481DF095F8F8E751
:10CB5000956855B1284650492DF058FC90B96CB1F4
:10CB6000082120464D4A1EF09AFC012511F010FBC9
:10CB7000002865D1002C61D0494A5AE047481DF091
:10CB80007BF8F2E7284647492DF040FC58B934B10C
:10CB900008212046444A1EF082FC0525E6E742486B
:10CBA0001DF06AF8F9E7284640492DF02FFC58B9E6
:10CBB00034B1082120463E4A1EF071FC0C25D5E711
:10CBC0003B481DF059F8F9E728463A492DF01EFC7C
:10CBD00058B934B108212046374A1EF060FC1025B0
:10CBE000C4E735481DF048F8F9E7284633492DF0E9
:10CBF0000DFC58B934B108212046314A1EF04FFCD3
:10CC00001C25B3E72E481DF037F8F9E728462D49D3
:10CC10002DF0FCFB58B934B1082120462A4A1EF0F9
:10CC20003EFC2125A2E728481DF026F8F9E71CB1B3
:10CC3000264A0321204682E7244886E7184884E7ED
:10CC40004FF4FA63CDE90143214B2A460093314664
:10CC5000002329F0EEF9021E0FDA4CB100923346A0
:10CC6000032120461B4A1EF01AFC002004B070BDB0
:10CC7000314618481DF000F8F7E734B13346082173
:10CC80002046154A1EF00BFCEFE7314612481CF017
:10CC9000F3FFEAE7931A04000D1B0400AC1A04002A
:10CCA000851B0400C51A0400CB1A0400DD1A040019
:10CCB000E11A0400F51A0400F91A04000A1B040022
:10CCC0000F1B0400281B04002C1B0400401B040045
:10CCD00035D40000A41B0400BE1B040010B504469C
:10CCE00011F056FA034618BB3CB103212046164A00
:10CCF0001EF0D5FB6FF0070010E013481CF0BCFFDE
:10CD0000F8E7B3F8AE1229F091F9A8B93CB10123C4
:10CD1000082120460D4A1EF0C2FB002010BD012153
:10CD20000A481CF0A9FFF8E709481CF0A5FFF4E742
:10CD3000D0F89422002AE4D1002CF5D00821204616
:10CD4000034A1EF0ACFBE8E7851B0400D41B04007B
:10CD5000F41B040007B550B1084B02210093084AA8
:10CD6000084B1EF09CFB002003B05DF804FB034A57
:10CD7000044903481CF080FFF5E700BF1C1C0400B9
:10CD8000051304000E1C04002DE9F04F53680546FE
:10CD90008BB01BB1FFF7CCFE00200BE011F0F8F9CF
:10CDA000064670B94DB103212846A74A1EF077FB0D
:10CDB0006FF007000BB0BDE8F08FA3481CF05CFFDC
:10CDC000F6E7002D00F08880082128469F4A1EF0D3
:10CDD00066FB4FF00008341D06F50979CDE9088897
:10CDE000A06900280DDD07F015FA082208A923F034
:10CDF000B7F8002805DA0821A369954A08A81BF0AE
:10CE000039F934F8040C012840F0A1802146002DA6
:10CE100071D009F0B1FA34F8027C9DF820307FBA65
:10CE20008246BFB2002B5BD1DFF828B25B46207F81
:10CE3000002859D0079310F0D7FF227F079B002AC4
:10CE400056D0854A8549CDE902325346CDE90401E1
:10CE5000CDE9007B824A082128461EF020FB883459
:10CE60004C45BBD1002D00F0CB80082128467D4ADF
:10CE70001EF015FBD6F89432002B8DD0D6F8A832D0
:10CE8000002B89D006F51C702DF01CF84FF47A7237
:10CE9000A0FB020302FB013147F61123C01847F63D
:10CEA000122241F100010023F4F722FBB6F8AC1284
:10CEB000D6F8A8420129B6F8AE2240F0AC80002D89
:10CEC00000F0A280CDE90140674B00920821674A3B
:10CED00028461EF0E4FA5FE75C481CF0CDFE78E7D8
:10CEE000DFF88CB108ABA2E75A4A10461146AAE710
:10CEF000594A5849A7E709F03FFA34F8027C8246BC
:10CF00007FBABBB207939DF82030ABB1DFF860B1B8
:10CF100008AF207FA0B110F067FF227FA2B14E4A78
:10CF20004E49CDE902015B465146CDE900724C48BD
:10CF3000079A1CF0A1FE92E7DFF818B15F46E8E718
:10CF4000444A10461146ECE7434A4249E9E70228C1
:10CF500085D1214655B309F00FFA34F8027C9DF8CB
:10CF600020307FBA8246BFB2ABB1DFF804B108AB64
:10CF7000207FA0B1079310F037FF227F079B92B16B
:10CF8000354A3649CDE90232CDE904015346CDE9AF
:10CF9000007B384A5FE7DFF8BCB05B46E8E72D4A24
:10CFA00010461146EEE72C4A2A49EBE709F0E4F96E
:10CFB00034F8027C82467FBABBB207939DF82030DA
:10CFC0009BB1DFF8ACB008AF207F90B110F00CFF40
:10CFD000227F92B1204A2149CDE90201CDE90072B8
:10CFE0005B465146079A2348A3E7DFF868B05F46DF
:10CFF000EAE7184A10461146EEE7174A1549EBE7EB
:10D0000018481CF039FE35E72346174900901748A9
:10D010001CF032FEC0E61C2909D125B1CDE9014042
:10D02000154B009252E7234613490090EFE70C2975
:10D0300026D125B1CDE90140104B009246E72346A9
:10D040000E490090E3E700BF851B0400381C040074
:10D050000C110400EC6704002B0A0400773D040067
:10D06000461C04006C1C04007E1C0400831C04008D
:10D07000321C0400581C0400F32D0400DD1A0400C7
:10D0800035B10B46CDE901200321044A00941FE786
:10D090001346009022460148BAE700BF9D1C0400D9
:10D0A00010F1650F10B514460CD132B12046BDE821
:10D0B00010400321104A1EF0F2B90F48BDE810409D
:10D0C0001CF0DABD643015D1A1B1002300220B4859
:10D0D0002CF0F6F8031E0DDA34B12046BDE81040FE
:10D0E0000321074A1EF0DBB91946BDE81040044889
:10D0F0001CF0C2BD10BD00BFD31C0400F42A0020E8
:10D10000FA1C040070B501298CBF5668364E9AB0DF
:10D11000044636482CF0DBF811F03AF860B93CB11F
:10D1200003212046324A1EF0BAF96FF0070519E0D4
:10D130002F481CF0A1FDF8E74FF4FA63CDE9014355
:10D140002C4B0C22009331460DF1160328F071FF91
:10D15000051E10DA4CB1334603212046264A0095BD
:10D160001EF09DF928461AB070BD2A463146224865
:10D170001CF082FDF6E7F4B13346082120461F4A31
:10D180001EF08DF900254FF224420023174806A90E
:10D1900019F00CF8002818DB9DF81830062BF2D196
:10D1A000079B0EAA64B1009208212046144A1EF083
:10D1B00076F90135E7E7314610481CF05DFDE1E7FF
:10D1C00019460F481CF058FDF3E73CB12B460821E7
:10D1D00020460C4A1EF063F90025C3E7294609489A
:10D1E0001CF04AFDF8E700BF131D0400F42A0020DC
:10D1F000851B0400A1D00000301D0400491D04005F
:10D200005F1D0400671D04002DE9F041D2F8048081
:10D210000446A6B0B8F1000F0ED148B10321784AF8
:10D220001EF03DF96FF00705284626B0BDE8F081F5
:10D2300073481CF021FDF5E772482CF048F810F017
:10D24000A7FF064630B91CB1032120466E4AE7E726
:10D250006D48EEE74FF4FA636C4FCDE901430C22C1
:10D26000414600970DF1160328F0E3FE051E0EDA85
:10D270003CB1434603212046654A00951EF00FF954
:10D28000D2E72A46414662481CF0F6FCCCE7E4B1FE
:10D290004346082120465F4A1EF001F94FF000087E
:10D2A0004FF224420023574812A918F07FFF0028AC
:10D2B000C0F2A4809DF84830062B00F29380DFE88E
:10D2C00003F06209269191913D00414651481CF0BE
:10D2D000D3FCE3E71023012006AA15A908F054FFA8
:10D2E00003465CB14C4ACDF80080002808BF1346C5
:10D2F0004A4A082120461EF0D2F8D1E74246464964
:10D30000002818BF014645481CF0B6FCC8E72E238C
:10D31000022006AA15A908F037FF03463CB13E4A91
:10D32000CDF80080002808BF13463D4AE1E73A499E
:10D330004246002818BF01463948E5E7139B1AAD5D
:10D34000DCB108212046374A00951EF0A8F8139B4F
:10D35000354A2F21009506A81AF08CFE4FF4FA6387
:10D360002122CDE9014300970DF11603304606A9AD
:10D3700028F05FFE051E93DA56E72A46194629482B
:10D380001CF07AFCE3E79DF84C20022A2AD1BDF874
:10D390005010BDF85220BDF85430169817ADDCB1CE
:10D3A000CDE90023CDE902050B46204608211F4A9E
:10D3B0001EF075F8169B1C4A2F21009506A8BDF893
:10D3C00054801AF057FE4FF4FA631C22CDE9014352
:10D3D00000970DF11603C9E7CDE9000513481CF0CD
:10D3E0004BFCE7E72CB103212046114A1EF057F809
:10D3F00056E719460E481CF03FFC51E7002513E79D
:10D40000871D0400F42A0020851B0400A1D0000021
:10D41000A41B04009F1D04007D1D0400BF1D04000B
:10D42000CE1D0400E01D04004F1E0400EF1D04008B
:10D43000021E040030B510F1650F03460C46154678
:10D4400091B009D112B1494A03216CE0474811B0AB
:10D45000BDE830401CF010BC10F1640F5DD1002914
:10D4600070D00B78062B4DD8DFE803F02B04174C57
:10D470004C4C1C002F23012004AA0C3108F084FE20
:10D4800000238DF83E30002D42D008212846384A2E
:10D4900004AB1EF004F811B030BD2F23022004AA03
:10D4A0000C31EBE72E22002104A82CF093FF6268D8
:10D4B00004F120012E2A28BF2E2204A82CF064FF9C
:10D4C000DEE70B79012B0BD12E22002104A82CF0D2
:10D4D00081FFA26804F10C012E2A28BF2E22ECE75E
:10D4E000022B0FD101F1140303930B69214A02931C
:10D4F0008B8904A801934B8900930B892F211AF083
:10D50000B9FDBDE72E221C4904A82CF0CFFFB7E7D8
:10D51000174804A91CF0B0FBBDE710F1670F0AD152
:10D520003AB10821154A284611B0BDE830401DF037
:10D53000B6BF12488BE7021D04D10DB1104A83E734
:10D540000F4884E7F9F7EAFF0E4A125835B1009206
:10D55000032128460C4A1DF0A2FF9CE719460A4801
:10D5600011B0BDE830401CF087BB00BF221E040094
:10D57000691E0400461E0400541E0400721E0400AE
:10D580008D1E04000C000000A71E040038B5134BCC
:10D59000154604461B7898B1114A1249002B18BF52
:10D5A0001146114A0B4608211DF079FF6B682BB913
:10D5B0007CB1022120460D4A1DF071FF002038BDCC
:10D5C000084A07490848002B08BF11461CF054FBC5
:10D5D000ECE706481CF050FBF0E700BF938000200A
:10D5E000242004002C2004003520040056200400D0
:10D5F00070B5044694B016460021402204A81D468A
:10D600002CF0E8FEE3681899402B1A4628BF402208
:10D610000395CDE9012600911BB1A16804A82CF067
:10D62000B3FE002340F23912694607482BF048FE4A
:10D63000031E07DA05480268520703D00121044A95
:10D640001DF01BFA14B070BD282B0020B02800205C
:10D650009520040070B5274E0446337888B073B126
:10D6600040B10221244B254A1DF019FF6FF007003D
:10D6700008B070BD204921481CF0FEFAF6E74FF0D3
:10D68000FF304FF0FF316FF00D02CDE90601CDE91B
:10D690000232CDE9004304934FF48062184B1949DC
:10D6A000194819F061FB054650B92CB101212046FB
:10D6B000164A1DF0F4FED9E714481CF0DDFAD5E750
:10D6C000134919F007FA7CB1022120460A4B114A8E
:10D6D0001DF0E5FE0123002433700F4B1C7028461B
:10D6E00019F01EFB2046C3E703490A481CF0C4FAA0
:10D6F000F0E700BF9380002024200400B020040045
:10D700001DD70000B8C40020183E0020D920040016
:10D71000052104000F2104009280002000222DE941
:10D72000F04DA849A84CA94BB0B006460846C1E93F
:10D7300004234C6009F082F84FF0FF326FF0FE5383
:10D74000A349DFF890820846C1E904234C6009F040
:10D7500075F84FF0FF32A049A04B0846C1E90423F9
:10D760004C6009F06BF84FF0FF326FF07A639C4920
:10D770009C4D0846C1E904234C6009F05FF898F815
:10D780000030FBB18F4809F081F8914809F07EF82C
:10D79000914809F07BF8924809F078F892482BF00C
:10D7A00096FD0023914A88F800301370002E00F097
:10D7B000ED83022130468E4B8E4A1DF070FE30B054
:10D7C000BDE8F08D4FF0FF324FF0FF3386481CA9C3
:10D7D00018F0ECFCDDE91E32DDF870C0BCF1000F82
:10D7E00005D153EA020102D11D990029C7D0C2F325
:10D7F00001700128804F35D18049013B42EB010285
:10D80000082B72F1000280F07A83072B00F27783F5
:10D81000DFE813F0C103C303750326007503750326
:10D8200075030800764A0024764B77491C98002E31
:10D8300040F08D83CDE90A32099107F05BFFDDE905
:10D8400009130B9A002C00F09E83DFF8ACC1CDE9E0
:10D850000072CDE902C402466C481CF00DFA8EE756
:10D860006B4AE0E7022840F081824FF0080E6949D8
:10D870009E4571EB0204C0F0DF8000249C42914180
:10D8800013D3802064498A4208BF834200F01E827D
:10D89000984271EB02005AD39E4571EB02003FD3D0
:10D8A0009C4291411ED35D4C2AE35D49013B42EB12
:10D8B0000102082B72F10002F5D2072BF3D801A266
:10D8C00052F823F085DB000099DB0000A7D80000A8
:10D8D000A9DB0000A7D80000A7D80000A7D8000047
:10D8E000BBDB00004F49013B42EB0102082B72F108
:10D8F0000002D8D2072BD6D801A252F823F000BFDD
:10D9000067DC000079DC0000A7D8000089DC00009B
:10D91000A7D80000A7D80000A7D800009BDC000013
:10D920008A4208BF202B00F0C0818A4208BF402BEA
:10D9300000F0C3818A4208BF102BB4D10CAA012089
:10D9400020A920F0A4F80446374A384B22E14FF4CE
:10D9500000608A4208BF834200F0C081984271EBA8
:10D96000020013D38A4208BFB3F5007F00F017838B
:10D970008A4208BFB3F5806F00F0148326498A42BB
:10D9800008BFB3F5807F8ED1294A0CE38A4208BFD5
:10D99000B3F5005F00F0AB818A4208BFB3F5804F5A
:10D9A00000F0AE811C498A4208BFB3F5805F7FF466
:10D9B0007AAF0CAA012020A920F069F81D4A04467C
:10D9C00093E100BF303F0020F1D50000000010D0EF
:10D9D000183F002092800020003F0020FFFF4FE012
:10D9E000E83E0020EC670400282B002093800020F4
:10D9F0002C2004000F210400A4420400FFFFEF2F9D
:10DA000036210400E247040030210400EF22040024
:10DA10003F210400000040E0000030E0332104001A
:10DA2000FFFFBF1FFFFFCF1F63210400012204007F
:10DA300081180400962104004FF480548A4208BFE4
:10DA4000A34200F0EA809C4271EB02044ED34FF4F3
:10DA500080748A4208BFA34200F0C8809C4271EBE8
:10DA6000020429D340248A4208BFA34200F0B680B2
:10DA70009C4271EB020012D38A4208BF102B00F0C7
:10DA8000A48012F1FE5F08BF202B7FF40CAF0CAA1C
:10DA9000022020A91FF0FBFF9D4A04469CE08A4219
:10DAA00008BF802B7FF4FFAE0CAA022020A91FF034
:10DAB000EEFF984A044697E08A4208BFB3F5806FAC
:10DAC00000F09C808A4208BFB3F5006F00F09E8092
:10DAD0008A4208BFB3F5007F7FF4E5AE0CAA0220AE
:10DAE00020A91FF0D4FF8A4A044685E04FF4801431
:10DAF0008A4208BFA34200F059829C4271EB0204A3
:10DB00002ED34FF400448A4208BFA34200F0958010
:10DB10009C4271EB020015D38A4208BFB3F5005F47
:10DB200000F0838012F1FE5F08BFB3F5804F7FF4F1
:10DB3000BAAE0CAA022020A91FF0A9FF0446764A1B
:10DB4000764B27E08A4208BFB3F5002F7FF4ABAED7
:10DB50000CAA022020A91FF09AFF714A044618E07F
:10DB60008A4208BFB3F5800F6ED08A4208BFB3F572
:10DB7000000F71D08A4208BFB3F5001F7FF493AE47
:10DB8000684A14E20CAA022020A91FF080FF044674
:10DB9000614A654B654949E60CAA022020A91FF09D
:10DBA00076FF5B4A0446F4E70CAA022020A91FF086
:10DBB0006EFF0446584A5E4BECE70CAA022020A9EF
:10DBC0001FF065FF524A0446F5E70CAA022020A97F
:10DBD0001FF05DFF0446504A564BDBE70CAA20A914
:10DBE0001FF055FF0446544A544BD3E70CAA20A912
:10DBF0001FF04DFF0446484A514BCBE70CAA20A921
:10DC00001FF045FF0446444A4E4BC3E70CAA20A927
:10DC10001FF03DFF3E4A0446F6E70CAA20A91FF07C
:10DC200036FF0446484A494BB4E70CAA022020A913
:10DC30001FF02DFF464A0446F5E70CAA20A91FF065
:10DC400026FF334A04467BE70CAA20A91FF01FFFDA
:10DC50000446314A3F4B9DE70CAA20A91FF017FF4D
:10DC60002B4A0446F6E70CAA012020A91FF00FFF5B
:10DC70000446294A384B8DE70CAA012020A91FF041
:10DC800006FF234A0446F5E70CAA012020A91FF04D
:10DC9000FEFE0446204A314B7CE70CAA012020A955
:10DCA0001FF0F5FE1A4A0446F5E70CAA012020A948
:10DCB0001FF0EDFE164A044647E60CAA012020A9F3
:10DCC0001FF0E5FE0446144A254B63E70CAA012029
:10DCD00020A91FF0DCFE0E4A0446F5E70CAA01203D
:10DCE00020A91FF0D4FE0446134A1E4B52E70CAA8B
:10DCF000012020A91FF0CBFE0446134A1A4B49E726
:10DD00000CAA012020A91FF0C2FE114A0446F5E723
:10DD10005F2104009621040063210400C421040053
:10DD20009C1204002C200400522104003321040022
:10DD3000672104007A210400862104008B2104005D
:10DD40009C210400A8210400B3210400B621040092
:10DD5000BF210400D2210400E1210400EE210400CF
:10DD60000D2204001822040023220400032840F09E
:10DD7000208120209B498A4208BF834200F01E81F7
:10DD8000984271EB020058D30820984271EB0200D0
:10DD90004DD300209842914109D39349581E42EB3C
:10DDA0000104082874F1000422D3904CA8E09049A3
:10DDB000013B42EB0102082B72F10002F5D2072B66
:10DDC000F3D801A252F823F0E9DD0000C3DF000020
:10DDD000ABDD0000D9DE0000ABDD0000ABDD0000F4
:10DDE000ABDD0000DFDE0000824A834B00247FE0D1
:10DDF000013B42EB0101082871F10001D5D207284F
:10DE0000D3D801A353F820F0C9DF000029DE0000B9
:10DE1000ABDD0000F5DE0000ABDD0000ABDD000097
:10DE2000ABDD0000FBDE0000744A754BDEE78A4282
:10DE300008BF102BB9D1734AC1E04FF480608A4209
:10DE400008BF834200F0C280984271EB020021D3E8
:10DE50004FF480708A4208BF834200F0BA80984233
:10DE600071EB02000FD38A4208BF402B39D012F168
:10DE70007B6F08BF802B98D10CA920A81FF00AFE49
:10DE8000614A044633E08A4208BFB3F5007F8CD173
:10DE90005E4A9CE04FF400508A4208BF834200F083
:10DEA0009B80984271EB02000ED38A4208BFB3F503
:10DEB000006F00F0948012F17B6F08BFB3F5805FB4
:10DEC0007FF473AF524A8BE08A4208BFB3F5804FAC
:10DED0007FF46BAF4C4A80E04A4A4E4B86E74E4A8D
:10DEE000FBE70CA920A81FF0D5FD04464B4A4C4B7C
:10DEF0003E499BE44B4A4C4B78E74C4AFBE74C4C81
:10DF000060469EB107F0F6FBDDE91E23CDE906234E
:10DF1000484B0221CDE90003CDE9045523463046A4
:10DF2000CDE90275444A1DF0BAFA28E407F0E2FB95
:10DF3000DDE91EAB02462146CDE904ABCDE9025531
:10DF4000CDE900753B4B3C481BF096FE17E4CDE94C
:10DF50000A32099107F0CEFBDDE909130B9A7CB177
:10DF6000DFF8D8C0CDE90003CDE902720B46304698
:10DF70000221CDE904C4324A1DF091FAFFF7FFBB3C
:10DF80002C46AC46EEE71B4CA44660E42D492E48D7
:10DF90001BF072FE13E42D4A45E42D4A43E42D4A5A
:10DFA0002D4BF7E52D4A2C4B0024F3E52C4A2D4B45
:10DFB000FAE72A462B4600242B4937E4164A2B4B16
:10DFC00014E70C4A124B11E7104A2EE70B4A284B74
:10DFD0000CE7084A274B09E7104A274B06E7064A91
:10DFE000264B03E7000050F0FFFF9F4F2D21040058
:10DFF000FFFFAF0FEC670400B08204007B22040037
:10E000006E2204004C1004005F210400662204000C
:10E010009E8204002C2204003E220400632104009E
:10E02000B022040083220400892204009722040005
:10E030003021040025940400CB220400A4420400F3
:10E04000EF2204002C2004000F2104006665040068
:10E05000C62C0400122E0400FB17040087180400CD
:10E06000242004004A210400BB22040043220400AF
:10E070009F22040055220400A72204004C580400EB
:10E0800038B5144B04461B786BB938B10221124BDA
:10E09000124A1DF004FA6FF0070038BD0E490F4810
:10E0A0001BF0EAFDF7E701250D4B1D70002340F63C
:10E0B00035420C490C482BF003F9031E07DA1CB15A
:10E0C00029462046094AE4E719460848E8E70020BF
:10E0D000E3E700BF938000202C200400B020040060
:10E0E0009280002098C00300282B00209520040077
:10E0F00008B5F6F7C3FFBDE808400121014AFFF764
:10E10000A9BA00BFF8CD030007B550B1084B0221F2
:10E110000093084A084B1DF0C2F9002003B05DF8D7
:10E1200004FB034A044903481BF0A6FDF5E700BFC2
:10E1300089230400051304007723040007B550B1B8
:10E14000084B02210093084A084B1DF0A8F9002053
:10E1500003B05DF804FB034A044903481BF08CFD3F
:10E16000F5E700BF892304000513040077230400AA
:10E1700007B550B1084B02210093084A084B1DF027
:10E180008EF9002003B05DF804FB034A04490348FC
:10E190001BF072FDF5E700BFA9250400051304007C
:10E1A0009925040007B550B1084B02210093084A95
:10E1B000084B1DF074F9002003B05DF804FB034A1E
:10E1C000044903481BF058FDF5E700BF2126040071
:10E1D000051304000E26040007B550B1084B0221B8
:10E1E0000093084A084B1DF05AF9002003B05DF86F
:10E1F00004FB034A044903481BF03EFDF5E700BF5A
:10E20000A525040005130400CB26040007B550B172
:10E21000084B02210093084A084B1DF040F90020EA
:10E2200003B05DF804FB034A044903481BF024FDD6
:10E23000F5E700BF38270400051304002527040074
:10E2400008B530B10321054A1DF029F96FF0070028
:10E2500008BD02481BF010FDF8E700BF6F2704005F
:10E2600070B5012106461FF045FC044620B1334934
:10E270003348F3F761F90C24022130461FF03AFCD1
:10E280002F4D30B1C4F1510128192E4A19F0F2FE78
:10E290000834032130461FF02DFC0346C4F1510120
:10E2A0002819002B45D0284A19F0E4FE0E34052128
:10E2B00030461FF01FFC30B1C4F151012819234A28
:10E2C00019F0D8FE0E34062130461FF013FC30B191
:10E2D000C4F1510128191E4A19F0CCFE053407215A
:10E2E00030461FF007FC30B1C4F151012819194A1A
:10E2F00019F0C0FE05340B2130461FF0FBFB30B196
:10E30000C4F151012819144A19F0B4FE06340C2145
:10E3100030461FF0EFFB30B1C4F1510128190F4A0C
:10E3200019F0A8FE07340023254405F8013C0448F1
:10E3300070BD0B4A19F09EFE0B34B8E7CA270400E3
:10E3400094800020D7270400E0270400EF27040072
:10E35000FE270400042804000A28040011280400F1
:10E36000E32704002DE9F04F4B6805460E468DB0BB
:10E370000BB183425DD100230822284609A9CDE9CB
:10E38000093334688DF82C3021F0EAFD002802DDD5
:10E390009DF824301BB9844909A8F3F7CDF8284625
:10E3A00008A92CB3FEF724F90746284607F0A2F97E
:10E3B0000821CDE901707D4A204609AB00951DF08A
:10E3C0006EF808212046089B794A1DF068F845B38D
:10E3D00028461FF098FB10B305F118064FF0FF32E6
:10E3E0004FF0FF33304617F045FF2DBB6B78FFDE53
:10E3F000FEF7FEF80746284607F07CF909A90090C9
:10E400003B466A482A461BF037FC089968481BF0CF
:10E4100033FC002DDCD167481BF02EFC06E0002CFD
:10E42000F9D002212046634A1DF039F87368002BA9
:10E43000D2D10DB0BDE8F08F2868417C61B11823BE
:10E440005D4A1230002C6FD007F072FE082103469F
:10E450005A4A20461DF023F8304617F07DFF2B68FE
:10E46000002C68D008215B8B554A20461DF017F818
:10E470002846FFF7F5FE534A0346082120461DF0C3
:10E480000EF82B681A68002A40F083804E4B082152
:10E49000204600924D4A1DF002F82B684C4E187F22
:10E4A00007F040FC0021024628461FF023FB494BA1
:10E4B000884218BF1E46092128461FF01BFB46490B
:10E4C000464B002818BF0B460821CDE900632046C3
:10E4D0001346434A1CF0E3FF072128466E681FF0ED
:10E4E00009FB10B1002E40F08580002C55D03D4B2B
:10E4F0000821009320463C4B3C4A1CF0D0FF0621EB
:10E500002846AE681FF0F6FA10B1002E40F04A829D
:10E51000002C00F04182334B082100932046344BFD
:10E52000324A1CF0BCFF84E707F002FE0146234894
:10E530001BF0A2FB90E7598B21481BF09DFB28465E
:10E54000FFF78EFE01461F481BF096FB2B681A68EA
:10E550000ABB1D491D481BF08FFB2B68187F07F075
:10E56000E1FB0021064628461FF0C4FA194A184B61
:10E57000884208BF1A46092128461FF0BBFA1749EE
:10E58000154B002808BF0B46314615481BF074FB9D
:10E59000A2E713687BE71168DCE7124A12491348C7
:10E5A0001BF06AFBABE700BF4F28040051280400B2
:10E5B000993904006F280400E580002083280400B6
:10E5C00093280400A328040019280400B328040099
:10E5D000C98104001D280400C8850400D5850400F5
:10E5E000C828040024200400F32D0400F3280400AC
:10E5F0007E1C0400002C00F0178102230821204615
:10E60000BE4A1CF04CFF4FF00008C146371D06EB18
:10E61000881A9AF83D309B0731D539460220002CE4
:10E6200000F0078107F0A8FE079097F82400FDF797
:10E630004BFF834697F92500FDF752FF9AF83DC03E
:10E64000AF4A1CF0010FAF4B08BF13461CF0040F7C
:10E65000AD4908BF11461CF0080FDFF8B0C2CDE984
:10E66000010318BF62462046CDE90312079B08212B
:10E67000A74ACDF800B01CF012FF09F1010908F11A
:10E680000103022B4FF0010807F14007BFD1B9F198
:10E69000000F40F0FF80002C00F0F480082120469D
:10E6A0009C4A1CF0FCFE0323082120469A4A1CF0D9
:10E6B000F6FE0027BA46DFF848B206F1840906EBF9
:10E6C000471393F89C30D80719D5494602204FEAE2
:10E6D0004718002C00F0E280B04407F04DFE98F897
:10E6E0009C20034612F0020F8C4A18BF5A4608219C
:10E6F000009220468A4A1CF0D2FE0AF1010A013734
:10E70000032F09F12009DAD1BAF1000F40F0DE80C1
:10E71000002C00F0D380082120467E4A1CF0BFFE6A
:10E720000223082120467F4A1CF0B9FE4FF0000862
:10E730004FF0280AC14606F1F0070AFB086303F10F
:10E74000E00B93F80531990719D539460220002CC2
:10E7500000F0C08007F010FE9BF8252003466948B2
:10E7600012F0010F664A18BF0246397D2046CDE9F6
:10E77000001208216C4A1CF092FE09F1010908F10F
:10E780000103022B4FF0010807F12807D5D1B9F199
:10E79000000F07D1002C00F0AD80082120465D4A13
:10E7A0001CF07DFE0021284621F02AF807460028AB
:10E7B00000F0EE8000F10808002C00F0C1805B4AF8
:10E7C000082120461CF06BFE4146022007F0D4FDD4
:10E7D00097F822204B4912F0040F494A18BF0A4605
:10E7E00003460092082120464D4A1CF058FE204660
:10E7F00096F8453108214E4A1CF051FE2046D6F8C5
:10E80000303108214B4A1CF04AFE2046D6F83431FC
:10E810000821494A1CF043FE08212046D6F8383129
:10E82000464A1CF03CFE6AE6022134481BF024FAFA
:10E83000E9E607F0A1FD079097F82400FDF744FEF4
:10E84000834697F92500FDF74BFE9AF83D202C4BA7
:10E8500012F0010F2B4908BF194612F0040FDFF820
:10E86000A8C008BF9C4612F0080F284A08BF1A46E5
:10E8700000910346CDE901C207995A4624481BF08E
:10E88000FBF9FAE623481BF0F7F9032122481BF0B5
:10E89000F3F90EE7002C7FF406AFF6E707F06CFD06
:10E8A000B04498F89C30014613F0020F144B1B4AF9
:10E8B0001B4818BF1A461BF0DFF91EE715481BF06E
:10E8C000DBF9022117481BF0D7F92FE7002C7FF462
:10E8D00027AFF6E707F050FD9BF82530084A13F004
:10E8E000010F0146074B104808BF13463A7D1BF045
:10E8F000C3F942E707481BF0BFF953E712290400A8
:10E90000EC670400202804002A28040035280400AD
:10E9100034290400452904004E290400402804003D
:10E92000722904007929040024400400922904007B
:10E93000A9290400C8290400E7290400062A0400C4
:10E9400081481BF099F94146022007F015FD97F820
:10E950002230014613F0040F7C4B7D4A7D4818BFDE
:10E960001A461BF089F996F845117B481BF084F98B
:10E97000D6F8301179481BF07FF9D6F83411784871
:10E980001BF07AF9D6F8381176481BF075F9B6E520
:10E99000002C7FF42CAFE6E7734A744974481BF0EF
:10E9A0006BF946E584B1012308212046714A1CF029
:10E9B00076FD96F83D309A070BD4002C40F09E80EF
:10E9C0006D481BF059F994E001216A481BF054F995
:10E9D000EFE70120311D06F14007002C68D007F059
:10E9E000CBFC39460546012007F0C6FC074696F8E1
:10E9F0002800FDF769FD804696F92900FDF770FDB6
:10EA000096F83D30514A13F0010F514B18BF134691
:10EA10000821CDE90203CDE900782B462046574A6C
:10EA20001CF03DFD022308212046554A1CF037FD0D
:10EA30000027B84606F1480906EB471393F8603003
:10EA4000DB0718D5494601207D01002C5CD03544F8
:10EA500007F092FC95F860203D4912F0020F494AF8
:10EA600018BF0A460346009208212046394A1CF086
:10EA700016FD08F101087B1C022B4FF0010709F17C
:10EA80002009D9D18436B8F1000F59D1002C4BD0D0
:10EA900008212046384A1CF002FD3146012007F0CB
:10EAA0006BFC08210346384A20461CF0F8FCC0E401
:10EAB00007F062FC39460546012007F05DFC074679
:10EAC00096F82800FDF700FD804696F92900FDF72D
:10EAD00007FD96F83D301D4A13F0010F1C4B18BF7F
:10EAE00013462946CDE900033A46434623481BF026
:10EAF000C3F8022122481BF0BFF899E708212046FD
:10EB00001D4A1CF0CCFC8DE707F036FC354495F827
:10EB10006030014613F0020F0D4B1A4A0D4818BF22
:10EB20001A461BF0A9F8A4E713481BF0A5F83146D4
:10EB3000012007F021FC014613481BF09DF878E402
:10EB4000002CAAD1F3E700BF92290400202804007A
:10EB5000EC67040072290400A9290400C8290400F4
:10EB6000E7290400062A0400242004007E1C040077
:10EB7000F3280400252A040045290400472A04003C
:10EB8000572A0400402804007B2A040073B551680A
:10EB90000546FDF759FC041E0ADB05F03BFB064663
:10EBA00070B945B123461D4A032128461CF077FC65
:10EBB0006FF0070629E0214618481BF05DF8F7E7DB
:10EBC0001EF0A1FF30B115B12346154AECE72146EE
:10EBD0001348F2E7304607F0B1F8064670B13DB190
:10EBE00000902346032128460E4A1CF058FCDFE71C
:10EBF000024621460B481BF03FF8D9E745B12346B2
:10EC000008212846084A1CF04AFC304602B070BD74
:10EC1000214605481BF030F8F7E700BF8E2A0400B4
:10EC2000AD2A0400CA2A0400EC2A040073B5516816
:10EC30000546FDF709FC041E09DB05F0EBFA70B987
:10EC400045B1234603212846164A1CF028FC6FF0E4
:10EC500007061EE0214613481BF00EF8F7E707F001
:10EC6000B3F8064670B13DB1009023460321284613
:10EC70000D4A1CF014FCEAE7024621460A481AF045
:10EC8000FBFFE4E745B1234608212846074A1CF06C
:10EC900006FC304602B070BD214604481AF0ECFF75
:10ECA000F7E700BF8E2A0400002B0400242B040089
:10ECB000012938B504461FD805F036FB60B93CB1D0
:10ECC000032120461D4A1CF0EAFB6FF0070012E00A
:10ECD0001A481AF0D1FFF8E706F00CFD03462CB1F4
:10ECE00008212046164A1CF0DAFB03E001461448CE
:10ECF0001AF0C2FF002038BD5168FDF7A5FB051EC4
:10ED0000E3DB05F087FA05F009FB05F00DFB06F0E3
:10ED1000F1FC85420CD034B12B4603212046094A30
:10ED20001CF0BDFBD1E7294606481AF0A5FFCCE749
:10ED30000CB12B46D4E72946D9E700BF3A2B040093
:10ED4000502B0400672B040073B555680446C5B109
:10ED50002946FDF779FB061E0ADB05F05BFA05463E
:10ED600078B94CB13346032120461B4A1CF097FB6F
:10ED70006FF0070002B070BD314617481AF07CFFF3
:10ED8000F6E7CCB1FBF7B8FD08210346134A20464D
:10ED90001CF085FB05F0C8FA06F0ACFC0821034620
:10EDA0000F4A20461CF07BFB0E486946CDE9004522
:10EDB00006F0A6FF0020DDE7FBF79EFD01460748B1
:10EDC0001AF05AFF05F0B0FA06F094FC0146044828
:10EDD0001AF052FFE8E700BF8E2A04008E2B0400D1
:10EDE0009C2B040065E30000F0B5002787B00546C2
:10EDF0000E46CF6005F00EFA04464DB3A0B1012DCA
:10EE000028D1082203A921F0ABF8394620468DF815
:10EE10001470FDF7EDFB1C21CDE90004104A1148E8
:10EE200003AB19F027F90F4C0F4B7460B360284601
:10EE300005F0F0F985B140B1012D0FD12B46042129
:10EE40000A4A0B4819F016F90948306007B0F0BDBE
:10EE5000084CE9E73C46E7E70648F6E70020F4E718
:10EE6000B42B040001810020ECBF03000C1104004E
:10EE7000FD800020EC67040018B1012801D00228B1
:10EE800003D1034B53F8300070470248704700BF6E
:10EE9000D8D20300C92C04002DE9F3411D460023FC
:10EEA00001932B6804468B42DDF820800CD338B1E7
:10EEB00001211B4A1CF0F3FA03236FF0150729E028
:10EEC00017481AF0D9FEF7E752F823600A213046B6
:10EED00001AAF7F75DF8019F67B134B13346114AD3
:10EEE000012120461CF0DBFAE6E731460D481AF016
:10EEF000C3FEE1E705F08EF9C8F8040030B914B19B
:10EF00003346094AECE731460748F0E72B680133FE
:10EF10002B603B46384688F8003002B0BDE8F081EF
:10EF2000D12C0400F92C04001B2D040018B1082179
:10EF3000024A1CF0B4BA01481AF09EBE422D0400E9
:10EF4000F0B587B004AF0D4608223946044621F0DB
:10EF500007F818B138460B49F2F7EEFA204606F0EA
:10EF6000C9FB002106462046FDF742FB3346CDE9AA
:10EF7000017030212846044A009419F07BF807B04C
:10EF8000F0BD00BF892D0400912D040030B5054669
:10EF90000C468DB06946FFF7D3FF28460FF058FAAC
:10EFA0003CB16B4608212046044A1CF078FA0DB0AB
:10EFB00030BD694601481AF05FFEF8E7A32D040052
:10EFC00030B505460C468DB06946FFF7B9FF2846B7
:10EFD0000FF05CFA3CB16B4608212046044A1CF055
:10EFE0005EFA0DB030BD694601481AF045FEF8E7FB
:10EFF000BA2D04002DE9F0411C6806468C421D46DE
:10F00000069F16D252F82480104940462BF0FEF994
:10F0100028B901342C6038700020BDE8F0814046EA
:10F020000B492BF0F3F920B9012301342C603B701C
:10F03000F2E73EB101213046064A1CF030FA6FF08B
:10F040001500EAE703481AF017FEF8E7DBF10300C2
:10F050007A8B0400D12D0400F0B593B004460E461F
:10F060000FF048FA06A905462046FFF769FF4FF65C
:10F07000FF739D420DD13EB108213046394A06AB9F
:10F080001CF00DFA13B0F0BD364806A91AF0F4FDD5
:10F09000F8E7204605F0800727F066F82CB12368D2
:10F0A0000C33D3E8AF4F04F001046A0705F0010EFA
:10F0B00005F0020305F4005C47BF2B4A2B4D2C4D95
:10F0C0002C4A002B18BF15463EB32B4A2B4B2C491C
:10F0D000002F18BF13462B4A2B4F002818BF0A4693
:10F0E0002A482B49CDE90032002C18BF0146294C93
:10F0F00029482A4ABEF1000F18BF2046284CCDE906
:10F100000210BCF1000F18BF3C4608213046CDE983
:10F11000045406AB1CF0C3F9B4E71C4A1C4B1E494F
:10F12000002C18BF13461B4A174CBEF1000F18BF26
:10F1300011461B4ACDE90031BCF1000F18BF224631
:10F140000F4BCDE902520F4A0C49002808BF134665
:10F15000094A1248002F08BF0A4606A91AF08CFD7A
:10F1600090E700BF382E0400EC2D04007E1C040044
:10F17000F82D0400F32D0400FE2D0400062E0400DB
:10F18000122E04000E2E0400B0820400BF350400CD
:10F190008D350400182E0400202E04004F2E04008C
:10F1A0002A2E04002DE9F04701290446884691469D
:10F1B0001D46089E01D8012307E0576835493846A7
:10F1C0002BF024F928B902232B6033700020BDE80E
:10F1D000F087384630492BF019F910B902232B601B
:10F1E000E9E738461EF09CFC38B12B464A464146BA
:10F1F0002046BDE8F047FFF74FBE384627492BF0C1
:10F2000005F9824670BB022398452B600ED14CB1A4
:10F2100001212046224A1CF042F903236FF0150019
:10F220003370D4E71E481AF027FDF6E7D9F80870C6
:10F23000384606F05BFE04F0EDFF706060B934B153
:10F240003B4601212046174A1CF029F9E5E73946DB
:10F2500014481AF011FDE0E72B6801332B6086F8A3
:10F2600000A0B3E7384610492BF0D0F810B90223BC
:10F270002B60BAE74CB13B46012120460B4A1CF0FB
:10F280000EF92046FFF752FEC7E7394607481AF045
:10F29000F3FCF6E7A58D0400792E04007E2E040011
:10F2A000812E0400A82E0400CE2E0400D22E0400CD
:10F2B000F0B5002787B0CDE904770125032704AB1B
:10F2C000009303AB04460E4603958DF81070FFF7CC
:10F2D00069FFB0B9039BB3420AD02CB1104A29464A
:10F2E00020461CF0DCF80CE00D481AF0C5FC08E0E4
:10F2F0009DF810305A1E012A06D82146094806F00A
:10F30000FFFC002007B0F0BD23B921460598FFF7A8
:10F31000A3FEF6E70CB1044AE1E70348E5E700BFC6
:10F32000062F040059F00000162F0400F0B5002746
:10F3300087B0CDE904770125032704AB009303AB25
:10F3400004460E4603958DF81070FFF72BFFC8B9E1
:10F35000039BB3420AD02CB11C4A294620461CF01C
:10F360009EF80FE019481AF087FC0BE09DF810108A
:10F3700001290ED14CB12046154A1CF090F82046C8
:10F38000FFF7D4FD002007B0F0BD11481AF074FC5F
:10F39000F5E702290ED14CB1082120460D4A1CF098
:10F3A0007EF821460C4806F0ABFCEBE709481AF062
:10F3B00063FCF6E721B921460598FFF7E7FDE1E791
:10F3C0000CB1064AC9E70548CDE700BF062F040087
:10F3D000302F04004A2F04008DEF0000162F040088
:10F3E000F0B5002787B0CDE904770125032704ABEA
:10F3F000009303AB04460E4603958DF81070FFF79B
:10F40000D1FEC8B9039BB3420AD02CB11C4A29468D
:10F4100020461CF044F80FE019481AF02DFC0BE0D0
:10F420009DF8101001290ED14CB12046154A1CF050
:10F4300036F82046FFF77AFD002007B0F0BD1148EE
:10F440001AF01AFCF5E702290ED14CB1082120462A
:10F450000D4A1CF024F821460C4806F051FCEBE75D
:10F4600009481AF009FCF6E721B921460598FFF78B
:10F47000A7FDE1E70CB1064AC9E70548CDE700BFA3
:10F48000062F0400302F0400602F0400C1EF00009D
:10F49000162F0400F0B5002793B0CDE904770125BD
:10F4A000032704AB009303AB04460E4603958DF887
:10F4B0001070FFF777FEC8B9039BB3420AD02CB196
:10F4C0002C4A294620461BF0EAFF0FE029481AF093
:10F4D000D3FB0BE09DF8101001290ED14CB1204652
:10F4E000254A1BF0DCFF2046FFF720FD002013B06B
:10F4F000F0BD21481AF0C0FBF5E702290DD144B157
:10F50000082120461D4A1BF0CAFF01200FF064FAB3
:10F51000ECE71A481AF0B0FBF7E729BB059E06A9ED
:10F520003046FFF70DFD304626F01EFE60B934B1BF
:10F5300029462046124A06AB1BF0B1FFD6E7104819
:10F5400006A91AF099FBD1E74CB1082120460D4AD3
:10F5500006AB1BF0A4FF30460FF024F9C6E70948BC
:10F5600006A91AF089FBF6E70CB1074AA9E7064895
:10F57000ADE700BF062F0400302F0400762F0400F3
:10F58000A62F0400EF2F0400162F0400F0B500276B
:10F5900093B0CDE904770125032704AB009303ABB7
:10F5A00004460E4603958DF81070FFF7FBFDC8B9B1
:10F5B000039BB3420AD02CB12C4A294620461BF0AB
:10F5C0006EFF0FE029481AF057FB0BE09DF8101072
:10F5D00001290ED14CB12046254A1BF060FF204680
:10F5E000FFF7A4FC002013B0F0BD21481AF044FB43
:10F5F000F5E702290DD144B1082120461D4A1BF030
:10F600004EFF01200FF000FAECE71A481AF034FB25
:10F61000F7E729BB059E06A93046FFF791FC304667
:10F6200026F0A2FD60B934B129462046124A06AB45
:10F630001BF035FFD6E7104806A91AF01DFBD1E7ED
:10F640004CB1082120460D4A06AB1BF028FF30467E
:10F6500026F0DCFDC6E7094806A91AF00DFBF6E71F
:10F660000CB1074AA9E70648ADE700BF062F040022
:10F67000302F0400113004004430040090300400A6
:10F68000162F0400F0B5002793B0CDE904770125CB
:10F69000032704AB009303AB04460E4603958DF895
:10F6A0001070FFF77FFD98B9039BB34207D014B1E8
:10F6B000234A294609E022481AF0DEFA08E09DF8BC
:10F6C0001010012909D134B11E4A20461BF0E7FE73
:10F6D000002013B0F0BD1B48EEE702290DD144B164
:10F6E00008212046184A1BF0DAFE01200FF050F9DD
:10F6F000EEE715481AF0C0FAF7E7E1B9059D06A94B
:10F700002846FFF71DFC74B1082120460F4A06ABBE
:10F710001BF0C5FE394620460D4A1BF0C0FE2846A8
:10F7200006F00CFBD4E7094806A91AF0A5FA084828
:10F730001AF0A2FAF3E70CB1064ABAE70548BBE7AC
:10F74000062F0400302F0400B5300400DE30040022
:10F75000F9300400162F0400F0B5002793B0CDE96E
:10F7600004770125032704AB009303AB04460E4640
:10F7700003958DF81070FFF715FDC8B9039BB342D0
:10F780000AD02CB1274A294620461BF088FE0FE0FC
:10F7900024481AF071FA0BE09DF8101001290ED1DF
:10F7A0004CB12046204A1BF07AFE2046FFF7BEFBF4
:10F7B000002013B0F0BD1C481AF05EFAF5E70229EC
:10F7C0000DD144B108212046184A1BF068FE0120E3
:10F7D0000FF0F0F8ECE715481AF04EFAF7E7E1B948
:10F7E000059D06A92846FFF7ABFB74B1082120460A
:10F7F0000F4A06AB1BF053FE394620460D4A1BF05C
:10F800004EFE284606F0E0FAD2E7094806A91AF0AB
:10F8100033FA08481AF030FAF3E70CB1064AB2E7B7
:10F820000548B6E7062F0400302F040035310400E8
:10F83000603104007D310400162F040000232DE9FF
:10F84000F04F93B0CDE904338DF80B3003234FF024
:10F85000010904AF8DF81030009703AB04460E4643
:10F860001546CDF80C90FFF79DFC58B99DF8101087
:10F8700049450FD154B120468E4A1BF010FE204658
:10F88000FFF754FB002013B0BDE8F08F89481AF051
:10F89000F3F9F4E702290AD12CB1874A0121204665
:10F8A0001BF0FDFDEEE784481AF0E6F9EAE721B126
:10F8B0000CB1824AF2E78148F6E70DF10B030093A1
:10F8C0002A463146204603ABDDF81480FFF792FB51
:10F8D00007460028D6D1DDF80CA0564523D8B4B190
:10F8E00049462046764A1BF0DAFD08212046754A33
:10F8F0001BF0D5FD744D55F837307CB108212046FA
:10F90000724A1BF0CCFD0137032FF4D1BAE76C48E3
:10F910001AF0B2F96B481AF0AFF9EBE719466B48E9
:10F920001AF0AAF9EFE755F82A70694938464FEA04
:10F930008A0B2AF06BFD50B1384666492AF066FD05
:10F94000A0B1384664492AF061FD88B902205E4AB8
:10F950009DF80B900AF1010302EBC002B9F1010F0F
:10F960001779039311D04FF0000A2BE04846EEE7D9
:10F9700034B13B46594A012120461BF090FD81E7F6
:10F98000394656481AF078F97CE7B34237D25D44DD
:10F990006D68534928462AF039FD70B1284651490F
:10F9A0002AF034FD48B128464F492AF02FFD20B1F6
:10F9B00028464E492AF02AFD48B90AF102034FF0C1
:10F9C000010A0393B34221D0F4B1494A66E72846BD
:10F9D00048492AF01BFD70B1284647492AF016FD18
:10F9E00048B1284645492AF011FD20B1284644492E
:10F9F0002AF00CFD18B90AF102030393B3E70CB126
:10FA0000404A4BE73F484FE739484DE706AD40468F
:10FA10002946FFF795FA404626F0A6FB30B914B107
:10FA20002B46394AA7E729463748ABE7B9F1010F1A
:10FA300023D139465246404626F09DFB3846FFF713
:10FA40001BFA014674B1274A2B4BBAF1000F18BFBD
:10FA50001346CDE9003503462C4A082120461BF009
:10FA60001EFD0FE72B4624481E4ABAF1000F08BFBF
:10FA7000024626481AF000F904E73946404626F0C7
:10FA800031FC02463846FFF7F7F901464CB11A4BF4
:10FA90001448002A18BF03461D4ACDE900530B46FF
:10FAA000DBE715480F4B002A08BF03462A461848D3
:10FAB000E0E700BF302F0400BB310400162F040024
:10FAC000E1310400F9310400D8D2030013320400FC
:10FAD000193204002432040034320400413204009C
:10FAE0005A3204009F8E04006C8004005E320400D1
:10FAF000062F040063320400EB7B04008C750400C5
:10FB0000663204006C3204008B320400E6320400DA
:10FB10001733040000232DE9F04792B0CDE90433F8
:10FB20008DF80B300323012504AE8DF810300096BC
:10FB300003AB0446884617460395FFF733FB58B9D5
:10FB40009DF81010A9420FD154B12046584A1BF01D
:10FB5000A6FC2046FFF7EAF9002012B0BDE8F087C6
:10FB600053481AF089F8F4E702290AD12CB1514A16
:10FB7000294620461BF093FCEEE74E481AF07CF82D
:10FB8000EAE721B10CB14C4AF2E74B48F6E70DF138
:10FB90000B0300933A464146204603ABDDF8149030
:10FBA000FFF728FA05460028D6D19DF80BA0BAF138
:10FBB000010F12D1039E0690464505D314B13F4A6A
:10FBC0000121D6E73D48D9E757F826703C49384629
:10FBD0002AF01CFC38B901360396039B43451FD01D
:10FBE000E4B1384AECE738461DF09AFF38B984B1E1
:10FBF0003B46354A012120461BF051FCACE70A2167
:10FC0000384606AAF6F7C4F9069B0546002BE2D053
:10FC1000EDE739462C481AF02FF89DE72948ADE763
:10FC2000484606A9FFF78CF9484626F09DFA30B9F8
:10FC300014B1264A06ABDDE7244806A9EBE7BAF182
:10FC4000010F1DD12946484626F062FB6CB1204ABF
:10FC5000204B002D08BF13461F4ACDE9005306ABC9
:10FC6000082120461BF01BFC76E71A4A184B1A485D
:10FC7000002D18BF13462A4606A919F0FDFF6BE7B1
:10FC8000484626F035FB02464CB1124B1049134A48
:10FC9000002808BF0B46CDE9000306ABE0E70D499D
:10FCA0000B4B002818BF0B460C4806A9E5E700BF20
:10FCB000302F040070330400162F04009833040022
:10FCC000792E0400062F0400C0330400DC33040046
:10FCD00059330400673304003A3404006E340400DE
:10FCE00013B50446002832D00821274B274A1BF0C1
:10FCF000D6FB08212046264B264A1BF0D0FB0821C4
:10FD00002046234B244A1BF0CAFB08212046204BE7
:10FD1000224A1BF0C4FB012308212046204A1BF085
:10FD2000BEFB0123082120461E4A1BF0B8FB02231C
:10FD3000082120461C4A1BF0B2FB009400246946AF
:10FD40001A48019405F0DCFF204602B010BD0E49B0
:10FD50000E4819F091FF0E490E4819F08DFF0C491D
:10FD60000D4819F089FF0A490C4819F085FF012157
:10FD70000B4819F081FF01210A4819F07DFF02218B
:10FD8000094819F079FFD8E72420040086360400DA
:10FD90002C200400B6360400E636040016370400B2
:10FDA0004637040089370400CC370400B500010051
:10FDB00003292DE9F3410446884616460ED048B182
:10FDC00001211F4A1BF06BFB6FF00705284602B0AC
:10FDD000BDE8F0811A4819F04FFFF5E75168FCF7CC
:10FDE00033FB051EF0DB04F015FA074660B934B1A9
:10FDF0002B4641462046134A1BF051FBE4E72946B7
:10FE0000104819F039FFDFE7B168012001AA06F0B8
:10FE1000C9FA054670B1B3683CB1012120460A4ACF
:10FE20001BF03DFB6FF01505D0E71946064819F0A9
:10FE300023FFF7E7384601A91FF03AFEC6E700BFE7
:10FE40000F3804008E2A0400453804002DE9F043E1
:10FE5000022904468946174687B00BD830B10121E4
:10FE60004C4A1BF01CFB6FF0150515E0494819F0D2
:10FE700003FFF8E75168FCF7E7FA061E0ADB04F017
:10FE8000C9F9804688B95CB1334603212046424A0D
:10FE90001BF005FB6FF00705284607B0BDE8F083AF
:10FEA00031463D4819F0E8FEF4E7B968012004AA9C
:10FEB00006F078FA054660B1BB682CB1374A0121DB
:10FEC00020461BF0ECFACEE71946344819F0D4FE70
:10FED000C9E7049B03F0F003E02B20D1024604A9FC
:10FEE000404608F0D7FA071ED6DA012004A964B10B
:10FEF00006F042FA01210090CDE901672046284B27
:10FF0000284A1BF0CCFA3D46C6E706F035FA3346E0
:10FF1000024623492348009719F0AEFEF3E7B9F1F2
:10FF2000030F06D11CB1012120461F4A99E71E4844
:10FF30009DE703460322404604A904F0A7FFB0B999
:10FF4000012004A95CB106F017FA01210346174A03
:10FF5000204600961BF0A3FA6FF00B059CE706F015
:10FF60000BFA32460146114819F086FEF4E7F968AB
:10FF7000012005AA06F016FA30B1FB680CB10C4A54
:10FF80009DE719460A48A1E7404605AA04A91FF0C3
:10FF900053FD81E75A3804008E2A040045380400D6
:10FFA0008621040095380400C9380400DE380400B6
:10FFB000053904002DE9F041032904460D46174692
:10FFC00086B00BD030B10121344A1BF068FA6FF0D3
:10FFD00015051AE0314819F04FFEF8E75168FCF7B3
:10FFE00033FA061E0FDB04F015F9804688B934B1E8
:10FFF000334629462A4A20461BF051FA03E031468F
:020000021000EC
:10000000274819F039FE6FF00705284606B0BDE80D
:10001000F081B968012005AA06F0C4F9054660B16F
:10002000BB682CB1012120461E4A1BF038FACEE7EE
:1000300019461C4819F020FEC9E7059B404603F00D
:10004000F003E02B05A91DD108F060FA071EDCDAE9
:10005000012005A964B106F08FF901210090CDE9D6
:1000600001672046104B114A1BF019FA3D46CCE7B8
:1000700006F082F9334602460B490C48009719F006
:10008000FBFDF3E71FF0CDFD0028BED1BB6814B126
:100090000121074AAFE719460548B2E719390400BC
:1000A0008E2A040045380400962104009538040087
:1000B000473904002DE9F04F0C680646856887B083
:1000C000ECB105F017FB05A907463046FCF790FA9E
:1000D0003B460821CDE90060684A20461BF0DFF965
:1000E00008212046059B664A1BF0D9F9F5B908217D
:1000F0002046644A1BF0D3F907B0BDE8F08F05F045
:10010000F9FA05A907463046FCF772FA3946034664
:1001100032465A4819F0B0FD0599594819F0ACFD1E
:10012000002D4BD1574819F0A7FDE5E708212046DF
:10013000554A1BF0B4F908212046544A1BF0AFF988
:1001400095F83D309A0740D4002C00F084800821B7
:1001500020464F4A1BF0A3F9082120464D4A1BF0C8
:100160009EF9002705F1580605EB471393F8602028
:10017000D3071BD536F8140C012817D1464BDFF8EE
:100180001C81C2F34002002A08BF9846A6F1100164
:10019000002C67D0D6E8AF9F06F0EEF84346CDE9D5
:1001A0000090082120463E4A1BF079F97B1C022B67
:1001B0004FF0010706F12006D6D19DE7324819F02D
:1001C0005BFD324819F058FDBAE72E88012EBBD1ED
:1001D00095F8280005F1140B05F1040905F1400A12
:1001E000ECB1FCF771F9074695F92900FCF778F9AD
:1001F0008046DBE8AFBF4946304606F0BDF85146C1
:100200008146304606F0B8F83B46CDE90290082119
:100210002046CDE9008B234A1BF041F994E7FCF717
:1002200053F9074695F92900FCF75AF98046DBE8AF
:10023000AFBF4946304606F09FF8514681463046EA
:1002400006F09AF85B46CDE90090424639461548DB
:1002500019F012FD78E70E4819F00EFD0D4819F05F
:100260000BFD7EE7D6E8AF9F06F086F84A460346C8
:1002700041460B4819F000FD98E700BF5C390400C7
:1002800088390400B8390400E2390400ED3904006B
:10029000263A0400343A0400633204005A3204005F
:1002A000483A04000F3A040010B5044650B1082142
:1002B000084A1BF0F4F808212046074A1BF0EFF823
:1002C000002010BD034819F0D7FC034819F0D4FCF6
:1002D000F6E700BF453B0400793B040013B5044634
:1002E000002862D008214F4B4F4A1BF0D8F8082154
:1002F00020464E4B4E4A1BF0D2F808212046494B6F
:100300004C4A1BF0CCF808212046464B4A4A1BF0C9
:10031000C6F808212046434B484A1BF0C0F8082184
:100320002046404B464A1BF0BAF8082120463D4B78
:10033000444A1BF0B4F8082120463C4B424A1BF0CB
:10034000AEF808212046394B404A1BF0A8F8082196
:1003500020463F4B3F4A1BF0A2F808212046334B72
:100360003D4A1BF09CF80123082120463B4A1BF024
:1003700096F8022308212046394A1BF090F80323FF
:1003800008212046374A1BF08AF80223082120461C
:10039000354A1BF084F800940024694633480194E0
:1003A00005F0AEFC204602B010BD1E491E4819F0F3
:1003B00063FC1E491E4819F05FFC1A491D4819F0DC
:1003C0005BFC18491C4819F057FC16491B4819F0EA
:1003D00053FC14491A4819F04FFC1249194819F0F6
:1003E0004BFC1249184819F047FC1049174819F0FE
:1003F00043FC1749174819F03FFC0C49164819F0FF
:100400003BFC0121154819F037FC0221144819F072
:1004100033FC0321134819F02FFC0221124819F074
:100420002BFCB8E724200400B73B04002C20040078
:10043000E73B0400173C0400473C0400773C040001
:10044000A73C0400D73C0400073D0400373D0400EE
:10045000673D0400793D040016370400A93D0400FF
:10046000EC3D04002F3E0400723E0400F50601003E
:100470002DE9F043032904468946904689B00BD004
:1004800030B10121444A1BF00AF86FF0150515E060
:10049000414819F0F1FBF8E75168FBF7D5FF071E5B
:1004A00077DB03F0B7FE064688B95CB13B464946A8
:1004B00020463A4A1AF0F3FF6FF00105284609B0CA
:1004C000BDE8F0833946354819F0D6FBF4E7D8F893
:1004D0000810022004AA05F065FF054668B1D8F8A7
:1004E00008302CB1012120462D4A1AF0D8FFCCE764
:1004F00019462B4819F0C0FBC7E79DF81030FF2BB9
:100500002FD1304604A909F051F8061ED6DA022090
:1005100004A9ACB105F030FF01210090CDE90176CE
:100520002046204B204A1AF0BAFF16F1860F05D15B
:10053000022120461D4B1E4A1AF0B1FF3546BDE789
:1005400005F01AFF3B46024616491748009619F077
:1005500093FB16F1860FF1D11449154819F08CFB65
:10056000ECE703464A46304604A905F01FF9002887
:10057000A4D1D8F8083034B1012120460D4A0096A4
:100580001AF08DFF9AE7324619460A4819F074FBB3
:1005900094E76FF0070591E7B53E04008E2A04004A
:1005A000453804008621040095380400E43E040028
:1005B000EC3E04001F3F04002DE9F04103290446EE
:1005C0000D46164688B00BD030B10121414A1AF0D1
:1005D00066FF6FF0150515E03E4819F04DFBF8E792
:1005E0005168FBF731FF071E70DB03F013FE8046F6
:1005F00088B95CB13B4629462046374A1AF04FFF7E
:100600006FF00105284608B0BDE8F0813946324850
:1006100019F032FBF4E7B168022004AA05F0C2FE2B
:10062000054660B1B3682CB1012120462B4A1AF06F
:1006300036FFCEE71946294819F01EFBC9E79DF899
:1006400010304046FF2B04A92DD108F0EBFF061E09
:10065000D8DA022004A9ACB105F08EFE0121009089
:10066000CDE9017620461E4B1E4A1AF018FF16F1FE
:10067000860F05D1022120461B4B1C4A1AF00FFFA2
:100680003546BFE705F078FE3B460246144915485B
:10069000009619F0F1FA16F1860FF1D112491348BC
:1006A00019F0EAFAECE71FF060FA0028AAD1B36863
:1006B0003CB1012120460E4A1AF0F1FE4FF0FF3501
:1006C000A0E719460A4819F0D7FAF7E76FF00705CF
:1006D00098E700BF493F04008E2A04004538040013
:1006E0009621040095380400783F0400EC3E040095
:1006F000473904002DE9F04F0C68074646688FB073
:10070000ECB104F0F7FF0AA905463846FBF770FF85
:100710002B460821CDE90070924A20461AF0BFFE10
:10072000082120460A9B904A1AF0B9FEF6B9082122
:1007300020468E4A1AF0B3FE0FB0BDE8F08F04F0E9
:10074000D9FF0AA905463846FBF752FF294603465A
:100750003A46844819F090FA0A99834819F08CFABD
:10076000002E5ED1814819F087FAE5E7082120467E
:100770007F4A1AF094FE082120467E4A1AF08FFE26
:100780004FF0000906F1140506EB891393F83D308C
:100790004FEA891B9A0703D535F8143C022B47D042
:1007A00009F10103022B4FF0010905F14005EBD1DE
:1007B000002C00F0C480082120466F4A1AF06FFE1A
:1007C000082120466D4A1AF06AFE002706F19405BA
:1007D00006EB471393F89C20D3071CD535F8140C6F
:1007E000022818D1664BDFF89C81C2F34002002A30
:1007F00008BF9846A5F11001002C00F0A780D5E8AD
:10080000AF9F05F0B9FD4346CDE900900821204691
:100810005D4A1AF044FE0137032F05F12005D7D1B8
:100820008AE7534819F028FA524819F025FAA7E741
:1008300029F067FB4FF47A7CA0FB0C0E002347F6EF
:1008400012220CFB01E1F0F753FE0146281D1FF0B8
:10085000C2FBA5F1100382461946384607931EF0E5
:100860005DFF00283BD090F82430079306EB0B0384
:1008700093F83D300DF12C0813F0010F31D04046B4
:100880004249F0F759FE287D94B3FBF71DFE09900D
:1008900095F91500FBF724FE8246D5E8AF3F089393
:1008A0000220A5F1100105F067FD06EB0B0292F89E
:1008B0003D20374912F0080F364A18BF0A46079BF9
:1008C0000592CDE90303089B0821CDE90183204669
:1008D000099B314ACDF800A01AF0E1FD60E78023C2
:1008E000C3E753460B2140462C4A17F0C3FBCAE727
:1008F000FBF7EAFD824695F91500FBF7F1FD09903B
:10090000D5E8AF3F08930220A5F1100105F034FDB2
:1009100006EB0B0191F83D101D4B11F0080F1D491E
:1009200018BF1946079B0391CDE90103089B514667
:100930000093099A4346184819F09EF930E70E488B
:1009400019F09AF90D4819F097F93EE7D5E8AF9FED
:1009500005F012FD4A46034641460B4819F08CF952
:1009600059E700BF8D3F040088390400B93F0400F7
:10097000E2390400E33F0400263A0400343A04005C
:10098000633204005A320400483A0400212804006B
:10099000803F0400EC670400144004007F11040051
:1009A00010B5044686B005AB04AA03A902A806F058
:1009B00001FF002C3BD04FF48073082120462E4AC3
:1009C0001AF06DFD082120462C4A1AF068FD082116
:1009D00020462B4A1AF063FD029B08215A692046E3
:1009E0000092284A1AF05BFD039B08215A692046B1
:1009F0000092254A1AF053FD049B0821DA8B204609
:100A00000092224A1AF04BFD059B0821DA8B204602
:100A100000921F4A1AF043FD1E4B0221009320460C
:100A20001D4B1E4A1AF03BFD002006B010BD4FF4CE
:100A30008071114819F020F9104819F01DF910487B
:100A400019F01AF902990F484A6919F015F9039932
:100A50000D484A6919F010F904990C48CA8B19F02D
:100A60000BF905990A48CA8B19F006F9094A0A498F
:100A70000A4819F001F9D7E75B4104007541040009
:100A80008C410400A1410400AB410400B5410400C5
:100A9000C4410400ED410400D341040005130400E7
:100AA000002337B5CB604B600E4B0D4604468B6080
:100AB00088B901464FF4B8720B4829F08BFC0B48FB
:100AC00001A9019407F04AFF2E235C43064A13193B
:100AD000125D1AB901E00728F6D900232B6003B094
:100AE00030BD00BFF4BF030035810020F10A0100D2
:100AF00038B50D680C46072D0FDC816802201C31CB
:100B000005F03AFC2E2103460448054A01FB050086
:100B100017F0B0FA23680133236038BD3581002017
:100B200068F903001FB500230446CDE9013002A98E
:100B300001AB0948039307F011FF019B2BB93CB1AE
:100B400008212046054A1AF0AAFC002004B010BD76
:100B5000024819F091F8F8E7090C01002E42040050
:100B600030B551680446154685B059B930B10321F6
:100B7000214A1AF094FC6FF0070033E01E4819F088
:100B80007BF8F8E702206A4605F00CFC00280CDA36
:100B90006B682CB1194A032120461AF080FCEAE761
:100BA0001946164819F068F8E5E76946002007F08D
:100BB000E1FE694658B9022024B105F0DDFB104A78
:100BC0000346E8E705F0D8FB01460D48EAE70220B6
:100BD00054B105F0D1FB082103460A4A20461AF019
:100BE0005EFC002005B030BD05F0C6FB014605489F
:100BF00019F042F8F5E700BF3D4204005D420400F1
:100C0000704204008B4204002DE9F04FD1E90068E6
:100C1000D8F80030044691B03BB9002E7DD00821B1
:100C20003046604B604A1AF03AFCD8F80030DFF8E2
:100C300074910133C8F80030A36893F8480007F0B6
:100C400081FE0D90F0F780FC584BA268052818BF74
:100C50004B46D2E90C570C93936B5D1947EBE37746
:100C600029F04FF94FF47A7CA0FB0C0ED8F8003035
:100C700047F612220E930CFB01E10023F0F738FC3B
:100C80002D1AD4F8048067EB0107002FB8BF0025A8
:100C90004046002E48D004F02DFDA3680F906078E8
:100CA00093F84D80FF28B3F84A9094F800A093F889
:100CB0004CB008F0010835D007F00CFD074660780D
:100CC00007F008FD18234178394AB81C05F030FABE
:100CD00007466078FF2801D007F0FCFCA1680220DD
:100CE0001C3105F049FB2F4B0B90CDE909730C9B90
:100CF000082107930D9B3046CDE905830F9BCDE975
:100D000003ABCDE900432B4A0E9B0895CDF8089024
:100D10001AF0C5FB11B0BDE8F08F2249224818F047
:100D2000ABFF82E7244FD4E704F0E4FCA3680F9004
:100D3000607893F84D80FF28B3F84A7094F800A0CB
:100D400093F84CB008F0010829D007F0C3FC064620
:100D5000607807F0BFFC18234178154AB01C05F0F5
:100D6000E7F906466078FF2801D007F0B3FCA168D8
:100D700002201C3105F000FB0C9BCDE90890059387
:100D80000D9B2246CDE90383CDE90656CDE901ABA3
:100D90000F9B0E990748009718F06EFFBAE7064EB2
:100DA000E0E700BFEC670400A6420400A142040093
:100DB0001D810020F84204004F2804002DE9F34172
:100DC0000446303005F0D4FF0022206E11461AF0A0
:100DD000B6FB206E00283FD00821294A1AF05FFB9D
:100DE000D4E9221200293BD091423BD964208B1ACE
:100DF0004343B3FBF1F3206EB0B3CDE900230B46C0
:100E0000204A08211AF04BFBD4F890200AB3D4E909
:100E1000200100234FF47A78F0F76AFBD4F894505D
:100E2000D4F8983008FB05F508FB00F208FB03F343
:100E3000154F266EB5FBF7F5B2FBF7F2B3FBF7F3F0
:100E4000B6B1CDE9002308212B4630460F4A1AF0EF
:100E500026FB02B0BDE8F081094818F00DFFBFE79E
:100E60006423C8E70023C6E7064818F005FFCBE770
:100E70002946064802B0BDE8F04118F0FDBE00BFAB
:100E8000694304008243040040420F00B943040058
:100E900010B5044628F0ABFC2046FFF78FFF206E0C
:100EA0000821BDE81040014A1AF0F9BAEC670400C5
:100EB00073B5036852F823409D00A67896B10234BA
:100EC0000E490222204629F0DFFA0023002814BF31
:100ED0000A211021204601AA0193F5F735F8019B5C
:100EE0002BB102E001338B4203D34FF0FF3002B04D
:100EF00070BD03602A445468E2E700BFD843040091
:100F000008B50A44914200D108BD11F8013B032BFA
:100F1000F8D1044828F06BFCBDE808400148FFF711
:100F20004DBF00BF483F00202DE9F04704460D4665
:100F300000218CB00DF120081646404610221F46B5
:100F40000791DDF850909DF854A029F043FA20460F
:100F500020F047FD032836D9204607A920F0E3FCFE
:100F600000285FD127F012FD2F4C079BC01A94F880
:100F70007730079053B94FF47A7358432B4B1021B5
:100F8000B0FBF3F32A4A404617F074F8D4F89030D7
:100F9000079A0133C4F89030D4E920319B1841F10D
:100FA0000001C4E92031D4F89430934294BFC4F8CE
:100FB0009430C4F89420D4F8983093422CBFC4F8ED
:100FC0009830C4F89820184CD4F88C300133C4F809
:100FD0008C3094F877307BB9206E8DF8183006ABE2
:100FE00088B1CDE9043808213346CDE9025ACDE96C
:100FF0000079104A1AF053FA636E9D420ED0002019
:101000000CB0BDE8F087CDE902383A464B46314690
:10101000CDE9005A074818F02FFEEDE70248FFF728
:1010200037FFECE70220EBE7483F002040420F008B
:10103000DB430400E64304002DE9FF410D46002395
:101040000426284602A9CDE90236176820F0D7FD0C
:101050000446B8B303881D4A5BBAB2F86C109BB261
:1010600099422FD14388126F5BBA9BB2934229D128
:101070003146284620F02CFC002825DBB5F842300C
:1010800066887C88C3F57F43FC3307F10C0101209F
:1010900064BA13FA84F405F06FF907F11001804681
:1010A000012005F069F976BA3B7AB6B2A4B2CDE96F
:1010B00000032246434631462846FFF735FF04B079
:1010C000BDE8F0810120FAE70220F8E7483F002060
:1010D0002DE9FF410D4600230426284602A9CDE94B
:1010E0000236176820F08BFD0446B8B303881D4A0A
:1010F0005BBAB2F86C109BB299422FD14388126F41
:101100005BBA9BB2934229D13146284620F0E0FBDE
:10111000002825DBB5F842306688BC88C3F57F43DC
:10112000FC3307F10801022064BA13FA84F405F0D5
:1011300023F907F118018046022005F01DF976BA5F
:10114000FB79B6B2A4B2CDE900032246434631464C
:101150002846FFF7E9FE04B0BDE8F0810120FAE778
:101160000220F8E7483F002070B50446056E88B0BD
:10117000022103A81BF07CFABDF80C30626EA4F8C3
:101180006C30236F01339342236712D994F8773080
:101190002BB955B1022128462D4A1AF080F9204674
:1011A00008B0BDE87040FFF773BE294818F064FD31
:1011B000F5E743D247F6122C40F2E7300021A66E45
:1011C0004FF47A720023E6FB0C01F0F791F9024626
:1011D0000B46204615F0E6FBD4F8883004F14402B3
:1011E0000133C4F88830B4F86C3004F13000ADF845
:1011F0000C30236FADF80E3094F876308DF8103047
:10120000A36F059300230693B4F8743000940793FA
:10121000E16D03AB1FF0A6F9034668B195B1032158
:1012200028460C4A1AF03BF9D4F888302046013B96
:10123000C4F88830FFF72CFE08B070BD4FF224428E
:101240000023C6E70146034818F016FDECE700BF8F
:1012500017440400254404002DE9F04F4FF0000B23
:101260000D4690464FF47A7103224FF0FF37044643
:1012700001234FF00409DA465E4689B0CDE9032127
:101280000597AB4207930BD3002E40F09180002CC2
:1012900000F08A8003212046984A1AF000F941E0C4
:1012A00058F8233019782D2979D15878732807D820
:1012B000682809D8512858D0632821D049283CD023
:1012C000002C69D08E4A29E069380A28F8D801A193
:1012D00051F820F02B130100C1120100C1120100CE
:1012E000C1120100C1120100C1120100C1120100AE
:1012F00059130100A3130100C11201007B13010067
:101300004246294607A8FFF7D3FD031E039320DAC0
:10131000079B58F82330002C39D07A4A0321204605
:101320001AF0BDF86FF007007EE04246294607A894
:10133000FFF7BEFD031E0493E9E74246294607A8CE
:10134000FFF7B6FD031E0593E2DB02F063FF002802
:10135000DED0079B013394E74246294607A8FFF7F2
:10136000A7FD0746FF28F4D9D2E74246294607A839
:10137000FFF79EFD8246FF28F5E74246294607A86B
:10138000FFF796FDB0F5803F8146E2D3C0E71946EE
:101390005C4818F071FCC5E719465948F9E71E4644
:1013A000D7E74FF0010BD4E7544818F065FCB9E7D4
:1013B000554DA0220021284629F00CF82846534913
:1013C00028F007FA039B20226B66049B002105F19D
:1013D0008000AB662C66AF6785F876A0A5F87490A0
:1013E00028F0F8FF4FF0FF3385F877B0C5F8943058
:1013F0000220314605F1480204F0D4FF0346D8B973
:101400000221434AA5F8441005F1300000928122E0
:1014100005F07AFC002833DA4CB13E4B032120461C
:101420003D4A1AF03CF8002009B0BDE8F08F394978
:10143000394818F021FCF6E70120314605F1480251
:1014400004F0B0FF034680B90121344AA5F84410E6
:101450000092024605F1300005F056FC00280FDA34
:101460000CB12F4BDAE72E49E2E72CB103212046DD
:101470002C4A1AF014F8D6E72A4818F0FDFBD2E7F8
:10148000059802F0C7FE0346C0B9B5F84420012A0A
:1014900008D125481EF0CDFA034678B902F044FF82
:1014A00003460BE0022A09D11F481EF05BFA0346EF
:1014B00020B91D4922F012F898B14368EB65BCB120
:1014C000334608212046194A19F0E9FF2046002238
:1014D00017491AF034F8002200230B4815F062FA7D
:1014E000A1E711490AF0CEF90028D7D04368E5E713
:1014F00031460E4818F0C0FBE8E700BF6F44040017
:101500005444040043440400483F00206911010092
:10151000D1100100F32D04008444040039100100AF
:101520007E1C0400AB440400903F0020BF44040034
:10153000010F01002DE9F041556804462B7817464C
:10154000302B86B003D16B78782B08BF0235284644
:10155000EFF7FAFF0DF1140801460423424628462E
:1015600018F01BFE28B100231E46013800280ADAB5
:10157000AEB97B6874B1644A0121204619F08FFF2F
:101580006FF0070044E018F8002001389A40164335
:101590000833EBE719465C4818F06EFBF0E70023D0
:1015A000414604A81A4606F005F9314604981CF095
:1015B000C8FA58B9314605981CF0C3FA30B97B68AF
:1015C0000CB1524AD8E719465048E5E7B56806F12C
:1015D000240704B33346082120464D4A19F05FFF23
:1015E000D7E8AF3F0821009320463346494A19F017
:1015F00056FF15BB08212046474A19F050FF082125
:101600002046454A19F04BFFB568002D54D1002003
:1016100006B0BDE8F08131463D4818F02DFBD7E813
:10162000AF2F3C48314618F027FB2DBB3A4818F045
:1016300023FB394818F020FBE6E708212046374A0B
:1016400019F02DFFADB12CB3D7E8AF1F6B8A039310
:101650006869EA68121A9B1A9BB202932B8A204689
:10166000CDE900132E4A2B46082119F018FF6D68AA
:1016700035B9002CBED1D9E7284818F0FDFAE1E7CA
:101680002CB108212046254A19F009FFDBE7234841
:1016900018F0F2FAD7E8AF2F698AB5F810C00191B7
:1016A0006B69E868C01A091A89B200916346294635
:1016B0001B4818F0E1FADAE72B7A002BA7D0C4B167
:1016C000334608212046174A19F0E9FE0026334622
:1016D00001369CB108212046134A009519F0DFFE1F
:1016E0002A8AE96820461AF073F96D68002DEED158
:1016F0008DE731460B4818F0BFFAE7E72A4619464E
:10170000094818F0B9FAEBE780450400AD4504003C
:10171000D9450400F34504009EF60300FB45040090
:10172000FE450400114604003346040007B550B1DD
:10173000084B02210093084A084B19F0B0FE002024
:1017400003B05DF804FB034A0449034818F094FA17
:10175000F5E700BFA1460400051304008B46040012
:1017600007B548B1084B02210093084A084B19F00D
:1017700096FE03B05DF804FB034A0549034803B035
:101780005DF804EB18F078BA134704000513040061
:10179000EB46040007B550B1084B02210093084AFC
:1017A000084B19F07CFE002003B05DF804FB034AEF
:1017B0000449034818F060FAF5E700BFC447040085
:1017C000051304006347040007B550B1084B02211C
:1017D0000093084A084B19F062FE002003B05DF840
:1017E00004FB034A0449034818F046FAF5E700BF32
:1017F000C4470400051304008847040008B528B155
:101800000221044A19F04BFE002008BD014818F0DF
:1018100033FAF9E7EC4704002DE9F04116461822A7
:101820000D468CB0044600210DEB020028F0D2FDDD
:10183000022D0ED04CB1012120468D4A19F02FFE09
:101840006FF015000CB0BDE8F081894818F014FA6B
:10185000F6E775682846EFF777FE06AA01462846A0
:101860001EF03EFE60B973682CB10121814A20460A
:1018700019F015FEE4E719467E4818F0FDF9DFE798
:10188000BDF81830022B43D107A81EF06BF80546AF
:1018900070B973683CB101212046774A19F0FFFD09
:1018A0006FF00700CEE71946734818F0E5F9F7E73F
:1018B00007A909F0E7FF0746002840F0B580BDF80A
:1018C0001880B8F1010F60D1014607A81EF094F806
:1018D000002844D128461EF0D7F8059004F0A0FE59
:1018E000059B026876689A4227D0404605A9B4B1A4
:1018F00004F042FD0746284603F0FCFECDE90170E6
:101900005E4B0096082120465D4A19F0C8FD33E081
:1019100014B108215B4AAAE719465A48ADE704F01A
:101920002BFD0446284603F0E5FE23463246534984
:101930000090534818F0A0F91EE0284634B103F097
:10194000D9FECDE900604D4B4F4A11E003F0D2FEC5
:101950003246034649494C4818F08EF90CE02846B7
:1019600076685CB103F0C6FECDE90060434B474AA0
:101970000821204619F093FD002063E703F0BAFE2A
:10198000324603463D494148E6E7B8F1020F40D1EF
:10199000014607A81DF0D4FD60BB07A91DF030FF6C
:1019A0007668C8B100F10801022054B104F0E4FCEB
:1019B0000746284603F09EFECDE90170344B0096A1
:1019C000A0E704F0D9FC0446284603F093FE234622
:1019D00032462F490090ACE728462CB103F08AFE2E
:1019E0002B4BCDE90060AFE703F084FE324603469F
:1019F0002749B0E7284676682CB103F07BFE244BDC
:101A0000CDE90060B3E703F075FE32460346204996
:101A1000B9E72CB1012120461E4A19F040FD3FE7ED
:101A20001C4818F029F93BE7058B022D1AD109F063
:101A300085FF7668014664B148B1284604F09CFCF5
:101A40000546786803F056FECDE90150B6E7124D21
:101A5000F7E728B1284604F08FFC04467868B4E71D
:101A60000D4CFBE70CB12B4653E7294655E700BF69
:101A70004948040077480400904804007E1C040094
:101A8000D1480400B8480400FA4804001E49040084
:101A9000F32D04004E4904003F4804001FB50446DE
:101AA000029002A90A4804F02BF954B1094B022113
:101AB00000932046084B094A19F0F1FC002004B0BD
:101AC00010BD044A0449054818F0D6F8F6E700BFEF
:101AD000E11A010079490400634904000513040078
:101AE000F0B50D46044685B008B30E6803680C33A4
:101AF000D3E8AF3F1B061AD5DEB103F0FBFD03A907
:101B000007462046FAF774FD3B460821CDE9004020
:101B1000114A304619F0C3FC08213046039B0F4A96
:101B200019F0BDFC29460E486C6009F017FF05B09E
:101B3000F0BD03F0DFFD03A906462046FAF758FD85
:101B4000314603462246044818F096F803990348A4
:101B500018F092F8E6E700BF874904008B390400CB
:101B6000411D0100F0B50429044616468FB00BD084
:101B700030B101213A4A19F092FC6FF0150515E0D9
:101B8000374818F079F8F8E75168FAF75DFC051E58
:101B90000ADB02F03FFB074680B954B12B46032114
:101BA0002046304A19F07BFC6FF0070528460FB03D
:101BB000F0BD29462B4818F05FF8F5E7B5682846D0
:101BC000EFF7C2FC0DF10F03014608AA284604F006
:101BD000C3FC60B9B3682CB1234A0121204619F037
:101BE0005EFCCAE71946204818F046F8C5E7BDF87C
:101BF0002050022D27D1102200210DEB020028F0E9
:101C0000E9FBF168284604AA04F0CCFB054630B194
:101C1000F3680CB1154AE0E719461448E4E74FF0C1
:101C2000FF330190009338469DF80F2004AB09A9BB
:101C300009F038FE0028B9D16CB1012120460C4AC8
:101C400019F02DFCB0E71CB12B460821094AC5E765
:101C500029460848C8E7064818F00EF8A4E700BF70
:101C6000B04904008E2A040077480400EE490400BD
:101C7000034A0400B84804002DE9F0410329044652
:101C80008846154688B00BD030B10121284A19F09A
:101C900006FC6FF015001AE0254817F0EDFFF8E795
:101CA0005168FAF7D1FB061E0FDB02F0B3FA0746C4
:101CB00080B934B1334641461E4A204619F0EFFB45
:101CC00003E031461B4817F0D7FF6FF0070008B05C
:101CD000BDE8F081AE683046EFF736FC0DF1070342
:101CE000014602AA304604F037FC60B9AB682CB15B
:101CF00001212046104A19F0D2FBCAE719460E48C6
:101D000017F0BAFFC5E7BDF80830022B08D13846F6
:101D100003A909F0B7FD18B109F0FAFD0020D6E7D4
:101D2000AB6814B10121054AC7E719460348CAE761
:101D3000184A04008E2A0400774804004C4A040024
:101D40002DE9F0430546D1E9004687B028F0D9F8DF
:101D50006B680746B34289463ED1288B022840F083
:101D6000948005F11C01002C39D004F005FB95F896
:101D7000402003460092082120464C4A19F08FFB70
:101D8000284609F0DBFD0646284623F0AFFC95F80F
:101D9000413080465B072BD5454902A8EFF7CCFBC5
:101DA000002C52D0002E3AD03146022004F0E4FA42
:101DB0000346082120463F4A19F071FBB8F1000F95
:101DC0002FD1082120463C4A19F069FB0821204602
:101DD0003A4A02AB19F063FB07B0BDE8F08304F0A8
:101DE000CBFA95F840200146304817F045FFC7E789
:101DF0004FF47A71A7FB010747F61222002301FB7B
:101E00000971EFF775FB014605F108001EF0E3F8D4
:101E10000F2103462A4A02A816F02CF9C0E7294BE5
:101E2000C7E798F80100FF282CD006F053FC1823D0
:101E30004178254A0230D4B104F07AF908210346EA
:101E4000224A204619F02BFBC0E776B1314602202A
:101E500004F092FA0146174817F00EFFB8F1000F90
:101E6000DFD1154817F008FF07E01649F3E704F043
:101E70005FF90146154817F0FFFE104802A917F058
:101E8000FBFEA9E7002C9CD1EBE744B103460821F7
:101E900020460F4A07B0BDE8F04319F000BB0146E9
:101EA0000B4807B0BDE8F04317F0E6BE704A0400E7
:101EB000212804008C4A04009C4A0400BF4A040004
:101EC000854A0400664A0400A5820020B14A040045
:101ED000B8480400002310B586B0CDE9033003AB49
:101EE0000446059300282FD008212F4A19F0D7FA6D
:101EF0002E4B082101932E4B20462E4A00932E4B49
:101F000019F0CDFA082120462C4A19F0C8FA2C48BD
:101F100004A9FAF71BF9039B002B2ED10CB308215F
:101F20002046284A19F0BBFA08212046234A19F016
:101F3000B6FA254B022100932046244B244A19F07F
:101F4000AEFA002006B010BD174817F095FE174BEB
:101F5000174A1949174817F08FFE184817F08CFEDA
:101F6000D5E7184817F088FE144817F085FE164A82
:101F70001649174817F080FEE3E75CB11549164A89
:101F80002046012B08BF0A4608210092134A19F087
:101F900086FAC9E710490F4A1048012B18BF0A46B4
:101FA000194617F069FEDFE79B4B0400BB4B0400AA
:101FB000BF4B0400AC4B0400A64B04009EF603008C
:101FC000E11F0100C54B04002D4C0400FD4B040033
:101FD00005130400EC67040069F90300E04B0400FA
:101FE0002DE9F3470026D1E90087054634464FF036
:101FF0001409DFF870A06B68B3421FDC002CC4BF6B
:102000000022184B1849C8BF1B191848C8BF03F84D
